:100000000C9464170C9495170C9495170C949517F1
:100010000C9495170C9495170C9495170C949517B0
:100020000C9495170C9495170C9495170C949517A0
:100030000C9495170C94A4620C9495170C94951736
:100040000C9495170C9474CD0C9495170C949517EB
:100050000C9495170C9495170C9413590C945A62A0
:100060000C9495170C94DC3E0C9495170C949517F2
:100070000C9495170C9495170C9495170C94951750
:100080000C9495170C9495170C9495170C94951740
:100090000C9495170C9495170C9495170C94951730
:1000A0000C9495170C9495170C9495170C94951720
:1000B0000C9495170C9495170C9495170C94951710
:1000C0000C9495170C9495170C9495170C94951700
:1000D0000C9495170C9495170C940B4C0C94CC4BDA
:1000E0000C949517672F842FB52FD22FE72F103040
:1000F0007D30E3308C31253633362C366536693623
:1001000083360F3B9836E4360B3732375B37B137DF
:10011000C237D637E737F83709380F3B1A3A0F3B63
:10012000253A953A9B3ABB3A0F3F153F263F313F60
:10013000393F4E3F3D3F4E3F413F453F4E3F4B3F96
:10014000AEB4B1B4A0B4A4B4AAB4E8B4B5B4B9B46C
:10015000BFB4C3B4C7B4CDB4D1B4D5B4E8B4DBB480
:10016000DFB4E3B4C4BAC9BACEBAD8BAE2BA5BBB98
:10017000ECBAF4BAFCBA06BB10BB1ABB29BB33BB42
:100180005BBB3DBB47BB51BB084AD73B3BCE016E77
:1001900084BCBFFDC12F3D6C74319ABD56833DDADE
:1001A0003D00C77F11BED9E4BB4C3E916BAAAABEED
:1001B000000000803F05A84CCDB2D44EB93836A916
:1001C000020C50B9918688083CA6AAAA2ABE000053
:1001D00000803F004E414E494E495459494E46CD4C
:1001E000CCCC3D0AD7233C17B7D13877CC2B3295EE
:1001F00095E6241FB14F0A000020410000C84200CC
:10020000401C4620BCBE4CCA1B0E5AAEC59D744352
:100210004F4D4D554E49434154494F4E004452595C
:1002200052554E004552524F525300494E464F00D0
:100230004543484F0047322F4733206261642070A6
:100240006172616D65746572730A00206F662000CB
:100250004D424C2047323920706F696E742000295E
:100260000A0059206F7574206F662072616E676591
:100270002028312D00290A0058206F7574206F66E0
:100280002072616E67652028312D004D65736820EE
:1002900070726F62696E6720646F6E652E0A00531C
:1002A00074617274206D6573682070726F62696E1C
:1002B0006720776974682022473239205331222021
:1002C00066697273742E0A004732380A4732392041
:1002D00053320053746174653A20004D6573682091
:1002E000626564206C6576656C696E672068617311
:1002F000206E6F20646174612E0A0053206F757444
:10030000206F662072616E67652028302D35292E9A
:100310000A004D65736820706F696E742063616EAA
:100320006E6F74206265207265736F6C7665640A07
:1003300000456E642066696C65206C6973740A0000
:10034000426567696E2066696C65206C6973740A22
:10035000004D31323500286E6F2066696C652900CA
:100360005344207072696E74696E67206279746597
:1003700020004E6F74205344207072696E74696E51
:10038000670A0043757272656E742066696C653A1F
:10039000200046696C652064656C657465643A008C
:1003A00044656C6574696F6E206661696C65642C68
:1003B0002046696C653A20005072696E7420746939
:1003C0006D653A20006F6E2E0A006F66662E0A0079
:1003D000473236204465627567200030022B0224C4
:1003E000021D020F026F66660044454255473A00FF
:1003F0004D3131332053006F6B002C20002C200036
:10040000544845524D414C5F50524F544543544916
:100410004F4E004155544F5245504F52545F534434
:100420005F53544154555300454D455247454E4343
:10043000595F50415253455200434153455F4C4927
:100440004748545F4252494748544E45535300541D
:100450004F47474C455F4C494748545300534F461C
:1004600054574152455F504F574552004255494CF1
:10047000445F50455243454E54004C4556454C4907
:100480004E475F44415441005A5F50524F4245002D
:100490004155544F4C4556454C005052494E545FBF
:1004A0004A4F420050524F47524553530041555412
:1004B0004F5245504F52545F54454D5000564F4C8B
:1004C000554D455452494300454550524F4D0053F8
:1004D000455249414C5F584F4E5F584F4646004683
:1004E00049524D574152455F4E414D453A4D61721B
:1004F0006C696E20312E312E392028476974687559
:10050000622C20646176696472616D69726F292062
:10051000534F555243455F434F44455F55524C3A04
:1005200068747470733A2F2F6769746875622E63EC
:100530006F6D2F4D61726C696E4669726D77617275
:10054000652F4D61726C696E2050524F544F434F6E
:100550004C5F56455253494F4E3A312E30204D4153
:100560004348494E455F545950453A416E79637549
:10057000626963206933204D656761204558545294
:10058000554445525F434F554E543A3120555549D5
:10059000443A63656465326132662D343161322DCF
:1005A000343734382D396231322D63353563363284
:1005B0006633363766660A002F2F2000205400204D
:1005C0005200416363656C65726174696F6E3A20B5
:1005D00050005741524E494E4721204C6F77205AC8
:1005E000204A65726B206D6179206C6561642074AE
:1005F0006F20756E77616E746564207061757365C8
:10060000732E0A00546F6F206661722066726F6DE0
:10061000207265666572656E636520706F696E74C1
:100620000A0020466C6F773A200000013637260317
:100630002BFFFFFF3C3D382AFFFFFFFF2E303E120D
:10064000FFFFFFFFFFFFFF0809FF2C071A1C18FF21
:10065000FFFF08440A2C4324221E20643A0020692C
:100660003A0020703A00496E76616C6964206578C2
:100670007472756465720A0043290A0061626C65D0
:100680006420286D696E2074656D702000436F6C66
:1006900064206578747275646573206172652000EA
:1006A00020643A0020693A0020703A004E6F2063BF
:1006B000617365206C696768740A00454550524F44
:1006C0004D204F4B0A00205A004475616C20456E46
:1006D0006473746F702041646A7573746D656E74B1
:1006E00020286D6D293A20003F4B2076616C75659E
:1006F000206F7574206F662072616E6765202830E8
:100700002D3130292E0A00416476616E6365204BDD
:100710003D0041637469766520457874727564653F
:10072000723A2000496E76616C6964206578747253
:10073000756465720A0043616E6E6F7420656E7435
:100740006572207375626469723A20004D313038E9
:10075000005370656369616C204D656E753A204D7C
:1007600031303820526573756D650A004D36303072
:10077000005370656369616C204D656E753A204D5C
:100780003630302050617573650A004739310A47A9
:1007900031205A2D302E310A4739300053706563AD
:1007A00069616C204D656E753A205A20446F776EF2
:1007B00020302E310A004739310A4731205A2D3076
:1007C0002E30320A473930005370656369616C20FE
:1007D0004D656E753A205A20446F776E20302E306A
:1007E000320A004739310A4731205A2B302E303235
:1007F0000A473930005370656369616C204D656E3E
:10080000753A205A20557020302E30320A00473970
:10081000310A4731205A2B302E310A4739300053E4
:1008200070656369616C204D656E753A205A20557C
:100830007020302E310A0047323920533200537075
:10084000656369616C204D656E753A204E657874FC
:10085000204D65736820506F696E740A0047323905
:10086000205331005370656369616C204D656E756E
:100870003A205374617274204D657368204C65761C
:10088000656C696E670A004D313430205336300094
:100890005370656369616C204D656E753A205072C6
:1008A0006568656174204265640A004D3530320028
:1008B0005370656369616C204D656E753A204C6FAD
:1008C00061642046572044656661756C74730A0044
:1008D0004D353030005370656369616C204D656E35
:1008E000753A205361766520454550524F4D0A00B8
:1008F0004D33303320452D312053363020433620C0
:100900005531005370656369616C204D656E753AB1
:10091000204175746F2054756E6520486F74626550
:1009200064205069640A004D31303620533230342F
:100930000A4D333033204530205332313020433696
:10094000205531005370656369616C204D656E758B
:100950003A204175746F2054756E6520486F746538
:100960006E64205049440A003C5370656369616CB1
:100970005F4D656E753E003C5370656369616C5FE9
:100980004D656E753E002F002F002F002F2E2E0A72
:10099000002F2E2E002F2E2E003C537065636961B0
:1009A0006C5F4D656E753E0A003C5370656369610E
:1009B0006C204D656E753E003C5370656369616CDB
:1009C000204D656E753E003C4D31303820526573C8
:1009D000756D653E003C4D31303820526573756D44
:1009E000653E003C4D3630302050617573653E00E9
:1009F0003C4D3630302050617573653E003C4C6F85
:100A000061642046572044656661756C74733E00CE
:100A10003C4C6F61642046572044656661756C7478
:100A2000733E003C4175746F2054756E6520486FAD
:100A300074626564205049443E003C4175746F20E7
:100A400054756E6520486F74626564205049443E59
:100A5000003C4175746F2054756E6520486F746555
:100A60006E64205049443E003C4175746F205475BB
:100A70006E6520486F74656E64205049443E003CAA
:100A8000457869743E003C457869743E003C53618A
:100A9000766520454550524F4D3E003C536176658A
:100AA00020454550524F4D3E003C4E657874204DD8
:100AB00065736820506F696E743E003C4E657874B3
:100AC000204D65736820506F696E743E003C53740E
:100AD000617274204D657368204C6576656C696E33
:100AE000673E003C5374617274204D657368204CFE
:100AF0006576656C696E673E003C5072656865613D
:100B000074206265643E003C5072656865617420C3
:100B10006265643E003C5A20446F776E20302E316F
:100B20003E003C5A20446F776E20302E313E003C10
:100B30005A20446F776E20302E30323E003C5A20CF
:100B4000446F776E20302E30323E003C5A20557074
:100B500020302E30323E003C5A20557020302E304E
:100B6000323E003C5A20557020302E313E003C5A17
:100B700020557020302E313E0056313136004A3338
:100B80003320004D3530300A4D3432302053310A95
:100B90004731205A313020463234300A473120580C
:100BA00030205930204636303030004A3232004A48
:100BB0003232004731205A3520463234300A47312C
:100BC0002058313930205932302046363030300A02
:100BD0004731205A302046323430004731205A35D0
:100BE00020463234300A47312058313930205931CB
:100BF00039302046363030300A4731205A302046CE
:100C0000323430004731205A3520463234300A47DA
:100C1000312058313930205932302046363030308A
:100C20000A4731205A302046323430004739310AE1
:100C30004731205A313020463234300A4739300AA1
:100C40004732380A4732390A473120583230205962
:100C500032302046363030300A4731205A30204674
:100C6000323430004A3032004A3132004731205AA3
:100C70003130004F4B004731205A31300047393076
:100C80000047312045256946353030004731204541
:100C90002D302E314625690047312045302E314612
:100CA0002569004731205A256946256900473120CA
:100CB0005A2D302E31462569004731205A302E31C9
:100CC0004625690047312059256946256900473185
:100CD00020592D302E314625690047312059302EBC
:100CE0003146256900473120582569462569004766
:100CF0003120582D302E314625690047312058309B
:100D00002E314625690047393100473238004732D5
:100D100038205A00473238205900473238205800CE
:100D20004132305620004731205A3130004A3034A9
:100D3000004A3231004A3230004B494C4C45442E77
:100D400020004A303400454E4400464E20004A30D0
:100D500032003939393A393939004D0048004137C4
:100D6000562000413656202D2D2D004A30320041AC
:100D7000365620005A3A2000593A2000583A2000AE
:100D8000413556004134562000413356200041324F
:100D9000562000413156200041305620004D383455
:100DA00000473930004731205A3120463234300074
:100DB00047393100473930004731205A3520463213
:100DC00034300047393100473930004731205A313B
:100DD000302046323430004739310047393000473F
:100DE00031205A3130204632343000473931004A00
:100DF0003136004A3138004A3134004A3030004A36
:100E00003031004A313000696E206D6F76655F7455
:100E10006F282920666565645F76616C756520665C
:100E20006F722058593A002C2065793D0029202DF9
:100E30003E202865783D002C2073793D0020436FCB
:100E40006E6E656374696E67207769746820766575
:100E500072746963616C206C696E65202873783DDB
:100E6000002C2065793D0029202D3E202865783D05
:100E7000002C2073793D0020436F6E6E65637469AA
:100E80006E67207769746820686F72697A6F6E7414
:100E9000616C206C696E65202873783D003F53704B
:100EA0006563696669656420582C5920636F6F72A9
:100EB00064696E617465206F7574206F6620626F5F
:100EC000756E64732E0A003F28522965706561743F
:100ED0002076616C7565206E6F7420706C6175731F
:100EE00069626C653B206D75737420626520617466
:100EF000206C6561737420312E0A003F28522965E9
:100F000070656174206D75737420626520737065FF
:100F1000636966696564207768656E206E6F74200A
:100F20007573696E6720616E204C43442E0A003F42
:100F3000537065636966696564206E6F7A7A6C6563
:100F40002074656D7065726174757265206E6F7462
:100F500020706C61757369626C652E0A003F537076
:100F6000656369666965642066696C616D656E7448
:100F70002073697A65206E6F7420706C6175736977
:100F8000626C652E0A003F5370656369666965642B
:100F9000207072696D65206C656E677468206E6F75
:100FA0007420706C61757369626C652E0A003F5025
:100FB00072696D65206C656E677468206D757374F9
:100FC000206265207370656369666965642077686F
:100FD000656E206E6F74207573696E6720616E2078
:100FE0004C43442E0A003F5370656369666965642B
:100FF000206E6F7A7A6C652073697A65206E6F74E3
:1010000020706C61757369626C652E0A003F5370C5
:1010100065636966696564205265747261637469A9
:101020006F6E204D756C7469706C696572206E6F9F
:101030007420706C61757369626C652E0A003F5292
:10104000657472616374696F6E204D756C7469703C
:101050006C696572206D75737420626520737065AC
:101060006369666965642E0A003F5370656369664B
:10107000696564206C617965722068656967687468
:10108000206E6F7420706C61757369626C652E0AD6
:10109000003F53706563696669656420626564201A
:1010A00074656D7065726174757265206E6F742001
:1010B000706C61757369626C65202834302D313431
:1010C0003043292E0A0047323620636F6D6D616E02
:1010D0006420737461727465642E20576169746949
:1010E0006E6720666F722068656174657228732967
:1010F0002E0A0024F4D43050C38E20C2A24017829E
:101100008B7011127A910D816CD90AA861E108C720
:10111000586607615143061E4B5D05C145A7041A79
:10112000411104093D9803713931034036DB0265F2
:10113000339102D4305402802E1D02632CEE0175CF
:101140002AC501B028A001102781018F2564012B39
:10115000244B01E0223401AC211F018D200D0180C0
:101160001FFC00841EED00971DDF00B81CD200E6B6
:101170001BC600201BBC00641AB200B219A8000AEA
:1011800019A0006A189900D117910040178B00B57B
:1011900016840031167E00B31579003A157300C726
:1011A000146F0058146A00EE13660088136300255C
:1011B000135E00C7125B006C12570015125400C179
:1011C00011510070114F0021114B00D61049008DB4
:1011D0001047004610440002104200C00F4000803B
:1011E0000F3E00420F3C00060F3B00CB0E38009331
:1011F0000E37005C0E3500270E3400F30D3200C1AF
:101200000D3100900D3000600D2E00320D2D0005C7
:101210000D2C00D90C2B00AE0C2900850C29005C8C
:101220000C2700350C27000E0C2600E80B2400C408
:101230000B2400A00B23007D0B23005A0B21003947
:101240000B2100180B2000F80A1F00D90A1E00BB52
:101250000A1E009D0A1D00800A1D00630A1C00472B
:101260000A1B002C0A1B00110A1A00F7091A00DDDC
:10127000091900C4091900AB091900920917007B6C
:10128000091800630917004C0916003609160020DA
:101290000916000A091500F5081500E0081400CC2D
:1012A000081400B8081400A4081400900813007D66
:1012B0000812006B08130058081200460812003488
:1012C000081100230811001208110001081100F094
:1012D000071000E0071000D0071000C0071000B092
:1012E000070F00A107100091070E0083070F00747D
:1012F000070F0065070E0057070E0049070E003B59
:10130000070D002E070E0020070D0013070D000625
:10131000070D00F9060C00ED060D00E0060C00D4E8
:10132000060C00C8060C00BC060C00B0060C00A49D
:10133000060B0099060C008D060B0082060B007749
:10134000060B006C060B0061060A0057060B004CEA
:10135000060A0042060A0038060A002E060A002481
:10136000060A001A060A001006090007060A00FD10
:10137000050900F4050900EB050900E2050900D99B
:10138000050900D0050900C7050900BE050900B51B
:10139000050800AD050800A50509009C0508009496
:1013A0000508008C050800840508007C0508007409
:1013B0000508006C050700650508005D0507005677
:1013C0000508004E050700470507004005080038DE
:1013D000050700310507002A050700230507001C43
:1013E000050600160507000F0507000805060002A0
:1013F000050700FB040600F5040700EE040600E8FC
:10140000040600E2040700DB040600D5040600CF52
:10141000040600C9040600C3040600BD040600B7A4
:10142000040600B1040500AC040600A6040600A0F2
:101430000405009B04060095040500900406008A3C
:1014400004050085040500800406007A0405007583
:10145000040500700405006B0405006604050061C6
:101460000405005C04050057040500520405004D06
:1014700004050048040500430405003E0404003A46
:1014800004050035040500300404002C0405002781
:10149000040400230405001E0404001A04040016BA
:1014A000040500110404000D0404000904050004EF
:1014B00004040000040400FC030400F8030400F426
:1014C000030400F0030400EC030400E8030400E458
:1014D000030400E0030400DC030400D8030400D488
:1014E000030400D0030400CC030400C8030300C5B8
:1014F00003030024F404D9201BC40C5C0E9804C41C
:10150000095F0265077101F405F900FB04B30048A7
:10151000048700C10369005803550003034500BE5A
:10152000023A008402310053022A002902250004F5
:10153000022000E4011C00C8011900AF0117009847
:1015400001140084011300710110006101100051A9
:10155000010E0043010D0036010B002B010B002092
:10156000010B00150109000C01090003010800FB33
:10157000000800F3000800EB000700E4000600DEAE
:10158000000600D8000600D2000600CC000500C707
:10159000000500C2000500BD000400B9000400B54C
:1015A000000400B1000400AD000400A9000400A57F
:1015B000000300A20003009F0004009B00030098AA
:1015C0000003009500020093000300900003008DCB
:1015D0000002008B000300880002008600020084E5
:1015E000000300810002007F0002007D0002007BFA
:1015F000000200790002007700010076000200740A
:1016000000020072000100710002006F0002006D14
:101610000001006C0002006A00010069000200671E
:101620000001006600010065000100640002006224
:1016300000010061000100600001005F0002005D28
:101640000001005C0001005B0001005A000100592C
:10165000000100580001005700010056000100552C
:10166000000100540001005300000053000100522B
:1016700000010051000100500001004F0001004E28
:101680000000004E0001004D0001004C0001004B25
:101690000000004B0001004A000100490001004821
:1016A000000000480001004700010046000000461D
:1016B0000001004500000045000100440001004316
:1016C0000000004300010042000000420001004110
:1016D00000000041000100400001003F0000003F09
:1016E0000001003E0000003E0001003D0000003D02
:1016F0000001003C0000003C0000003C0001003BF9
:101700000000003B0001003A0000003A00010039EF
:1017100000000039000100380000003800000038E7
:1017200000010037000000370001003600000036DD
:1017300000000036000100350000003500000035D3
:1017400000010034000000340000003400010033C8
:1017500000000033000000330001003200000032BE
:1017600000000032000100310000003100000031B3
:101770000001003000000030000000300001002FA8
:101780000000002F0000002F0000002F0001002E9D
:101790000000002E0000002E0001002D0000002D92
:1017A0000000002D0000002D0001002C0000002C86
:1017B0000000002C0000002C0001002B0000002B7A
:1017C0000000002B0000002B0001002A0000002A6E
:1017D0000000002A0000002A000100290000002962
:1017E0000000002900000029000000290001002855
:1017F0000000002800000028000000280000002849
:10180000000100270000002700000027000000273B
:10181000000000270001002600000026000000262E
:101820000000002600000026000100250000002521
:101830000000002500000025000000250000002514
:101840000001002400000024000000240000002407
:1018500000000024000100230000002300000023FA
:1018600000000023000000230000002300000023EC
:1018700000010022000000220000002200000022DF
:1018800000000022000000220001002100000021D1
:1018900000000021000000210000002100000021C4
:1018A00000000021000100200000002000000020B6
:1018B00000000020000000200000002000000020A8
:1018C000000000200001001F0000001F0000001F9A
:1018D0000000001F0000001F0000001F0000001F8C
:1018E0000001001E0000001E0000001E0000001E7F
:1018F000000000232C0000B8220000561800003A17
:101900000F0000B8080000B1040000710200003EA2
:101910000100001000C90210012C014001220170D9
:10192000011801B0010E01F00104015002FA00B0EB
:1019300002F0003003E600D003DC009004D2007017
:1019400005C800A006BE000008B400B009AA00D077
:101950000BA000600E960060118C00001582002024
:10196000197800C01D6E00A0226400B0275A0090B4
:101970002C500000314600E0343C0010383200901A
:101980003A2800603C1E00A03D1400803E0A002062
:101990003F00002CFFFFFFFFFF000101010101627A
:1019A00065640A002C2073797374656D2073746FFD
:1019B0007070656421204865617465725F49443ABE
:1019C00020004265642068656174696E6720666105
:1019D000696C65640048656174696E672066616959
:1019E0006C65640045312048656174696E672066E6
:1019F00061696C65640048656174696E6720666141
:101A0000696C6564004B494C4C45442E20007001C4
:101A10002C0190012701B0012201C0011D01F0013C
:101A200018011002130130020E0160020901900238
:101A30000401C002FF000003FA004003F500800328
:101A4000F000D003EB002004E6007004E100E004A5
:101A5000DC004005D700C005D2004006CD00D0060E
:101A6000C8008007C3003008BE00F008B900C009F4
:101A7000B400B00AAF00B00BAA00D00CA500000E55
:101A8000A000500F9B00C01096005012910000144F
:101A90008C00C0158700B0178200B0197D00D01BE4
:101AA0007800001E730040206E0090226900F02430
:101AB000640040275F0090295A00E02B5500102E4B
:101AC000500020304B0010324600E033410090358A
:101AD0003C001037370070383200A0392D00B03A82
:101AE0002800A03B2300603C1E00103D1900903DE3
:101AF0001400103E0F00703E0A00C03E0500003F7B
:101B00000000403FFBFF803FF6FFC03FF1FF453143
:101B100020544845524D414C2052554E4157415951
:101B20000042454420544845524D414C2052554EA8
:101B30004157415900546865726D616C2052756E51
:101B400061776179004531204572723A204D4158E4
:101B500054454D50004572723A204D415854454D00
:101B60005020424544004D415854454D5020747218
:101B700069676765726564004531204572723A2075
:101B80004D494E54454D50004572723A204D494ED4
:101B900054454D5020424544004D494E54454D500A
:101BA00020747269676765726564004D3834205827
:101BB0002059205A204500202F002042403A002082
:101BC000403A00024A3135004A3132004A3137008A
:101BD0002020506C616E6E65724275666665724259
:101BE000797465733A20002046726565204D656DF5
:101BF0006F72793A2000436F6D70696C65643A20AA
:101C000046656220313220323031390A00207C2092
:101C1000417574686F723A202864617669647261F4
:101C20006D69726F2C20666F7220416E79637562E8
:101C30006963206933204D656761290A00323031BC
:101C4000392D30322D313100204C617374205570A4
:101C500064617465643A2000312E312E390A004DDA
:101C600061726C696E0020536F66747761726520D3
:101C700052657365740A00205761746368646F6706
:101C80002052657365740A002042726F776E206F70
:101C900075742052657365740A0020457874657206
:101CA0006E616C2052657365740A00506F776572BF
:101CB00055700A0073746172740A004D3234004D1D
:101CC0003233202573006175746F25692E670065B6
:101CD00072726F722077726974696E6720746F20F8
:101CE00066696C650A00205A3A0020593A0020586B
:101CF0003A00656E6473746F7073206869743A207B
:101D000000446F6E6520736176696E672066696C4A
:101D1000652E0A004D3239003A004361703A0020C6
:101D20005A00205900580020204D61783A200020A8
:101D30005A00205900580020204D696E3A20004F6B
:101D40006E20004F666600536F667420656E647384
:101D5000746F70733A20004B6420002364656669D9
:101D60006E652044454641554C545F004B69200048
:101D700023646566696E652044454641554C545F51
:101D8000004B70200023646566696E6520444546FB
:101D900041554C545F00504944204175746F74752F
:101DA0006E652066696E697368656421205075747C
:101DB00020746865206C617374204B702C204B6913
:101DC00020616E64204B6420636F6E7374616E7467
:101DD000732066726F6D2062656C6F7720696E7418
:101DE0006F20436F6E66696775726174696F6E2EDE
:101DF000680A00504944204175746F74756E6520FF
:101E00006661696C6564212074696D656F75740A1B
:101E100000453120544845524D414C2052554E41C9
:101E20005741590042454420544845524D414C20A9
:101E300052554E4157415900546865726D616C208E
:101E400052756E617761790045312048656174692A
:101E50006E67206661696C65640042656420686530
:101E60006174696E67206661696C656400486561CC
:101E700074696E67206661696C656400504944202E
:101E80004175746F74756E65206661696C65642157
:101E90002054656D706572617475726520746F6F22
:101EA00020686967680A00204B643A2000204B696B
:101EB0003A2000204B703A20000A20436C61737373
:101EC000696320504944200A002054753A200020BC
:101ED0004B753A2000206D61783A2000206D696EC4
:101EE0003A200020643A200020626961733A2000A1
:101EF000504944204175746F74756E652066616940
:101F00006C6564212054656D7065726174757265CD
:101F100020746F6F20686967680A00504944204147
:101F200075746F74756E652073746172740A0050F5
:101F30004944204175746F74756E65206661696CE3
:101F400065642120426164206578747275646572ED
:101F5000206E756D6265720A004F66660A00466102
:101F60006465204865696768742000426564204C98
:101F70006576656C696E6720004661696C656420F2
:101F8000746F20656E61626C6520426564204C65EB
:101F900076656C696E670A004D65736820426564FA
:101FA000204C6576656C20646174613A0A004D6569
:101FB000736820706F696E742063616E6E6F742039
:101FC0006265207265736F6C7665640A004D343209
:101FD0003120696E636F7272656374207061726123
:101FE0006D657465722075736167650A00496E736B
:101FF0006572742066696C616D656E7420616E64D3
:102000002073656E64204D3130380A0053656E646C
:10201000204D31303820746F2068656174206E6FF8
:102020007A7A6C650A00496E736572742066696C11
:10203000616D656E7420616E6420707265737320CB
:10204000627574746F6E20286F72204D313038299C
:102050000A0020746F6F206C6F6E67206578747251
:102060007573696F6E2070726576656E7465640A4B
:102070000020636F6C6420657874727573696F6E8D
:102080002070726576656E7465640A00486F6D69CC
:102090006E67206661696C656400206E6F742065F0
:1020A0006E74657265642E0A0050726F7465637495
:1020B00065642050696E0A0046696C616D656E74D6
:1020C00020757365643A200053746174733A20007C
:1020D0002C204C6F6E67657374206A6F623A200023
:1020E000546F74616C2074696D653A20005374619B
:1020F00074733A20002C204661696C65643A2000B4
:102100002C2046696E69736865643A2000507269D4
:102110006E74733A200053746174733A20004A302D
:1021200036004A3034004A30370020573A004A30EF
:1021300038004A30390020573A00205A3A002059D6
:102140003A0020436F756E7420583A0020453A00DB
:10215000205A3A0020593A00583A00256973002560
:10216000696D20256973002569682025696D202522
:10217000697300256964202569682025696D20251B
:1021800069730025697920256964202569682025FF
:10219000696D2025697300656E7175657565696E79
:1021A000672022005072696E7465722073746F70BC
:1021B0007065642064756520746F206572726F723B
:1021C000732E2046697820746865206572726F727C
:1021D00020616E6420757365204D39393920746F24
:1021E00020726573746172742E202854656D706559
:1021F0007261747572652069732072657365742EDF
:10220000205365742069742061667465722072655C
:102210007374617274696E67290A004E6F20436897
:1022200065636B73756D2077697468206C696E6582
:10223000206E756D6265722C204C617374204C6940
:102240006E653A20004E6F20436865636B73756D51
:102250002077697468206C696E65206E756D6265A3
:10226000722C204C617374204C696E653A200063B7
:102270006865636B73756D206D69736D61746368F8
:102280002C204C617374204C696E653A20004C69B7
:102290006E65204E756D626572206973206E6F7475
:1022A000204C617374204C696E65204E756D6265BB
:1022B000722B312C204C617374204C696E653A206E
:1022C000004D313130004D3331005344207265618F
:1022D00064206572726F720A00446F6E65207072BE
:1022E000696E74696E672066696C650A0020496EC4
:1022F00076616C696420657874727564657220001B
:102300000000A0C0000000000000000000005743D3
:102310000000574300004D43454550524F4D206447
:1023200061746173697A65206572726F722E0A003A
:10233000290A002062797465733B20637263200070
:1023400053657474696E67732053746F726564208B
:102350002800290A002062797465733B2063726348
:1023600020002073746F7265642073657474696EE5
:102370006773207265747269657665642028002031
:102380002863616C63756C6174656429210A00209F
:10239000213D2000454550524F4D20435243206D72
:1023A00069736D61746368202D202873746F726582
:1023B000642920002053697A653A2000496E6465DB
:1023C000783A2000204D61726C696E3D5635352992
:1023D0000A0028454550524F4D3D00454550524F4B
:1023E0004D2076657273696F6E206D69736D6174CF
:1023F000636820006F70656E206661696C65642C8F
:102400002046696C653A200043616E6E6F74206FE0
:1024100070656E2073756264697220004A30350001
:102420004A32330053442063617264206F6B0A00A8
:102430006F70656E526F6F74206661696C65640AB7
:1024400000766F6C756D652E696E697420666169C2
:102450006C65640A004572726F723A0053442069D9
:102460006E6974206661696C0A006563686F3A0082
:102470007C3C3E5E2B3D3F2F5B5D3B2C2A225C006B
:10248000627573793A2070617573656420666F7246
:1024900020696E7075740A00627573793A207061F4
:1024A0007573656420666F7220757365720A0062C9
:1024B0007573793A2070726F63657373696E670A1A
:1024C000004A3135004B494C4C45442E20004B49C5
:1024D0004C4C20636175736564206279204B494CD4
:1024E0004C20627574746F6E2F70696E0A004B49D0
:1024F0004C4C45442E20004B494C4C206361757375
:10250000656420627920746F6F206D75636820693F
:102510006E6163746976652074696D65202D206332
:10252000757272656E7420636F6D6D616E643A20B2
:10253000004A3131005072696E7465722068616CB6
:102540007465642E206B696C6C28292063616C6C47
:102550006564210A000000A0C00000000000000027
:102560000000004842000048420000804000000097
:10257000005761726E696E673A20486F6D696E67C9
:102580002042756D702044697669736F72203C201B
:10259000310A000202040000A0400000A040000038
:1025A000004000005C430000574300004D43FFFF24
:1025B000FF486F74656E6420746F6F20636F6C6486
:1025C0000A00486F74656E6420746F6F20636F6CCF
:1025D000640A0000002100240027002A002D00309A
:1025E00000330001010000040107010A010000227C
:1025F00000250028002B002E0031003400020100CD
:1026000000050108010B010000200023002600291D
:10261000002C002F00320000010000030106010918
:102620000105050505070508080808020202020A57
:102630000A08080404040401010101010101010365
:1026400003030303030303040707070C0C0C0C0C20
:102650000C0C0C0202020206060606060606060B13
:102660000B0B0B0B0B0B0B0102102020080810208A
:10267000401020408002010201080402010102040E
:1026800008102040808040201008040201800402CD
:102690000180402010080402010804020101020424
:1026A0000810204080010204081020408000000A29
:1026B0000B02090C0D0E08070304010000000000C6
:1026C000000000000000000000000000000000000A
:1026D00000000000000000000012111000000000C7
:1026E00000000000000000000000000000000000EA
:1026F000000000556E6B6E6F776E20636F6D6D61BD
:102700006E643A202200496E736572742066696CAB
:10271000616D656E7420616E6420707265737320E4
:10272000627574746F6E20286F72204D31303829B5
:102730000A002066697273740A005A005900580032
:10274000486F6D6520005452494747455245440043
:102750006F70656E003A20007A325F6D696E007AA4
:102760005F6D696E00795F6D696E00785F6D696E8F
:10277000005265706F7274696E6720656E64737461
:102780006F70207374617475730A000A4D6561730C
:102790007572656420706F696E74733A0A005A200E
:1027A0006F66667365743A20004E756D20582C591B
:1027B0003A20352C350A000000000100000001001D
:1027C000008000555555000000400033333300AA07
:1027D000AA2A004992240000002000C7711C009919
:1027E000991900D1451700555515003BB113002428
:1027F00049120011111100000010000F0F0F00E32B
:10280000380E0043790D00CCCC0C00C3300C00E82E
:10281000A20B0064210B00AAAA0A00703D0A009DC9
:10282000D80900427B090092240900DCD308008803
:102830008808001042080000000800F0C107008767
:1028400087070075500700711C07003EEB0600A1CA
:10285000BC06006990060066660600703E060061D0
:1028600018060017F4050074D105005BB00500B22E
:10287000900500627205005555050078390500B8CD
:102880001E0500050505004EEC040087D40400A1D8
:10289000BD040090A7040049920400C17D0400EE2D
:1028A000690400C7560400444404005C3204000874
:1028B00021040041100400000004003FF00300F870
:1028C000E0030026D20300C3C30300CCB503003AE3
:1028D000A803000A9B0300388E0300C08103009FF9
:1028E000750300D0690300505E03001D53030034DC
:1028F000480300913D0300333303001629030038D9
:102900001F030097150300300C0300030303000BA3
:10291000FA020049F10200BAE802005CE002002D70
:10292000D802002DD0020059C80200B0C002003108
:10293000B90200DAB10200AAAA0200A0A30200BCF8
:102940009C0200FA9502005C8F0200DF8802008280
:10295000820200457C0200277602002770020043B5
:102960006A02007C640200D05E02003F590200C887
:10297000530200526573656E643A20006F6B00204D
:10298000746F6F206C6F6E672065787472757369F1
:102990006F6E2070726576656E7465640A002063E0
:1029A0006F6C6420657874727573696F6E207072D5
:1029B0006576656E7465640A00FFFDFCFAF8F6F44E
:1029C000F2F0EEECEAE9E7E5E3E1E0DEDCDAD9D7C4
:1029D000D5D4D2D0CFCDCBCAC8C7C5C3C2C0BFBD66
:1029E000BCBAB9B7B6B4B3B2B0AFADACAAA9A8A6D9
:1029F000A5A4A2A1A09E9D9C9A9998979594939224
:102A0000908F8E8D8B8A8988878684838281807F50
:102A10007E7D7B7A797877767574737271706F6E5C
:102A20006D6C6B6A696867666564636261605F5E4E
:102A30005D5C5B5A59585857565554535251505033
:102A40004F4E4D4C4B4A4A494847464645444342FF
:102A50004241403F3E3E3D3C3B3B3A3938383736B9
:102A60003535343332323130302F2E2E2D2C2B2B66
:102A70002A29292827272625252423232221212006
:102A8000201F1E1E1D1C1C1B1B1A19191818171697
:102A900016151514131312121111100F0F0E0E0D1F
:102AA0000D0C0C0B0A0A090908080707060605059C
:102AB00004040303020201000048617264636F644E
:102AC00065642044656661756C742053657474692F
:102AD0006E6773204C6F616465640A00D007000064
:102AE000B00400003C000000102700000000FA4382
:102AF0000000F0420000C040000070420000A04210
:102B00000000A0420000C8433333B94220286D6D55
:102B1000290020204D36303320002055004C00463F
:102B2000696C616D656E74206C6F61642F756E6C7D
:102B30006F6164206C656E677468733A0A002020C8
:102B40004D393030204B004C696E65617220416414
:102B500076616E63653A0A00204400204900202017
:102B60004D33303420500020440020490020204DB7
:102B70003330312050005049442073657474696EBD
:102B800067733A0A00205A0020204D363636004539
:102B90006E6473746F702061646A7573746D656EB2
:102BA000743A0A00205A0020590020204732392068
:102BB0005333205800205A0020204D343230205307
:102BC000004D65736820426564204C6576656C69CC
:102BD0006E673A0A00205A0020590020204D3230FA
:102BE00036205800486F6D65206F66667365743ACD
:102BF0000A00204500205A00205900205800205487
:102C00000020530020204D32303520510020453C1B
:102C10006D61785F655F6A65726B3E0020583C6D40
:102C200061785F785F6A65726B3E20593C6D6178B0
:102C30005F795F6A65726B3E205A3C6D61785F7A9E
:102C40005F6A65726B3E00416476616E6365643AEB
:102C500020513C6D696E5F7365676D656E745F745E
:102C6000696D655F75733E20533C6D696E5F666587
:102C70006564726174653E20543C6D696E5F747268
:102C80006176656C5F66656564726174653E00209F
:102C9000540020520020204D323034205000416337
:102CA00063656C65726174696F6E2028756E6974F6
:102CB000732F7332293A20503C7072696E745F61D1
:102CC0006363656C3E20523C726574726163745F2D
:102CD000616363656C3E20543C74726176656C5F21
:102CE000616363656C3E0A00204500205A0020594C
:102CF0000020204D3230312058004D6178696D75CB
:102D00006D20416363656C65726174696F6E202824
:102D1000756E6974732F7332293A0A0020450020BA
:102D20005A0020590020204D3230332058004D6188
:102D300078696D756D206665656472617465732070
:102D400028756E6974732F73293A0A002045002094
:102D50005A0020590020204D393220580053746504
:102D600070732070657220756E69743A0A002020B5
:102D70004D3230302044300A0020204D3230302097
:102D800044002044697361626C65640A0046696CA2
:102D9000616D656E742073657474696E67733A0053
:102DA0002020473231202020203B004572726F7274
:102DB0002077726974696E6720746F2045455052A0
:102DC0004F4D210A0057726974696E6720746F2035
:102DD00066696C653A20006F70656E206661696C8B
:102DE00065642C2046696C653A20006F70656E2022
:102DF0006661696C65642C2046696C653A20004602
:102E0000696C652073656C65637465640A002053A2
:102E1000697A653A200046696C65206F70656E6559
:102E2000643A20002066696C653A2000646F696E20
:102E300067006672657368004E6F772000454E44E8
:102E400020535542524F5554494E450A0022207096
:102E50006F73002220706172656E743A22005355C0
:102E600042524F5554494E452043414C4C207461C9
:102E7000726765743A22004B494C4C45442E200041
:102E8000747279696E6720746F2063616C6C207353
:102E900075622D67636F64652066696C6573207762
:102EA00069746820746F6F206D616E79206C65762F
:102EB000656C732E204D4158206C6576656C2069D9
:102EC000733A0000DBE891EA11241FBECFEFD1E294
:102ED000DEBFCDBF00E00CBF14E0A0E0B2E0E8EE42
:102EE000FEEE01E00BBF02C007900D92A432B107C5
:102EF000D9F729E1A4E2B4E001C01D92A133B207E1
:102F0000E1F717E1C3E6D7E100E006C02197010928
:102F1000802FFE010E94CCF6C236D10780E0080760
:102F2000A9F70E94FCE20C9463F70C9400002F9226
:102F30003F924F925F926F927F928F929F92AF9249
:102F4000BF92CF92DF92EF92FF920F931F93CF9396
:102F5000DF93CDB7DEB7C354D1090FB6F894DEBF07
:102F60000FBECDBF21E020934711809140128D34D8
:102F700009F459C5843511F40C94FB2B873411F0F6
:102F80000C94472C80913E1290913F128B31910509
:102F900009F403C2A4F48430910534F4823091051D
:102FA00094F597FF29C03BC58430910509F4BFC152
:102FB0004A9709F034C50E94D1410C94492C8A32B9
:102FC000910509F421C444F48C31910509F415C22A
:102FD0004D9709F417C223C58B35910509F49FC499
:102FE0008C35910509F49FC48A35910509F017C500
:102FF000109235040C94492C8091190281110C9483
:103000004E2C0C94492C20911902222311F40C947B
:10301000492C11E0029709F010E00E949683198272
:103020001A821B821C821D821E821F82188682E5E4
:103030000E943440882309F42AC10E94B43F4B0106
:103040005C0120E030E0A9010E9453EF882309F4DD
:1030500034C140914C0450914D0460914E047091E4
:103060004F0448A759A76AA77BA7609150047091A5
:10307000510480915204909153046CA77DA78EA7B0
:103080009FA78091941190919511A0919611B09164
:10309000971188AB99ABAAABBBAB409198115091FB
:1030A000991160919A1170919B114CAB5DAB6EAB15
:1030B0007FAB9C01AD0168A579A58AA59BA50E945F
:1030C00053EF81110DC02CA93DA94EA95FA96CA594
:1030D0007DA58EA59FA50E9453EF882309F4EDC01E
:1030E00020E030E0A901C501B4010E9453EF881F20
:1030F0008827881F181749F060E070E080E89FEB90
:103100006CAF7DAF8EAF9FAF08C080E090E0A0E8CD
:10311000BFE38CAF9DAFAEAFBFAF28A539A54AA521
:103120005BA568A979A98AA99BA90E94CFF368AF7A
:1031300079AF8AAF9BAF2CA53DA54EA55FA56CA925
:103140007DA98EA99FA90E94CFF36B017C0128ADB8
:1031500039AD4AAD5BADCA01B9010E94B8EF2B0190
:103160003C01A7019601C701B6010E94B8EF9B017F
:10317000AC01C301B2010E94D0F30E943BF62B01C7
:103180003C0120E030E040E05FE30E94B8EF24968D
:103190006CAF7DAF8EAF9FAF2497A5019401C501A1
:1031A000B4010E94B8EF4B015C0124962CAD3DADFB
:1031B0004EAD5FAD2497CA01B9010E94B8EF9B01E3
:1031C000AC01C501B4010E94CFF30E943BF62CADC7
:1031D0003DAD4EAD5FAD0E94B8EF4B015C01C70144
:1031E000B6019058A30192010E94ACF4A50194018C
:1031F0000E94B8EF6B017C0128A939A94AA95BA9F3
:1032000068A579A58AA59BA50E94D0F320E030E0AF
:1032100040E05FE30E94B8EF9B01AC01C701B6013B
:103220000E94D0F328A539A54AA55BA50E94CFF33B
:1032300069837A838B839C832CA93DA94EA95FA9BE
:103240006CA57DA58EA59FA50E94D0F320E030E05F
:1032500040E05FE30E94B8EF6B017C01A3019201A3
:1032600068AD79AD8AAD9BAD0E94ACF4A501940127
:103270000E94B8EF9B01AC01C701B6010E94D0F3D8
:103280002CA53DA54EA55FA50E94CFF312C089E4F1
:103290000E943440882331F00E94B43F69837A83CE
:1032A0008B839C838AE40E943440882331F00E94FF
:1032B000B43F6D837E838F83988720E030E0A9013F
:1032C00069817A818B819C810E9453EF81110EC0AC
:1032D00020E030E0A9016D817E818F8198850E9478
:1032E00053EF811103C0E5E5F4E20DC0412FBE01AB
:1032F0006F5F7F4F84E991E10E94A6C30C94492C33
:103300000E94198FF80184918F010F5F1F4F811167
:10331000F7CFE5E3F2E084918F010F5F1F4F882321
:1033200011F40C94492C0E94198FF801F4CF80E518
:103330000E943440882329F00E94278E6B017C0173
:1033400003C0C12CD12C760183E50E943440882330
:1033500061F00E94B43F20E030E04AE754E40E946C
:10336000B8EF0E9419F56B017C010E94B67E0E94A5
:103370004E62C60ED71EE81EF91E0E944E62DC0188
:10338000CB018C199D09AE09BF09B7FD02C00C9491
:10339000492C80E00E948EAEF0CF0E9453B781117D
:1033A0000C94492C80E090E0A0EAB0E489839A83F1
:1033B000AB83BC8380E090E0ADE4B3E48D839E8377
:1033C000AF83B88780E090E0A0EAB1E489879A876C
:1033D000AB87BC8780E50E943440882319F00E94A7
:1033E000843F01C060E068A3BE016F5F7F4FCE01E4
:1033F00080960E9457C10C94492C80E00E94C3869D
:103400000C94492C83E50E943440882321F10E94CA
:10341000943F182F863070F0EBEFF2E084918F012B
:103420000F5F1F4F882311F40C94492C0E94198FB1
:10343000F801F4CF833009F44AC130F4813091F1BE
:10344000823009F43FC008C0843009F4ABC1853034
:1034500009F4B8C101C010E00E941485811103C0B5
:10346000EBEDF2E013C080916211882319F063E163
:1034700073E002C067E173E083ED92E00E94BBCE8F
:103480008AE00E94198F0E94FEC1A2C184917F012F
:103490009FEFE91AF90A882309F49AC10E94198F4B
:1034A000F701F4CF0E94B1C2109201021092000203
:1034B00088EC92E090934B0480934A040E94818FA1
:1034C0000C94492C809100029091010297FF0EC04C
:1034D000EFE9F2E084918F010F5F1F4F882311F411
:1034E0000C94492C0E94198FF801F4CF0097A1F495
:1034F000809142028093360419821A821B821C82B8
:1035000018A219A21AA21BA2BE016F5F7F4FCE01A3
:1035100080960E94A58627C0815065E00E9498F69B
:1035200080FF03C024E0291B922FA5E09A02F0013E
:103530001124E80FF11D87FDFA95EE0FFF1FEE0F26
:10354000FF1FE455FE4E8091540490915504A091C4
:103550005604B091570480839183A283B3838091F2
:1035600036048093420280910002909101028931D9
:1035700091050CF067C0109242029C012F5F3F4FF3
:10358000309301022093000265E00E9498F680FFCC
:1035900003C024E0291B922F4091540450915504FC
:1035A000609156047091570448A359A36AA37BA362
:1035B00019821A821B821C82B4E08B0290011124B2
:1035C000F901EA5EF44F4F0120813181428153813C
:1035D000F4E09F02C0011124BC01665D744F5B01E1
:1035E000DB016D917D918D919C91FE0131966F0172
:1035F000E12CF12C00EA10E40E94B78519821A82AE
:103600001B821C82B601CE0180960E94A586F50120
:1036100080819181A281B38180934C0490934D0469
:10362000A0934E04B0934F04F40180819181A28154
:10363000B3818093500490935104A0935204B093AB
:103640005304C8C080E090E0A0EAB0E48093540442
:1036500090935504A0935604B09357040E9460853C
:103660000E94B67E8FEF9FEF90930102809300023D
:10367000EBE8F2E084918F010F5F1F4F882321F068
:103680000E94198FF801F6CF83E992E09A8389832B
:1036900004E610E019A308A3BE016F5F7F4FCE01BF
:1036A00080960E9450B88AEB92E09A83898319A38E
:1036B00008A3BE016F5F7F4FCE0180960E9450B875
:1036C00081E00E94C38681E00E94418583C088E535
:1036D0000E9434408823D1F00E94843F1FEF160FD0
:1036E0001530D8F065E070E088E792E00E94A2CE45
:1036F000E5E7F2E084918F010F5F1F4F882311F4FB
:103700000C94492C0E94198FF801F4CF88E50E948F
:10371000198F0E94CBE80C94492C89E50E94344013
:103720008823D1F00E94843F0FEF060F0530D8F0B8
:1037300065E070E082E692E00E94A2CEEFE5F2E062
:1037400084918F010F5F1F4F882311F40C94492C33
:103750000E94198FF801F4CF89E50E94198F0E9409
:10376000CBE80C94492C8AE50E943440882399F0D8
:103770000E94B43F25E0129FF0011124E00FF11DDB
:10378000EE0FFF1FEE0FFF1FE455FE4E60837183A7
:103790008283938335C08AE50E94198F0E94CBE80B
:1037A0000C94492C8AE50E9434408823A1F30E949E
:1037B000B43F6093A8117093A9118093AA119093BC
:1037C000AB111EC080E00E9441850E94B1C218C0AA
:1037D0001230B1F4609100027091010269317105FB
:1037E00014F069E170E080E592E00E94A2CE69E108
:1037F00070E08BE492E00E94A2CE8AE00E94198FD2
:103800000E94C77E0C94492C80911902882311F4E0
:103810000C94492C89E40E943440E82E882321F03E
:103820000E94843F062F01C000E08AE40E943440D9
:10383000F82E882321F00E94843F162F01C010E04B
:10384000EE2011F0053020F4FF2081F0153070F0EB
:10385000E2E1F3E084918F010F5F1F4F882311F4A1
:103860000C94492C0E94198FF801F4CF0E9440401B
:10387000EE2091F044E00402F0011124E65DF44FE3
:1038800080819181A281B38180939411909395114D
:10389000A0939611B0939711FF2091F054E0150278
:1038A000F0011124EA5EF44F80819181A281B381FD
:1038B0008093981190939911A0939A11B0939B11B2
:1038C00080E50E943440882319F00E94A53F03C080
:1038D00080E50E94EB3F86E40E9434408823D9F0C3
:1038E0000E94B43F6B017C0120E030E0A9010E94FE
:1038F000F6F5181684F420E030E040E752E4C70102
:10390000B6010E94ACF4609343027093440280932A
:103910004502909346020E94B8C70C94492C20930C
:1039200035040C94492C27E5222E22E0322E38EF64
:10393000E32E30E1F32E6CE474E079A768A744E24B
:10394000C42E44E0D42E00E010E0D1018D911D0181
:103950000E943440882309F44BC00E94B43F2B01DD
:103960003C01133049F0F6012081318142815381BD
:103970000E94CFF32B013C01A8A5B9A52D913D9143
:103980004D915C91C301B2010E94CFF34B015C01E8
:103990002DEB37E346E855EB0E94F6F587FD0AC0AC
:1039A0002DEB37E346E855E3C501B4010E9453EF20
:1039B0001816F4F4133051F44092580450925904FC
:1039C00060925A0470925B0401E012C0A501940158
:1039D000F70160817181828193810E94D0F3D701C8
:1039E0006D937D938D939C931397812F0E94A08D4F
:1039F0001F5FB4E0EB0EF11CE8A5F9A53496F9A71A
:103A0000E8A7F4E0CF0ED11C143009F09ECF0023BC
:103A100009F4F6CE88E594E00E94F2B6F1CE0E9459
:103A2000EEB90C94492C80913E1290913F1285374B
:103A3000910511F40C94492C0CF0C0C08C34910504
:103A400009F408C50CF058C08931910509F4E8C2A1
:103A50001CF58431910509F4C9C17CF481319105CB
:103A600009F44AC22CF4029708F4C3C10C94F82B51
:103A7000429709F4E0C60C94F82B8631910509F4BD
:103A800089C20CF483C28731910509F489C2489731
:103A900009F49CC20C94F82B8E31910509F47EC375
:103AA00084F48B31910509F4D7C20CF4C7C28C3170
:103AB000910509F469C34D9711F40C94492C0C94A9
:103AC000F82B8A32910509F46CC44CF48F319105BE
:103AD00009F442C4809709F4F3C30C94F82B8133A2
:103AE000910509F492C48B34910511F00C94F82BD4
:103AF0000E94D6CE0C94492C8936910509F472C5E2
:103B000044F58335910509F492C69CF48E349105F1
:103B100009F4A8C40CF4A2C48135910509F475C652
:103B20008235910511F00C94F82B109234040C940A
:103B3000492C8535910509F4B1C60CF47CC68C3549
:103B4000910509F4C4C68836910509F48FC40C9414
:103B5000F82B8E36910509F4B2C4A4F48B36910586
:103B600009F4BAC50CF49AC58C36910511F40C947D
:103B7000492C8D36910511F00C94F82B0E94AF87DB
:103B80000C94492C8137910509F4FFC45CF48F36FD
:103B9000910509F4A7C48037910511F40C94492CC0
:103BA0000C94F82B8237910509F419C783379105D6
:103BB00011F00C94F82BEFEDF4E050C78E3221E0B9
:103BC000920711F40C94AB290CF082C0893C91054A
:103BD00011F40C942F267CF58D37910509F48EC5D0
:103BE000ACF48737910509F4E1C70CF492C7883724
:103BF000910509F4DEC78937910511F00C94F82B73
:103C00001092E6051092E5050C94492C8B3991052C
:103C100009F403C534F48C38910509F425C50C94D6
:103C2000F82B8E3B910509F435C5883C910509F4C4
:103C3000C6C70C94F82B833D910511F40C943B28D6
:103C400044F58C3C910511F40C9466266CF48B3C85
:103C5000910511F00C94F82BA7E5EA2EA2E0FA2EBC
:103C60000EE917E00C9456268D3C910511F40C9446
:103C7000DB268E3C910511F00C94F82BE7E5CE2E57
:103C8000E2E0DE2EF7EEEF2EF5E0FF2E10E00C94D2
:103C90006227823E910511F40C94B92864F48C3D9E
:103CA000910511F40C943E288D3D910511F40C946E
:103CB0004B280C94F82B8C3251E0950711F40C949E
:103CC000E2288D32914011F40C940B290C94F82BBE
:103CD000863F71E0970711F40C949B2A0CF043C0C7
:103CE0008A39B1E09B0711F40C94492CBCF4803361
:103CF000F1E09F0711F40C94022A14F40C94FF29AC
:103D0000833641E0940709F46DC08039914011F089
:103D10000C94F82B0E94B67E0C94492C8C3A61E0EE
:103D2000960711F40C9475277CF4843AA1E09A0765
:103D300011F40C94952A853A914011F00C94F82BCB
:103D40000E9415650C94492C843FE1E09E0711F414
:103D50000C94982A853F914011F00C94F82B0E9406
:103D6000A7990C94492C8B3522E0920711F40C94FE
:103D7000D72AC4F4883F51E0950711F40C94AA2A7D
:103D800014F40C949E2A8C3072E0970711F40C9472
:103D9000CE2A8835924011F00C94F82B0E94436390
:103DA0000C94492C8B38B3E09B0711F40C94492CEC
:103DB0006CF48A39F2E09F0711F40C94602B84387C
:103DC000934011F40C948D2B0C94F82B803A43E023
:103DD000940709F4B4C2873E934011F40C94E52B88
:103DE0000C94F82BE5E5F4E20C94822AE0E4F3E08D
:103DF0008FC0A0903C12B0903D1280E50E943440EC
:103E0000882359F00E94278E6B017C0111E0672BFB
:103E1000682B692B31F410E004C010E0C12CD12CC8
:103E2000760183E50E943440882311F40C94532CCE
:103E30000E94B43F20E030E04AE754E40E94B8EF2B
:103E40000E9419F56B017C0111110BC0672B682BC7
:103E5000692B39F4A114B10421F0D5018C918111A1
:103E600002C010E001C011E00E94B67E1123B9F03B
:103E7000EAE6F4E284918F010F5F1F4F882321F05F
:103E80000E94198FF801F6CFF50181915F01882317
:103E900019F00E94198FF8CF8AE00E94198F83E0F1
:103EA0008093471181E080934611C114D104E1044D
:103EB000F104B1F00E944E62C60ED71EE81EF91E34
:103EC0000E944E62DC01CB018C199D09AE09BF092D
:103ED000B7FF0EC08091461181110C94582C08C078
:103EE00080914611882321F080E00E948EAEF8CFA9
:103EF000109246110C94492C5F988A9847988091AB
:103F00000801817080930601479812980C94492CFF
:103F100084918F010F5F1F4F882321F00E94198F1A
:103F2000F801F6CF1092DC0D8FE89BE00E9436A7D7
:103F30008BE1EFE8FBE0DE01159601900D928A958A
:103F4000E1F780918D0B90918E0B9C838B838DEE8E
:103F500092E09A83898340E050E0BE016F5F7F4F1B
:103F600080E090E00E9414A2CE0101960E9424AE4F
:103F7000E1E3F3E084918F010F5F1F4F882311F479
:103F80000C94492C0E94198FF801F4CF0E9410A0C4
:103F90000C94492C10925E0B10925F0B0C94492CE0
:103FA000E0913C12F0913D128081882329F080320B
:103FB00009F410823196F8CF40E061E080913C1224
:103FC00090913D120E9487DE0C94492C80E090E095
:103FD000A0E2B1E489839A83AB83BC8318A219A2BF
:103FE0001AA21BA21CA21DA21EA21FA28091D10870
:103FF000882359F020E0AE014F5F5F4FBE01605E45
:104000007F4FCE0184960E9484B880915F0B8823F5
:1040100019F081E080935E0B0E94D6CE0C94492C5F
:1040200010925E0B0E94D76181E593E090934B0460
:1040300080934A040E94818F0C94492C80915F0BDD
:10404000882311F40C94492C83E50E94344081119B
:104050000C945D2C0C94492C83E40E94EB3F882344
:1040600009F450C0E3E8F3E084918F010F5F1F4F24
:10407000882321F00E94198FF801F6CF80912A0D34
:10408000811103C0E6E5F3E012C0BE016F5F7F4F10
:1040900087E29DE00E94FEA58E010F5F1F4FD801B1
:1040A0008D918D01882349F10E94198FF8CF849159
:1040B0008F010F5F1F4F882301F10E94198FF801B4
:1040C000F6CF9BEDC92E93E0D92EE12CF12C20E008
:1040D0008091BA0790E00E2C02C0959587950A94BE
:1040E000E2F780FD2FC24FEFE41AF40A52E0C50E4A
:1040F000D11C65E0E616F10459F78AE00E94198F99
:104100000C94492C80915F0B882339F080915E0BD1
:10411000882319F0E0E6F3E003C0E2E7F3E028C00B
:1041200084918F010F5F1F4F882321F00E94198F08
:10413000F801F6CF6091D80D7091D90D8091DA0D0C
:104140009091DB0D4AE00E9455928FE20E94198FF8
:104150006091D40D7091D50D8091D60D9091D70DB1
:104160004AE00E9455928AE00E94198F0C94492CD3
:1041700084918F010F5F1F4F882311F40C94492CF9
:104180000E94198FF801F4CF40E060E080913C126A
:1041900090913D120E9487DE0C94492C80915F0B18
:1041A000882311F40C94492C87E29DE00E94B4DC32
:1041B00087E29DE00E94D9A510925D0B10925C0BE6
:1041C00080915F0B882311F40C94492C00913C12D0
:1041D00010913D120E9406A2B801CE0180960E9465
:1041E0001AA48C01892B11F40C94492C68A179A193
:1041F0006115710511F06C5F7F4F19821C8222E0FE
:10420000A801CE0101960E9465AB811102C0F12C7C
:1042100014C0CE0101960E9476A18823C1F361E00B
:10422000CE0101960E94E2A5009789F325EEFC01DC
:1042300020831C820E945DDAF82ECE0101960E9436
:10424000138FF11003C0E0EAF3E022C0E2E9F3E0EB
:1042500084917F012FEFE21AF20A882321F00E9455
:10426000198FF701F5CFD8018D918D01882319F0B1
:104270000E94198FF8CF8AE00E94198F1092D80DF2
:104280001092D90D1092DA0D1092DB0D0C94492C7E
:1042900084917F01BFEFEB1AFB0A882321F00E9473
:1042A000198FF701F5CFF80181918F01882319F05B
:1042B0000E94198FF8CF8EE20E94198F0C94492C1E
:1042C00080915E0B81110E94B67E80915F0B8823E6
:1042D00011F40C94492C80E50E943440882319F095
:1042E0000E94A53F03C080E50E94EB3F182F482F96
:1042F00061E080913C1290913D120E9487DE83E53F
:104300000E943440882381F00E94843FAB01BC01AD
:104310004093D80D5093D90D6093DA0D7093DB0D57
:1043200087E29DE00E94EFA480915F0B882319F043
:1043300081E080935E0B11110C94492C6DCE80911D
:104340003C1290913D1221E020935D0B40E060E033
:104350000E9487DE0C94492C0E94896168A379A38E
:104360008AA39BA3BE016F5F7F4FCE0180960E9400
:10437000378EEAE6F4E284918F010F5F1F4F8823A6
:1043800021F00E94198FF801F6CFBE016F5F7F4FB9
:1043900088EB93E00E94BBCE8AE00E94198F0C94B8
:1043A000492C83E50E943440882311F40C94492C55
:1043B0000E94943FE82E80E50E943440882339F023
:1043C0000E94943F182F87FF03C00C94492C1DE0D6
:1043D00089E40E943440882341F00E94A53F811166
:1043E0000C94DA2CEAE2F6E00BC089E40E94EB3F81
:1043F000F6CF319626E0EA35F20711F40C94DA2C68
:1044000084911813F6CF0C94AE2CF090300481E018
:10441000F826F0923004E0EDF3E084918F010F5F15
:104420001F4F882321F00E94198FF801F6CFFF203B
:1044300019F0E5ECF3E002C0EAECF3E084918F01BF
:104440000F5F1F4F882311F40C94492C0E94198F81
:10445000F801F4CF0E94D7610C94492C0E941DCF23
:104460000C94492C0E947C810C94492C88E690E0A5
:104470000E94208F81110C94492C8091BA0783FFF0
:1044800002C00C94492C83E50E943440882399F0A3
:104490000E94B43F0E9414F5CB010E94E2590E9491
:1044A000B43F20E030E04AEA52E40E9453EF18168D
:1044B00014F00E941DCF0E94CFD00C94492C8EE4A2
:1044C0000E943440882311F40C94492C0E94843FAC
:1044D00060932719709328198093291990932A19AA
:1044E0000C94492C83E50E94EB3F882359F083E527
:1044F0000E943440882319F00E94943F01C080E05C
:104500008093BA07EAE6F4E284918F010F5F1F4FB0
:10451000811103C0E9EEF3E004C00E94198FF80195
:10452000F3CF84918F010F5F1F4F882321F00E94EA
:10453000198FF801F6CF8091BA078111C2CDE5EE4F
:10454000F3E018C0BB24B394B20E222319F08CE21E
:104550000E94198FF60185919491FC0184918F013D
:104560000F5F1F4F882321F00E94198FF801F6CFAB
:104570002B2DB9CD84918F010F5F1F4F882309F434
:10458000BCCD0E94198FF801F5CF83E50E9434401D
:10459000811103C0EAE6F4E20DC00E94943F8D331E
:1045A00020F4809329020C94492C8CE380932902F7
:1045B0000C94492C84918F010F5F1F4F882321F0A9
:1045C0000E94198FF801F6CF4091290250E060E077
:1045D00070E080EF93E00E9468CE8AE00E94198F1D
:1045E0000C94492C89E690E00E94208F811111C023
:1045F000E7EFF3E084918F010F5F1F4F882321F0D5
:104600000E94198FF801F6CF0E9490588AE00E940C
:10461000198F109247110C94EF2C83E50E943440BF
:10462000882311F40C94492C0E94943F182F8D3349
:1046300008F01CE31093F7100E944E626B017C019E
:10464000212F30E0A8EEB3E00E94C0F3C60ED71EC3
:10465000E81EF91EC092F310D092F410E092F5100B
:10466000F092F6100C94492C8091BA0783FF02C097
:104670000C94492C83E50E943440882311F40C9457
:10468000492C0E94B43F0E9414F5CB010E94C34103
:104690000C94492C0E94917F0C94492C80E50E9437
:1046A0003440811106C083E50E943440882361F0C4
:1046B00006C00E94943F81110C94492CF4CF0E94B3
:1046C000843F6F3F710510F06FEF70E0709341040D
:1046D000609340040C94492C80E50E943440811181
:1046E00006C010924104109240040C94492C0E9480
:1046F000843F672B11F00C94492CF3CF8CE40E947B
:10470000EB3F882381F00E94B43F6B017C0120E0E5
:1047100030E0A9010E94F6F587FF0BC0F7FAF0948C
:10472000F7F8F09406C0C12CD12C80E8E82E80E484
:10473000F82EF7FAF094F7F8F094CCA2DDA2EEA2EE
:10474000FFA280E090E0A0EAB0E489839A83AB8383
:10475000BC8380E090E0ADE4B3E48D839E83AF83BF
:10476000B88780E090E0A0EAB1E489879A87AB87B8
:10477000BC8788E50E943440882379F088E50E9450
:104780003440882319F00E94B43F03C060E070E019
:10479000CB0169837A838B839C8389E50E943440B3
:1047A000882379F089E50E943440882319F00E941B
:1047B000B43F03C060E070E0CB016D837E838F83E4
:1047C00098878AE50E943440882379F08AE50E9420
:1047D0003440882319F00E94B43F03C060E070E0C9
:1047E000CB0169877A878B879C8718A219A21AA2A6
:1047F0001BA2AE01405E5F4FBE016F5F7F4FCE01D7
:1048000084960E9466B30C94492C0E94F2590E942F
:10481000FEBB109241041092400468EE73E080E009
:1048200090E00E9467610E94092D0C94492C20930E
:1048300034040C94492C83E50E9434408823A1F071
:104840000E94B43F20E030E04AE754E40E94B8EF11
:104850000E9419F560932A0270932B0280932C0218
:1048600090932D020C94492C88E50E94EB3F811116
:104870000C946E2C89E50E94EB3F81110C946E2CF8
:104880008AE50E94EB3F81110C946E2C85E40E9416
:10489000EB3F81110C946E2C0C94A02C83E50E94AC
:1048A000EB3F882309F4F5C70E94B43F20E030E0D5
:1048B0004AE754E40E94B8EF0E9419F56093EF10A4
:1048C0007093F0108093F1109093F210E2C717E507
:1048D000C12E12E0D12E08E7E02E01E1F02E10E00B
:1048E000D6018D916D010E94EB3F882309F46DC0C4
:1048F000133009F063C00E94B43F4B015C0120E01B
:1049000030E040EA51E40E9453EF87FF4EC0A5011A
:10491000940160918411709185118091861190911C
:1049200087110E94ACF42B013C019B01AC0160910A
:104930008E0770918F0780919007909191070E9448
:10494000B8EF60938E0770938F07809390079093D2
:104950009107A30192016091AA077091AB07809122
:10496000AC079091AD070E94B8EF6093AA077093CF
:10497000AB078093AC079093AD076091691270917B
:104980006A1280916B1290916C120E9457EFA301F2
:1049900092010E94B8EF0E9419F56093691270931A
:1049A0006A1280936B1290936C1280928411909291
:1049B0008511A0928611B092871107C00E94B43F62
:1049C000F70160837183828393831F5FF4E0EF0EAE
:1049D000F11C143009F084CF0E9470D25AC70E9493
:1049E000B67E83E50E943440882311F40C94001CA9
:1049F0000E94843F6230710511F00C94001C0E94EB
:104A000092CB8BE50E94198F6091411270914212F6
:104A1000809143129091441242E00E94DA924091B8
:104A200045125091461260914712709148128DEFD5
:104A300093E00E9485CE4091491250914A126091B4
:104A40004B1270914C128AEF93E00E9485CE8DE557
:104A50000E94198F8AE00E94198F1BC784918F01D1
:104A60000F5F1F4F882321F00E94198FF801F6CFA6
:104A700060E08FEC94E00E94596E61E088EC94E075
:104A80000E94596E61E08DEB94E00E94596E61E0E6
:104A90008DEA94E00E94596E60E084EA94E00E94FE
:104AA000596E61E08AE994E00E94596E60E080E905
:104AB00094E00E94596E60E088E894E00E94596E8C
:104AC00061E08AE794E00E94596E60E08CE694E031
:104AD0000E94596E60E08DE594E00E94596E60E09E
:104AE0008FE494E00E94596E60E089E394E00E94B4
:104AF000596E61E088E294E00E94596E60E083E1C3
:104B000094E00E94596E61E080E094E00E94596E4A
:104B1000C0C600913C1210913D1283E0D12C40E0C0
:104B20008150E9F0D8019C91292F2B7F2134C1F7C6
:104B300011962C912133A1F7913421F0953421F471
:104B400041E002C0DD24D39498012E5F3F4F8901DC
:104B50002F5F3F4FF80190819032C9F3E1CF44239A
:104B600069F0EAE6F4E284917F012FEFE21AF20A9B
:104B7000882321F00E94198FF701F5CFDD2069F01D
:104B8000E8EBF5E084917F014FEFE41AF40A882303
:104B900021F00E94198FF701F5CFD8018D918D0179
:104BA000882309F4AACA0E94198FF7CF0E9470C304
:104BB00070C681E08093E6058093E5056AC688ECBF
:104BC00090E00E94208F811164C684E40E94EB3F34
:104BD000882309F441C00E94B43F6B017C0111E0BD
:104BE00020E030E0A9010E9453EF811101C010E0E4
:104BF0001093101220E030E0A901C701B6010E9415
:104C000053EF882349F10E94B43FE0917805B4E066
:104C1000EB9FF0011124EB5EFD4E60837183828374
:104C2000938320E030E0A901609115127091161273
:104C300080911712909118120E9453EF81110CC0AD
:104C400080E090E0A0EEBFE38093151290931612DF
:104C5000A0931712B09318120E943DBC1AC6B7E574
:104C6000EB2EB2E0FB2E0DE612E1F70181917F0100
:104C70000E94EB3F882351F00E94B43F0E9419F537
:104C8000D8016D937D938D939C9313970C5F1F4F69
:104C9000B2E10D371B0749F70E94FFD0FAC50C5F40
:104CA0001F4FB7E00E3A1B0709F4F3C5F7018191D6
:104CB0007F010E94EB3F882391F30E94B43FD8010B
:104CC0006D937D938D939C931397E9CF83E50E9419
:104CD00034408823A1F00E94B43F60939A077093F8
:104CE0009B0780939C0790939D0760939607709312
:104CF0009707809398079093990710E001C011E0FF
:104D000080E50E943440882359F00E94B43F6093AC
:104D10009A0770939B0780939C0790939D0710E0E0
:104D200082E50E943440882359F00E94B43F60938A
:104D3000421170934311809344119093451110E0F8
:104D400084E50E943440882359F00E94B43F609368
:104D5000960770939707809398079093990799C542
:104D6000112309F496C540919A0750919B076091D1
:104D70009C0770919D0782EC95E00E9485CE409142
:104D800042115091431160914411709145118FEB84
:104D900095E00E9485CE40919607509197076091CB
:104DA0009807709199078CEB95E00E9485CE8AE078
:104DB0000E94198F6EC581E50E94EB3F882351F058
:104DC0000E94278E6093AE077093AF078093B00761
:104DD0009093B10783E50E94EB3F882351F00E9436
:104DE000B43F6093B6077093B7078093B80790936A
:104DF000B90784E50E94EB3F882351F00E94B43F3D
:104E00006093B2077093B3078093B4079093B5078C
:104E100088E50E94EB3F882351F00E94B43F6093E5
:104E2000820770938307809384079093850789E5B1
:104E30000E94EB3F882351F00E94B43F60938607A5
:104E40007093870780938807909389078AE50E946B
:104E5000EB3F8823F1F00E94B43F60938A07709380
:104E60008B0780938C0790938D072DEC3CEC4CECDA
:104E70005DE30E9453EF181664F0E2EDF5E08491D3
:104E80008F010F5F1F4F882321F00E94198FF801B7
:104E9000F6CF85E40E94EB3F882309F4FAC40E9410
:104EA000B43F60938E0770938F0780939007909321
:104EB0009107EFC41F5FB4E0EB0EF11C133011F447
:104EC0000C94001CF60181916F010E94EB3F882336
:104ED00089F30E94B43FD7016D937D938D939C938A
:104EE0001397812F0E94A08DE5CF0E9453B78111A7
:104EF000D0C405E515E2ECE4F4E0F9A7E8A7AE01BB
:104F00004F5F5F4F4A017EEAA72E75E2B72E1A0166
:104F1000F8016591759185919491A8A5B9A5CD9059
:104F2000DD90ED90FD90B9A7A8A7A70196010E947A
:104F3000CFF32B013C01F101608371838283938362
:104F400020E030E040EA51EC0E94F6F587FD0AC00F
:104F500020E030E040EA51E4C301B2010E9453EF87
:104F600018162CF4F501849118160CF4ECC4D10138
:104F7000CD90DD90ED90FD901D0120E030E040EA05
:104F800051ECC701B6010E94F6F587FD0AC020E08A
:104F900030E040EA51E4C701B6010E9453EF181611
:104FA0004CF5E5E5F4E284918F010F5F1F4F81110D
:104FB00003C0E4E0F6E004C00E94198FF801F3CFCB
:104FC00084918F010F5F1F4F882321F00E94198F5A
:104FD000F801F6CF88E290E099A388A388EC90E0EE
:104FE0009DA38CA3BE01605E7F4FCE0184960E947C
:104FF00050B84FC40C5F1F4FBFEFAB1ABB0AE1E6BE
:10500000F5E2E017F10709F083CF67EEE62E65E0E1
:10501000F62E10E0F40181919191A191B1914F018F
:10502000F70181939193A193B1937F01812F0E9406
:10503000A08D1F5F133071F70E94C77E83E992E055
:105040009DA38CA304E610E019A308A3BE016C5D28
:105050007F4FCE0180960E9450B88AEB92E09DA3CC
:105060008CA319A308A3BE016C5D7F4FCE0180966F
:105070000E9450B80EC40E947B6D0BC483E50E9451
:105080003440882309F405C40E94843F70930302CE
:1050900060930202FEC38DED90E00E94208F81118B
:1050A000F8C383E50E943440811103C0EAE6F4E2CC
:1050B0003AC00091780510E00E94843F000F111F54
:1050C000F801E05CFD4F718360838091780590E08A
:1050D0007C01EE0CFF1CEE0CFF1C87010B5D1D4FCD
:1050E000880F991FFC01E05CFD4F60817181072EE4
:1050F000000C880B990B0E9459EF2AE037ED43E230
:105100005CE30E94B8EFF701EF5EFD4E2081318134
:10511000428153810E94B8EFD8016D937D938D93A6
:105120009C931397B6C384918F010F5F1F4F882301
:1051300021F00E94198FF801F6CF85E40E94198FA3
:1051400080917805805D0E94198FE0917805F0E0EC
:10515000EE0FFF1FE05CFD4F6081718182E296E0FF
:105160000E94A2CE85E20E94198F8AE00E94198FC8
:1051700090C380E50E94EB3F882309F48AC30E9414
:10518000843F6B017C0183E50E943440882321F039
:105190000E94843F8B0102C00FEF1FEFC8010196F0
:1051A000039708F076C3D7FC74C38C2DEAE2F6E0CF
:1051B0009491891709F4D2C33196B6E0EA35FB071A
:1051C000B9F7CFC383E50E943440882319F00E94C9
:1051D000843F02C064E071E079A368A380E50E9487
:1051E0003440882339F00E94843F6938E3E17E0728
:1051F00030F402C068EE73E07A83698304C088E803
:1052000093E19A838983BE01605E7F4FCE01019650
:105210000E9450B83EC385E40E943440811110C002
:1052200080E50E94EB3F882391F00E94B43F609399
:10523000650570936605809367059093680507C0C0
:105240000E94943F882361F3E5E5F4E271C089E4AC
:105250000E94EB3F882381F00E94B43F2CEA35EC9A
:1052600047E25EE30E94B8EF6093610570936205C8
:10527000809363059093640584E40E94EB3F882348
:1052800081F00E94B43F2CEA35EC47E25EE30E94D5
:10529000ACF46093690570936A0580936B059093F5
:1052A0006C05EAE6F4E284918F010F5F1F4F8823BB
:1052B00021F00E94198FF801F6CF409165055091B9
:1052C0006605609167057091680582E696E00E9428
:1052D00085CE2CEA35EC47E25EE360916105709182
:1052E000620580916305909164050E94ACF4AB0166
:1052F000BC018EE596E00E9485CE2CEA35EC47E2B3
:105300005EE36091690570916A0580916B059091EB
:105310006C050E94B8EFAB01BC018AE596E00E94E3
:1053200085CE8AE00E94198FB4C20E94198FF801BD
:1053300084918F010F5F1F4F8111F7CFE6E6F6E0F2
:1053400084918F010F5F1F4F882309F4A2C20E942E
:10535000198FF801F5CF83E50E94EB3F182F8823C2
:1053600071F00E94B43F0E9414F570933B02609369
:105370003A0221E0672B09F020E02093581180E5E4
:105380000E94EB3F882359F020913A0230913B0272
:10539000232B11F00E94A53F809358117AC211115E
:1053A00078C2EAE6F4E284918F010F5F1F4F8823F1
:1053B00021F00E94198FF801F6CF809158118823AF
:1053C00019F06BE173E002C06EE173E08DE896E0E6
:1053D0000E94BBCE60913A0270913B028CE796E04E
:1053E0000E94A2CEE8E7F6E084918F010F5F1F4F85
:1053F000882309F44EC20E94198FF801F5CF0E944C
:10540000046847C280E50E94EB3F882351F00E9468
:10541000B43F60935D0570935E0580935F05909344
:10542000600589E40E94EB3F882381F00E94B43F2D
:105430002CEA35EC47E25EE30E94B8EF6093590531
:1054400070935A0580935B0590935C0584E40E94F9
:10545000EB3F882381F00E94B43F2CEA35EC47E211
:105460005EE30E94ACF460935505709356058093FB
:10547000570590935805EAE6F4E284918F010F5F97
:105480001F4F882321F00E94198FF801F6CF409119
:105490005D0550915E0560915F057091600588EA39
:1054A00096E00E9485CE2CEA35EC47E25EE36091FF
:1054B000590570915A0580915B0590915C050E9499
:1054C000ACF4AB01BC0184EA96E00E9485CE2CEAE4
:1054D00035EC47E25EE36091550570915605809189
:1054E0005705909158050E94B8EFAB01BC0180EAC6
:1054F00096E00E9485CE8AE00E94198FCAC10E9460
:10550000198FF80184918F010F5F1F4F8111F7CF21
:10551000ECEAF6E084918F010F5F1F4F882309F4B6
:10552000B8C10E94198FF801F5CF0E940066B1C181
:105530000E94B399AEC10E94A5D7ABC183E50E947A
:10554000EB3F882321F00E94A53F91E089270E942C
:10555000E1D29FC181E08093D0080E946F931092A6
:10556000D008882309F495C1EAE6F4E284918F011A
:105570000F5F1F4F811103C0EBEBF6E004C00E94E8
:10558000198FF801F3CF84918F010F5F1F4F88238C
:1055900009F47FC10E94198FF801F5CF80915E0B4D
:1055A000882309F476C181E08093610B72C18BE599
:1055B00092E00E94208F81116CC185E50E94EB3F33
:1055C0008823D9F10091780510E00E94B43F6B0167
:1055D0007C0120E030E0A9010E94F6F587FF04C0BD
:1055E000F7FAF094F7F8F094000F111F000F111F55
:1055F000F801E75EF64EC082D182E282F38200912A
:105600007805F4E00F9F80011124075E164E20E01C
:1056100030E046E154E4D8016D917D918D919C91EB
:105620000E94F6F518164CF480E090E0A6E1B4E490
:10563000F80180839183A283B3838CE40E94EB3FC3
:10564000882309F426C10091780510E00E94B43F38
:105650006B017C0120E030E0A9010E94F6F587FF94
:1056600004C0F7FAF094F7F8F094000F111F000F40
:10567000111FF801E35EF64EC082D182E282F3820E
:1056800000917805F4E00F9F80011124035E164E0F
:1056900020E030E046E154E4D8016D917D918D9198
:1056A0009C910E94F6F518160CF0F3C080E090E093
:1056B000A6E1B4E4F80180839183A283B383E9C0B7
:1056C0008AE50E943440811103C0E9ECF6E00BC08A
:1056D0000E94B43F6093211970932219809323197B
:1056E00090932419D6C084918F010F5F1F4F882398
:1056F00021F00E94198FF801F6CF409121195091A5
:105700002219609123197091241986EC96E00E9469
:1057100085CE8AE00E94198FBCC08BE40E94344081
:10572000811103C0EAE6F4E236C08BE40E94344003
:105730008823C1F00E94B43F6B017C0120E030E07F
:10574000A9010E94F6F587FD0AC020E030E040E2A2
:1057500051E4C701B6010E9453EF181634F4E8EE85
:10576000F6E00EC0C12CD12C76010E94B67EC0920C
:105770009207D0929307E0929407F092950789C020
:1057800084918F010F5F1F4F882309F482C00E940C
:10579000198FF801F5CF84918F010F5F1F4F882378
:1057A00021F00E94198FF801F6CF40919207509195
:1057B0009307609194077091950787E097E00E94A6
:1057C00085CE8AE00E94198F64C081E0809319021F
:1057D00083E50E943440882339F00E94A53F81115F
:1057E00058C00E94CBCB55C083E50E94EB3FF7CF5A
:1057F0000E94EEB94EC0F0903E120E94B67E10910B
:10580000621180E00E944185FF2029F1EAE6F4E27E
:1058100084918F010F5F1F4F882321F00E94198F01
:10582000F801F6CF84E50E94198F6F2D70E080E0BB
:1058300090E04AE00E94559280E20E94198FE4E2D3
:10584000F7E084918F010F5F1F4F882311F10E94B1
:10585000198FF801F6CF10921011812F0E94418507
:10586000EAE6F4E284918F010F5F1F4F882321F055
:105870000E94198FF801F6CF6091101170E082E15B
:1058800097E00E94A2CE8AE00E94198F02C00E9477
:10589000EEB9109247110E94AECBA1C00E94968330
:1058A0000E94B8C7F6CF11110C94311F0C942A1F17
:1058B00080E00E948EAE0C94601F0E94843FAB017A
:1058C000BC014093D80D5093D90D6093DA0D7093BD
:1058D000DB0D87E29DE00E94EFA4DBCF0E94B67E45
:1058E00088E50E94EB3F882331F05F9A80913F0466
:1058F0008E7F80933F0489E50E94EB3F882339F037
:105900008A9A479A80913F048D7F80933F048AE56D
:105910000E94EB3F882361F080910801809581709F
:1059200080930601479A80913F048B7F80933F04C8
:1059300085E40E94EB3F882309F4ABCF129AA9CFEC
:105940000E94FEBBA6CFF7FAF094F7F8F094D101CD
:10595000CD92DD92ED92FC92139709CB0E94B0E8B4
:1059600098CF0E94B67EBC2C60E08C2D0E9461BA5C
:105970000F3FBFEF1B0759F48C2D0E940BBA31E08B
:1059800020E0892B09F030E0032F122F05C00130F1
:10599000110569F401E010E08B2D0E940BBA80170D
:1059A000910709F476CF80E00E948EAEF5CF00E03B
:1059B00010E0F2CF61E0812F0E9461BA6E2D812F3D
:1059C0000E9433BAF12CB701812F0E949DBA193081
:1059D00009F05FCFF0924104E09240045ACFCD5BD2
:1059E000DF4F0FB6F894DEBF0FBECDBFDF91CF9172
:1059F0001F910F91FF90EF90DF90CF90BF90AF90ED
:105A00009F908F907F906F905F904F903F902F90DE
:105A100008952F923F924F925F926F927F928F9252
:105A20009F92AF92BF92CF92DF92EF92FF920F932D
:105A30001F93CF93DF93CDB7DEB76F970FB6F89470
:105A4000DEBF0FBECDBFC0905C04D0905D04E0907F
:105A50005E04F0905F0420E030E040EA50E4C701CB
:105A6000B6010E9453EF87FD43C120E030E041E9D9
:105A700053E4C701B6010E94F6F518160CF438C1BC
:105A800010927B0F10927A0F809109014091790F4B
:105A9000042E000C550B817021E0822790E04817FE
:105AA000590709F433C08091090181702827209398
:105AB000790F81111BC00E9410A0EBEFFDE08491D3
:105AC0008F01882351F0082E000C990B0E940BA027
:105AD0000F5F1F4FF8018491F4CF8DE090E00E949A
:105AE0000BA08AE090E00E940BA010C0EFEFFDE059
:105AF00084918F01882389F3082E000C990B0E9452
:105B00000BA00F5F1F4FF8018491F4CF80916C0FB1
:105B1000833009F44CC02CF4882351F08130D9F043
:105B20009CC0843009F43EC0853009F44DC095C056
:105B300080915E0B882309F490C081E080936C0F04
:105B40000E944E626093700F7093710F8093720F7A
:105B50009093730F82C080915E0B81117EC0809103
:105B60002A0D882321F082E080936C0F76C010927A
:105B70006C0FE7EFFDE084918F01882351F0082E30
:105B8000000C990B0E940BA00F5F1F4FF80184912E
:105B9000F4CF8DE090E00E940BA08AE090E00E949C
:105BA0000BA05BC08091B90F8823E9F256C08091A9
:105BB0005E0B811152C08091E00A9091E10A891B2D
:105BC0008F7009F4C0C049C080915E0B811145C03F
:105BD0008091E00A9091E10A891B8F7009F4CDC091
:105BE0003CC08DE090E00E940BA08AE090E00E9413
:105BF0000BA010926C0FC0905404D0905504E0900C
:105C00005604F090570420E030E046E153E4C70129
:105C1000B6010E9453EF87FFC1C08BEE9DE09093C9
:105C20004B0480934A040E94818F8FED9DE09093F6
:105C30004B0480934A040E94818F8BED9DE09093EA
:105C40004B0480934A040E94818F8DE99DE09093DC
:105C50004B0480934A040E94818F8091610F909140
:105C6000620F03974CF571E9272E79E0372EE0E6B5
:105C70008E2EEAEE9E2EA12CB12C87EC90E10E9494
:105C8000883E18161906C4F48091610F9091620F36
:105C9000049794F487EC90E10E944C3E8093670F48
:105CA000E091680FF091690F8A3019F08D3009F09A
:105CB000CCC0309709F0D2C08091610F9091620FF3
:105CC000009711F40C94A93D01979093620F809373
:105CD000610F8091630F9091640F019664E070E012
:105CE0000E94B9F69093640F8093630F0C94A93DC2
:105CF00080917A0F90917B0F8136FAEE9F07E8F042
:105D000010927B0F10927A0FE3E0FEE084918F01F6
:105D1000882351F0082E000C990B0E940BA00F5FF6
:105D20001F4FF8018491F4CF8DE090E00E940BA00A
:105D30008AE090E00E940BA0A7CE019690937B0F83
:105D400080937A0FA1CE8091B90F882311F082E061
:105D500001C084E080936C0FE3EFFDE084918F013C
:105D6000882309F416CF082E000C990B0E940BA073
:105D70000F5F1F4FF8018491F3CFEFEEFDE08491A8
:105D80008F01882309F42DCF082E000C990B0E9457
:105D90000BA00F5F1F4FF8018491F3CF20E030E09C
:105DA0004EE353E4C701B6010E9453EF87FF13C0CF
:105DB00087ED9DE090934B0480934A040E94818F6D
:105DC0008BEC9DE090934B0480934A040E94818F5A
:105DD00087EC9DE034CF20E030E048E453E4C70195
:105DE000B6010E9453EF87FF13C083EC9DE09093B0
:105DF0004B0480934A040E94818F88EB9DE090932E
:105E00004B0480934A040E94818F84EB9DE017CF5E
:105E100020E030E048E453E4C701B6010E94F6F503
:105E200087FD13CF80EB9DE090934B0480934A0451
:105E30000E94818F85EA9DE090934B0480934A04F1
:105E40000E94818F81EA9DE0FACE8A3309F431CF36
:105E5000EF35F10514F40C942B3B2BCF8091650F9B
:105E60009091660F20E6289F7001299FF00C112465
:105E700087010F51124FE00FF11F108261E470E0B3
:105E8000C8010E9420F7009711F40C940F3B9093E7
:105E90006B0F80936A0F801B910B8E0D9F1D60E02E
:105EA00070E08E51924F0E9454EB0E9414F5CB018A
:105EB000770FAA0BBB0B8232910510F00C940F3BAD
:105EC000FC018827EE58FF4F8F4F0C94CCF6E8E981
:105ED000FDE084918F01882351F0082E000C990B6E
:105EE0000E940BA00F5F1F4FF8018491F4CF20E0B8
:105EF00030E040E05FE360915C0470915D0480916C
:105F00005E0490915F041EC0E3E9FDE084918F017F
:105F1000882351F0082E000C990B0E940BA00F5FF4
:105F20001F4FF8018491F4CF6091480470914904A7
:105F3000072E000C880B990B0E9459EF20E030E0EF
:105F400040E05FE30E94D0F30E9414F5CB010E9471
:105F50008D410E94C3E08DE090E00E940BA08AE09A
:105F600090E00E940BA00C940F3BEEE8FDE08491C2
:105F70008F01882351F0082E000C990B0E940BA072
:105F80000F5F1F4FF8018491F4CF20E030E040E034
:105F90005FE36091440470914504809146049091C0
:105FA0004704D0CFE9E8FDE084918F01882351F0C8
:105FB000082E000C990B0E940BA00F5F1F4FF801D9
:105FC0008491F4CF6091420470914304B1CF209149
:105FD00040043091410444E6429FC001439F900D2C
:105FE00011246FEF70E00E94B9F68B0165367105E0
:105FF00010F004E610E0E4E8FDE084917F018823DE
:1060000059F0082E000C990B0E940BA0FFEFEF1A1D
:10601000FF0AF7018491F3CFB80180E090E098C7C0
:10602000E0E8FDE084918F01882351F0082E000CF8
:10603000990B0E940BA00F5F1F4FF8018491F4CFC2
:1060400080E290E00E940BA0ECE7FDE084918F01DC
:10605000882351F0082E000C990B0E940BA00F5FB3
:106060001F4FF8018491F4CF60914C0470914D045E
:1060700080914E0490914F040E94C4E080E290E031
:106080000E940BA0E8E7FDE084918F01882351F086
:10609000082E000C990B0E940BA00F5F1F4FF801F8
:1060A0008491F4CF60915004709151048091520416
:1060B000909153040E94C4E080E290E00E940BA003
:1060C000E4E7FDE084918F01882351F0082E000C55
:1060D000990B0E940BA00F5F1F4FF8018491F4CF22
:1060E0006091540470915504809156049091570426
:1060F0000E94C4E080E290E003C680915E0B88239A
:1061000009F450C0EFE6FDE084918F01882351F03F
:10611000082E000C990B0E940BA00F5F1F4FF80177
:106120008491F4CF80915F0B882359F180912A0DDF
:10613000882329F18091D40D9091D50DA091D60D91
:10614000B091D70D0097A105B105C1F0BC01CD01FB
:106150006D597F4F8F4F9F4F24E630E040E050E075
:106160000E9472F36091D80D7091D90D8091DA0D73
:106170009091DB0D0E9472F3822F01C080E090E0CD
:10618000E6CEEBE6FDE084918F01882309F4E3CEAF
:10619000082E000C990B0E940BA00F5F1F4FF801F7
:1061A0008491F3CFE3E6FDE084918F01882309F425
:1061B000D2CE082E000C990B0E940BA00F5F1F4F30
:1061C000F8018491F3CFEEE5FDE084918F018823FF
:1061D00051F0082E000C990B0E940BA00F5F1F4F6F
:1061E000F8018491F4CF8091700F9091710FA0917C
:1061F000720FB091730F892B8A2B8B2B09F477C008
:106200000E944E62A50194010E9472F369017A0115
:106210006091700F7091710F8091720F9091730F58
:10622000A50194010E9472F38601021B130BC801A1
:106230006CE370E00E94A5F6CB019927EAE0F0E05C
:10624000BF010E94B9F6282FCB01BF010E94B9F609
:10625000805D80933704205D2093380410923904C8
:1062600087E394E00E94C3E080E290E00E940BA0EC
:10627000ECE5FDE084917F01882359F0082E000CA5
:10628000990B0E940BA0FFEFEF1AFF0AF701849110
:10629000F3CF80E290E00E940BA0C8016CE370E0B5
:1062A0000E94A5F66AE070E00E94B9F6605D609316
:1062B0003704805D809338041092390487E394E0BA
:1062C0000E94C3E080E290E00E940BA0EAE5FDE0BE
:1062D00084918F01882309F43ECE082E000C990B7F
:1062E0000E940BA00F5F1F4FF8018491F3CF80E253
:1062F00090E00E940BA0E2E5FDE084918F018823ED
:1063000009F429CE082E000C990B0E940BA00F5FF8
:106310001F4FF8018491F3CF10929A0F80910901D9
:1063200080FF11C0EEE4FDE084918F01882309F421
:1063300012CE082E000C990B0E940BA00F5F1F4F6E
:10634000F8018491F3CF83E50E9459E0882341F05E
:106350000E9474E00E9419F570936F0F60936E0FA6
:10636000EAE4FDE084918F01882351F0082E000CAF
:10637000990B0E940BA00F5F1F4FF8018491F4CF7F
:106380008DE090E00E940BA08AE090E00E940BA0BC
:106390008091B80F882309F4A1C280916E0F90916B
:1063A0006F0F8430910509F4D2C040F4892B09F0B5
:1063B0003BC4EEE6FBE084918F010CC08830910570
:1063C00009F47EC10C9709F02FC4E0EFF9E0849145
:1063D0008F012FC2882351F0082E000C990B0E94C8
:1063E0000BA00F5F1F4FF8018491F4CF8DE090E078
:1063F0000E940BA08AE090E00E940BA0E3E6FBE085
:1064000084918F01882351F0082E000C990B0E9473
:106410000BA00F5F1F4FF8018491F4CF8DE090E047
:106420000E940BA08AE090E00E940BA0E7E5FBE051
:1064300084918F01882351F0082E000C990B0E9443
:106440000BA00F5F1F4FF8018491F4CF8DE090E017
:106450000E940BA08AE090E00E940BA0EBE4FBE01E
:1064600084918F01882351F0082E000C990B0E9413
:106470000BA00F5F1F4FF8018491F4CF8DE090E0E7
:106480000E940BA08AE090E00E940BA0EDE3FBE0ED
:1064900084918F01882351F0082E000C990B0E94E3
:1064A0000BA00F5F1F4FF8018491F4CF8DE090E0B7
:1064B0000E940BA08AE090E00E940BA0EFE2FBE0BC
:1064C00084918F01882351F0082E000C990B0E94B3
:1064D0000BA00F5F1F4FF8018491F4CF8DE090E087
:1064E0000E940BA08AE090E00E940BA0E2E2FBE099
:1064F00084918F01882351F0082E000C990B0E9483
:106500000BA00F5F1F4FF8018491F4CF8DE090E056
:106510000E940BA08AE090E00E940BA0E5E1FBE066
:1065200084918F01882351F0082E000C990B0E9452
:106530000BA00F5F1F4FF8018491F4CF8DE090E026
:106540000E940BA08AE090E00E940BA06DC3E7E0E0
:10655000FBE084918F01882351F0082E000C990BE9
:106560000E940BA00F5F1F4FF8018491F4CF8DE0C4
:1065700090E00E940BA08AE090E00E940BA0E9EF5F
:10658000FAE084918F01882351F0082E000C990BBA
:106590000E940BA00F5F1F4FF8018491F4CF8DE094
:1065A00090E00E940BA08AE090E00E940BA0E3EE36
:1065B000FAE084918F01882351F0082E000C990B8A
:1065C0000E940BA00F5F1F4FF8018491F4CF8DE064
:1065D00090E00E940BA08AE090E00E940BA0EDECFE
:1065E000FAE084918F01882351F0082E000C990B5A
:1065F0000E940BA00F5F1F4FF8018491F4CF8DE034
:1066000090E00E940BA08AE090E00E940BA0EBEBD0
:10661000FAE084918F01882351F0082E000C990B29
:106620000E940BA00F5F1F4FF8018491F4CF8DE003
:1066300090E00E940BA08AE090E00E940BA0E9EAA3
:10664000FAE084918F01882351F0082E000C990BF9
:106650000E940BA00F5F1F4FF8018491F4CF8DE0D3
:1066600090E00E940BA08AE090E00E940BA0EBE972
:10667000FAE084918F01882351F0082E000C990BC9
:106680000E940BA00F5F1F4FF8018491F4CF8DE0A3
:1066900090E00E940BA08AE090E00E940BA0EDE841
:1066A000FAE084918F01882309F448CF082E000C6A
:1066B000990B0E940BA00F5F1F4FF8018491F3CF3D
:1066C000E6E8FAE084918F01882351F0082E000C4F
:1066D000990B0E940BA00F5F1F4FF8018491F4CF1C
:1066E0008DE090E00E940BA08AE090E00E940BA059
:1066F000EFE7FAE084918F01882351F0082E000C17
:10670000990B0E940BA00F5F1F4FF8018491F4CFEB
:106710008DE090E00E940BA08AE090E00E940BA028
:10672000E8E6FAE084918F01882351F0082E000CEE
:10673000990B0E940BA00F5F1F4FF8018491F4CFBB
:106740008DE090E00E940BA08AE090E00E940BA0F8
:10675000E1E5FAE084918F01882351F0082E000CC6
:10676000990B0E940BA00F5F1F4FF8018491F4CF8B
:106770008DE090E00E940BA08AE090E00E940BA0C8
:10678000EAE3FAE084918F01882351F0082E000C8F
:10679000990B0E940BA00F5F1F4FF8018491F4CF5B
:1067A0008DE090E00E940BA08AE090E00E940BA098
:1067B000E3E2FAE084918F01882351F0082E000C67
:1067C000990B0E940BA00F5F1F4FF8018491F4CF2B
:1067D0008DE090E00E940BA08AE090E00E940BA068
:1067E000E0E1FAE084918F01882351F0082E000C3B
:1067F000990B0E940BA00F5F1F4FF8018491F4CFFB
:106800008DE090E00E940BA08AE090E00E940BA037
:10681000EDEFF9E084918F01882309F48FCE082EE3
:10682000000C990B0E940BA00F5F1F4FF801849181
:10683000F3CF882351F0082E000C990B0E940BA077
:106840000F5F1F4FF8018491F4CF8DE090E00E941C
:106850000BA08AE090E00E940BA0E3EEF9E08491A7
:106860008F01882351F0082E000C990B0E940BA079
:106870000F5F1F4FF8018491F4CF8DE090E00E94EC
:106880000BA08AE090E00E940BA0E5EDF9E0849176
:106890008F01882351F0082E000C990B0E940BA049
:1068A0000F5F1F4FF8018491F4CF8DE090E00E94BC
:1068B0000BA08AE090E00E940BA0E7ECF9E0849145
:1068C0008F01882309F43ACE082E000C990B0E9400
:1068D0000BA00F5F1F4FF8018491F3CF80915F0BE6
:1068E000882309F478C181E08093DC0D1092DE0DDD
:1068F0001092DD0D8EEA9BE00E9436A78BE1EEEA56
:10690000FBE0DE01159601900D928A95E1F78091EA
:10691000AC0B9091AD0B9C838B838DEE92E09A83B0
:10692000898340E050E0BE016F5F7F4F80E090E0E0
:106930000E9414A2CE0101960E9424AEC090DD0DEB
:10694000D090DE0D00916E0F10916F0FC601801B6D
:10695000910B049720F06801F3E0CF0ED11C58EBA7
:10696000452E59E0552E69EA662E69E0762EC0164E
:10697000D10608F459C10115110509F09DC062E660
:106980007BE08EEA9BE00E94FEA562E273E082E675
:106990009BE00E942BF7892B09F048C0F2018491FB
:1069A00048EBE42E49E0F42E882359F0082E000C21
:1069B000990B0E940BA0FFEFEF1AFF0AF7018491D9
:1069C000F3CF8DE090E00E940BA08AE090E00E945F
:1069D0000BA0F301849139EAE32E39E0F32E8823EA
:1069E00059F0082E000C990B0E940BA0FFEFEF1A34
:1069F000FF0AF7018491F3CF8DE090E00E940BA095
:106A00008AE090E00E940BA080E090E00E94BDE050
:106A1000E9E9F9E084917F012FEFE21AF20A882375
:106A200009F4D6C00E94198FF701F4CFE5E9F9E027
:106A300084917F01882359F0082E000C990B0E9445
:106A40000BA0FFEFEF1AFF0AF7018491F3CF8DE05F
:106A500090E00E940BA08AE090E00E940BA0F10160
:106A6000849121E9E22E29E0F22E882359F0082EA4
:106A7000000C990B0E940BA0FFEFEF1AFF0AF70121
:106A80008491F3CF8DE090E00E940BA08AE090E02B
:106A90000E940BA080E090E00E94BDE0ECE8F9E0ED
:106AA00084917F012FEFE21AF20A882309F490C043
:106AB0000E94198FF701F4CF60E070E0C8010197E0
:106AC0000E94DAA38091600B882309F45AC0EAE897
:106AD000F9E084917F01882359F0082E000C990B6E
:106AE0000E940BA0FFEFEF1AFF0AF7018491F3CF8A
:106AF00082E69BE00E94C3E08DE090E00E940BA044
:106B00008AE090E00E940BA0E8E8F9E084917F0120
:106B1000882359F0082E000C990B0E940BA0FFEF60
:106B2000EF1AFF0AF7018491F3CF8FE69BE00E94F2
:106B3000C3E08DE090E00E940BA08AE090E00E940C
:106B40000BA0C8010E94BDE0E6E8F9E084917F0156
:106B50002FEFE21AF20A882321F00E94198FF70121
:106B6000F5CF9FE6E92E9BE0F92EF70181917F0199
:106B7000882319F00E94198FF8CF8AE00E94198F9C
:106B800027C082E69BE00E94C3E08DE090E00E9477
:106B90000BA08AE090E00E940BA08FE69BE00E9491
:106BA000C3E08DE090E00E940BA08AE090E00E949C
:106BB0000BA0C8010E94BDE08FE6E82E8BE0F82E06
:106BC000F70181917F018823C1F20E94198FF8CFCC
:106BD0000F5F1F4FCCCEE7E7F9E084918F01882348
:106BE00051F0082E000C990B0E940BA00F5F1F4F55
:106BF000F8018491F4CF8DE090E00E940BA08AE030
:106C000090E00E940BA0E8E6F9E084918F018823D0
:106C100009F494CC082E000C990B0E940BA00F5F76
:106C20001F4FF8018491F3CFE6E4FDE084918F01DA
:106C3000882309F490C9082E000C990B0E940BA020
:106C40000F5F1F4FF8018491F3CF80915E0B882373
:106C500039F00E9447A1E3C480915E0B882379F14B
:106C60000E94E9B4DCC480916C0F823019F0833645
:106C700009F0D5C40E944E626093700F7093710F3B
:106C80008093720F9093730F80915F0B882319F09C
:106C900081E080935E0B81E080936C0FE2E4FDE085
:106CA00084918F01882309F456C9082E000C990B92
:106CB0000E940BA00F5F1F4FF8018491F3CF8091CA
:106CC0006C0F833609F0ABC4CBCF89E39DE00E9403
:106CD00047AE8091E00A9091E10A891B8F7009F01C
:106CE0009EC480916C0F823009F499C4833609F0F8
:106CF000CAC495C48DE090E00E940BA08AE090E0A9
:106D00000E940BA028C98091E00A9091E10A891B9A
:106D10008F7009F084C480916C0F823009F47FC4B5
:106D2000833609F47CC480912A0D811100C577C493
:106D300083E50E9459E0811126C083E40E9459E056
:106D4000882309F46CC48091E00A9091E10A891BC0
:106D50008F7009F064C420E030E040E251E46091BB
:106D600054047091550480915604909157040E94E8
:106D700053EF87FF08C086E29DE090934B04809319
:106D80004A040E94818F0E9474E020E030E0A90153
:106D90000E9453EF87FD10C00E9474E020E030E8AD
:106DA00049E853E40E94F6F518164CF00E9474E08E
:106DB0000E9419F5CB0105C080E090E002C083E19C
:106DC00091E00E94E2592BC483E50E9459E0882398
:106DD00009F425C40E9474E020E030E0A9010E947B
:106DE00053EF87FD10C00E9474E020E030E046E1E0
:106DF00053E40E94F6F518164CF00E9474E00E94CD
:106E000019F5CB0105C080E090E002C086E990E072
:106E10000E94C34104C483E50E9459E08823D9F04D
:106E20000E9474E020E030E04FE753E40E94B8EFA6
:106E300020E030E048EC52E40E94ACF40E9419F5E6
:106E40006F3F710519F010F06FEF70E0709341041F
:106E50006093400480C88FEF90E09093410480934A
:106E6000400479C88091E00A9091E10A891B8F70F3
:106E700009F071C880915E0B81116DC80E94C767CF
:106E80005F9A80913F048E7F80933F048A9A479A4D
:106E900080913F048D7F80933F048091080180950D
:106EA000817080930601479A80913F048B7F809385
:106EB0003F04129A50C883E50E9459E0882319F1D3
:106EC0000E9474E020E030E040E252E40E9453EF80
:106ED00087FD0FC00E9474E020E030EC49E754E4E5
:106EE0000E94F6F5181644F00E9474E00E9414F512
:106EF00005C068E270E002C067EE73E070930302C1
:106F0000609302028CC3E0E2FDE084918F0188234C
:106F100051F0082E000C990B0E940BA00F5F1F4F21
:106F2000F8018491F4CFC0900202D09003020D2C9E
:106F3000000CEE08FF08F7FE0DC06DE287EC90E153
:106F40005ED666277727CB016C197D098E099F09CC
:106F50004AE003C04AE0C701B6010E947DE00C94FC
:106F6000AB2F8091E00A9091E10A891B8F7009F0A4
:106F700056C380916C0F823009F451C3833609F0F7
:106F80001CC34DC38091E00A9091E10A891B8F7068
:106F900011F00C94AB2F80916C0F823011F40C9493
:106FA000AB2F833609F0F7C30C94AB2F8091E00A26
:106FB0009091E10A891B8F7009F031C380916C0FA9
:106FC000823009F42CC3833609F03BC528C3809175
:106FD000E00A9091E10A891B8F7009F020C380912B
:106FE0006C0F823009F41BC3833609F060C517C3E8
:106FF0008091E00A9091E10A891B8F7009F00FC31C
:1070000080916C0F823009F40AC3833609F085C57C
:1070100006C380919A0F811103C00E9410A0F2C193
:107020008E3271F580919B0F8E3209F074C1809180
:10703000FF0C882309F4E6C181508093FF0C88235C
:1070400061F090E001974FE1489F9001499F300D1A
:107050001124C9018753944F02C08BE89BE02BE1B8
:10706000FC013496AEEABBE001900D922A95E1F75F
:10707000FC01828193819093AD0B8093AC0BC2C1D4
:107080008C3309F048C164E273E08AE99FE00E9412
:107090002BF7892B21F481E08093B80FB3C163E310
:1070A00073E08AE99FE00E942BF7892B79F4E4E4EE
:1070B000F9E084918F010F5F1F4F882321F00E9418
:1070C000198FF801F6CF87E299E012C16AE473E004
:1070D0008AE99FE00E942BF7892B79F4E3E0F9E03D
:1070E00084918F010F5F1F4F882321F00E94198F19
:1070F000F801F6CF80EF98E0FBC061E673E08AE923
:107100009FE00E942BF7892B79F4E5EDF8E084915C
:107110008F010F5F1F4F882321F00E94198FF80104
:10712000F6CF80ED98E0E4C06FE673E08AE99FE077
:107130000E942BF7892B79F4E0EBF8E084918F0122
:107140000F5F1F4F882321F00E94198FF801F6CF9F
:107150008BEA98E0CDC062E873E08AE99FE00E9484
:107160002BF7892B79F4E0E9F8E084918F010F5F28
:107170001F4F882321F00E94198FF801F6CF87E86E
:1071800098E0B6C060E973E08AE99FE00E942BF7BF
:10719000892B71F404E618E0F8018491882329F022
:1071A0000F5F1F4F0E94198FF7CF8DE598E0A0C0A9
:1071B00066EA73E08AE99FE00E942BF7892B79F455
:1071C000EEE3F8E084918F010F5F1F4F882321F0D9
:1071D0000E94198FF801F6CF87E398E089C068EB29
:1071E00073E08AE99FE00E942BF7892B79F4EFE1A5
:1071F000F8E084918F010F5F1F4F882321F00E94D8
:10720000198FF801F6CF8EE098E072C063EC73E05E
:107210008AE99FE00E942BF7892B79F4E5EFF7E0EC
:1072200084918F010F5F1F4F882321F00E94198FD7
:10723000F801F6CF83EE97E05BC06FEC73E08AE96C
:107240009FE00E942BF7892B79F4E8ECF7E084911A
:107250008F010F5F1F4F882321F00E94198FF801C3
:10726000F6CF86EB97E044C06DED73E08AE99FE0CE
:107270000E942BF7892B79F4ECE9F7E084918F01D8
:107280000F5F1F4F882321F00E94198FF801F6CF5E
:107290008BE897E02DC06AEE73E08AE99FE00E94D8
:1072A0002BF7892B79F4E1E7F7E084918F010F5FE9
:1072B0001F4F882321F00E94198FF801F6CF8CE62A
:1072C00097E016C067EF73E08AE99FE00E942BF712
:1072D000892BA9F4E1E5F7E084918F010F5F1F4F3F
:1072E000882321F00E94198FF801F6CF8CE497E0F3
:1072F00090934B0480934A040E94818F83C065E081
:1073000074E08AE99FE00E942BF7892B09F07AC08C
:107310001092B80F77C01D8218861C821B828DEEDA
:1073200092E09A8389838091B10B811103C06BE84D
:107330007BE002C06AEA7BE06115710519F06C5FC1
:107340007F4F02C060E070E021E04AE95FE0CE01DB
:1073500005960E9465AB882361F18BE1FE013596AD
:10736000AEEABBE001900D928A95E1F72B813C815A
:107370003093AD0B2093AC0B8091FF0C8A3008F05A
:107380003DC091E0980F9093FF0CFFE18F9FC001EB
:107390001124DC01A353B44F4BE1EEEAFBE0019072
:1073A0000D924A95E1F7FC01E753F44F33832283B2
:1073B00025C0EAE6F4E284918F010F5F1F4F882316
:1073C00021F00E94198FF801F6CFE6E3F7E08491EF
:1073D0008F010F5F1F4F882321F00E94198FF80142
:1073E000F6CF0AE91FE0F80181918F01882319F097
:1073F0000E94198FF8CF8AE00E94198FCE01019662
:107400000E9424AE10929A0F8091090180FF07C15B
:10741000E4E6FCE084918F01882311F40C94AB2FF7
:10742000082E000C990B0E940BA00F5F1F4FF80154
:107430008491F2CF8FE40E9459E081110C94AB2F1C
:1074400083E40E9459E00C94AB2F83E50E9459E03D
:10745000811159C08FE40E9459E0882319F08CE211
:107460009CE007C084E50E9459E0882349F084E04D
:107470009CE090934B0480934A040E94818F43C008
:1074800083E40E9459E0882319F08BED9BE0F1CF53
:1074900081E50E9459E0882319F083EB9BE0E9CF56
:1074A00088E40E9459E08823C9F0EFEAFBE0849168
:1074B0008F01882351F0082E000C990B0E940BA01D
:1074C0000F5F1F4FF8018491F4CF8DE090E00E9490
:1074D0000BA08AE090E00E940BA015C08CE40E94F3
:1074E00059E0882381F0EBEAFBE084918F01882347
:1074F00061F3082E000C990B0E940BA00F5F1F4F29
:10750000F8018491F4CFE3E7FCE084918F018823B4
:1075100011F40C94AB2F082E000C990B0E940BA0B9
:107520000F5F1F4FF8018491F2CF8091E00A8091A4
:10753000E10A0C94AB2F83E50E9459E0882309F4FB
:107540006EC083E89BE090934B0480934A040E94B2
:10755000818FE3E7FCE084918F01882311F40C9480
:10756000AB2F082E000C990B0E940BA00F5F1F4F32
:10757000F8018491F2CFEEE7FBE084918F0188233C
:1075800051F0082E000C990B0E940BA00F5F1F4FAB
:10759000F8018491F4CFE9E7FBE084918F0188231F
:1075A00011F40C94AB2F082E000C990B0E940BA029
:1075B0000F5F1F4FF8018491F2CF88E50E9459E0D8
:1075C000811106C089E50E9459E0882309F4D5C0DD
:1075D00088E50E9459E0882341F08AE19DE090937C
:1075E0004B0480934A040E94818F89E50E9459E0F0
:1075F000882341F084E19DE090934B0480934A04FA
:107600000E94818F8AE50E9459E0882341F08EE034
:107610009DE090934B0480934A040E94818F809157
:10762000650F9091660F019664E070E00E94B9F6D4
:107630009093660F8093650F8091610F9091620F18
:1076400001969093620F8093610F1092690F1092D0
:10765000680F0C943D2E4091650F5091660F9F016D
:107660002F5F3F4F3093690F2093680F90E6949FF0
:107670009001959F300D11242F51324FE20FF31FCF
:1076800080830C943D2E00916A0F10916B0F78014E
:1076900024E0E20EF11C6AE270E0C7010E9420F7CC
:1076A000F80124812F3221F4B8016B5F7F4F03C0B2
:1076B0002C3339F4B7018AE99FE00E9434F70C9427
:1076C000AB2F10929A0F009719F0FC01319710829E
:1076D00080916A0F90916B0F40E061E004960E94E8
:1076E00087DE80912A0D882389F0E5E3FDE084910F
:1076F0008F01882309F4FECA082E000C990B0E9402
:107700000BA00F5F1F4FF8018491F3CFE1E3FDE081
:1077100084918F01882309F4EDCA082E000C990B7F
:107720000E940BA00F5F1F4FF8018491F3CF0E94BE
:107730004E626093700F7093710F8093720F9093ED
:10774000730F80915F0B882319F081E080935E0BAB
:1077500081E080936C0FEDE2FDE084918F0188233E
:1077600011F40C94AB2F082E000C990B0E940BA067
:107770000F5F1F4FF8018491F2CF8AE50E9459E014
:10778000811126CF83E40E9459E0882309F447CF72
:107790008AE09DE03ECF86E40E9459E0882309F408
:1077A0004DC10E9474E00E9419F58B0186E09DE0B6
:1077B00090934B0480934A040E94818F88E50E9435
:1077C00059E0882309F451C00E9474E02B013C0168
:1077D0002DEC3CEC4CE45EE30E9453EF9E012F5FE6
:1077E0003F4F7901181674F020E030E0A901C30181
:1077F000B2010E94F6F518162CF41F930F938BEF2D
:107800009CE005C12DEC3CEC4CEC5DEBC301B201FE
:107810000E9453EF18167CF020E030E040E85FEB68
:10782000C301B2010E94F6F518162CF41F930F93B2
:107830008FEE9CE0ECC01F930F93C301B2010E9436
:1078400014F57F936F9385EE9CE09F938F93FF9247
:10785000EF920E9425EF0FB6F894DEBF0FBECDBFAA
:10786000CE0101960E945C8FDFC089E50E9459E03D
:10787000882309F441C00E9474E02B013C012DECE7
:107880003CEC4CE45EE30E9453EFFE0131967F0135
:10789000181674F020E030E0A901C301B2010E9483
:1078A000F6F518162CF41F930F938AED9CE0AFC0E9
:1078B0002DEC3CEC4CEC5DEBC301B2010E9453EFAC
:1078C00018167CF020E030E040E85FEBC301B20125
:1078D0000E94F6F518162CF41F930F938EEC9CE083
:1078E00096C01F930F93C301B2010E9414F57F93BA
:1078F0006F9384EC9CE0A9CF8AE50E9459E088232D
:1079000009F441C00E9474E02B013C012DEC3CECD9
:107910004CE45EE30E9453EFFE0131967F0118169E
:1079200074F020E030E0A901C301B2010E94F6F535
:1079300018162CF41F930F9389EB9CE068C02DEC74
:107940003CEC4CEC5DEBC301B2010E9453EF181606
:107950007CF020E030E040E85FEBC301B2010E9420
:10796000F6F518162CF41F930F938DEA9CE04FC088
:107970001F930F93C301B2010E9414F57F936F937D
:1079800083EA9CE062CF85E40E9459E0882309F4F1
:107990004BC00E9474E02B013C012DEC3CEC4CE40C
:1079A0005EE30E9453EFFE0131967F01181674F0DA
:1079B00020E030E0A901C301B2010E94F6F51816DB
:1079C0002CF41F930F9388E99CE021C02DEC3CEC34
:1079D0004CEC5DEBC301B2010E9453EF18167CF032
:1079E00020E030E040E85FEBC301B2010E94F6F511
:1079F00018162CF41F930F938CE89CE008C0C30169
:107A0000B2010E9414F57F936F9381E89CE09F93ED
:107A10008F93FF92EF920E9425EF0F900F900F909F
:107A20000F900F900F901CCF8DE79CE090934B042C
:107A300080934A040E94818F0C94AB2F00E010E0E9
:107A4000B5CE20E030E040E251E460915404709102
:107A5000550480915604909157040E9453EF87FF7C
:107A600008C086E79CE090934B0480934A040E94F0
:107A7000818F82E390E090934304809342040E94BC
:107A80004A5988EC90E00E94E259E3E7FCE08491D7
:107A90008F01882311F40C94AB2F082E000C990B46
:107AA0000E940BA00F5F1F4FF8018491F2CF20E0DE
:107AB00030E040E251E460915404709155048091AB
:107AC0005604909157040E9453EF87FF08C08CE63C
:107AD0009CE090934B0480934A040E94818F80E540
:107AE00090E090934304809342040E944A5980EFAF
:107AF00090E00E94E259E3E7FCE084918F01882343
:107B000011F40C94AB2F082E000C990B0E940BA0C3
:107B10000F5F1F4FF8018491F2CF80E090E00E9448
:107B2000E25910924304109242040E944A59E8E636
:107B3000FCE084918F01882311F40C94AB2F082E64
:107B4000000C990B0E940BA00F5F1F4FF80184914E
:107B5000F2CF6F960FB6F894DEBF0FBECDBFDF91A8
:107B6000CF911F910F91FF90EF90DF90CF90BF903A
:107B7000AF909F908F907F906F905F904F903F90CD
:107B80002F900895CF92DF92EF92FF92CF93DF93E1
:107B90006B017C01EA0121E338E040EA50EC0E94ED
:107BA000F6F587FD23C022E430E047E553E4C70142
:107BB000B6010E9453EF1816CCF0C880D980EA8035
:107BC000FB802FE632E143E85AEBC701B6010E9481
:107BD000F6F587FD0BC0C1E022E430E047E553E451
:107BE000C701B6010E9453EF18160CF4C0E08C2FA9
:107BF000DF91CF91FF90EF90DF90CF9008950F939A
:107C00001F93CF93DF93FC01A685B7858D010058A4
:107C10001F4FE8018881998101968F779927AD01DF
:107C20004E575F4FEA012881398128173907D1F370
:107C3000E80128813981A20FB31F6C93A685B7850F
:107C4000A058BF4F11969C938E93A689B7892C910B
:107C500081E090E0078C02C0880F991F0A94E2F738
:107C6000822B8C9381E081A30488F589E02D8081AB
:107C70008064808381E090E0DF91CF911F910F912C
:107C80000895FC0181A1882329F0A489B5898C91EC
:107C900086FFFBCF11A20895FC01A485B585FD01E7
:107CA000E058FF4F208131813296808191812817E1
:107CB000390779F080819181A80FB91F8C912081BB
:107CC00031812F5F3F4F2F7733273183208390E01F
:107CD00008958FEF9FEF0895DC011C96ED91FC91C4
:107CE0001D97DF01A058BF4F2D913C91119712961F
:107CF0008D919C9111972817390739F08D919C919E
:107D0000E80FF91F808190E008958FEF9FEF0895AD
:107D1000FC0124853585F901E058FF4F8081918170
:107D200032962081318180589F4F821B930B60E8EF
:107D300070E00C94B9F60895089580E090E00895FD
:107D4000CF92DF92EF92FF92C0904302D090440214
:107D5000E0904502F0904602FC0180819181A28171
:107D6000B3818093430290934402A0934502B09361
:107D700046020E94B8C7C0924302D0924402E092E9
:107D80004502F0924602FF90EF90DF90CF90089569
:107D900080914B0890914C08981759F0E92FF0E02A
:107DA000E553F84F80819F5F9F7790934C0890E058
:107DB00008958FEF9FEF08951F920F920FB60F92C5
:107DC00011240BB60F920F931F932F933F934F9352
:107DD0005F936F937F938F939F93AF93BF93CF9353
:107DE000DF93EF93FF9300914C08D0914B0811E083
:107DF0001D0F1F77C091C6009091E204492F092EF4
:107E0000000C550B660B770B4C30510508F046C043
:107E1000FA018827EC56FF4F8F4F0C94CCF6CD34E7
:107E200041F0CE34B9F481E005C0CA3330F0CD342E
:107E300071F582E08093E20446C0C03308F043C08D
:107E4000C03209F440C0CD3211F53DC0C13329F034
:107E5000C43329F0C032D9F436C083E0EBCF88E0D8
:107E6000E9CFC03321F0C13391F486E0E3CF84E061
:107E7000E1CFC83361F485E0DDCFC23341F487E060
:107E8000D9CFC13321F489E0D5CFC03311F08BE0D5
:107E9000D1CF8AE0CFCFCA30B1F413C0CA3099F441
:107EA000973049F09A3059F0953059F410922402E5
:107EB0001092461106C081E08093710502C00E94B5
:107EC000C7671092E204011731F0ED2FF0E0E5539F
:107ED000F84FC083D12FD0934B08FF91EF91DF91E2
:107EE000CF91BF91AF919F918F917F916F915F9152
:107EF0004F913F912F911F910F910F900BBE0F90BB
:107F00000FBE0F901F90189580914D0890914E08CC
:107F1000009731F04AE050E060E070E00C94A7EC8C
:107F200060E070E0CB010895EFDF97FD0AC0ECDF61
:107F30006F3F71058105910509F02CF4E5DF862F6F
:107F4000089580E008958FEF089580914D089091F5
:107F50004E08892B31F0E8DF91E0811103C090E0F9
:107F600001C091E0892F08950F931F93CF938091C3
:107F70004D0890914E08009711F1FC018F01C191BD
:107F80002C2F2F7DA9F0C53411F0C536B9F7F801B3
:107F9000108260E070E080914D0890914E080E9440
:107FA00054EBF801C083562F472F382F292F0BC0D1
:107FB00060E070E0CF911F910F910C9454EB50E072
:107FC00040E030E020E0652F742F832F922FCF9177
:107FD0001F910F91089581548A3108F042C0E82F13
:107FE000F0E0409138125091391260913A1270913C
:107FF0003B1204C076956795579547958A95D2F7B9
:10800000842F817040FF2FC0E25EFD4E9081992346
:1080100009F1E0913C11F0913D11E90FF11D9081C2
:1080200020ED290F2A3098F09E3211F491810CC076
:108030009D3211F09B3271F4918120ED290F2A308D
:1080400030F09E3239F4928190539A3018F42E2FEA
:108050009F2F02C020E090E020934D0890934E089F
:10806000089580E008950895B6DF882341F081E007
:1080700020914D0830914E08232B09F480E008959B
:1080800080E1ECE4F4E0A4E9B1E101900D928A957D
:10809000E1F708952F923F924F925F926F927F92F5
:1080A0008F929F92AF92BF92CF92DF92EF92FF9208
:1080B0000F931F93CF93DF9300D01F921F92CDB7E2
:1080C000DEB77C018B016A01190180904C0490900D
:1080D0004D04A0904E04B0904F04A5019401FC0102
:1080E00060817181828193810E9453EFF1E0FD8371
:1080F000811112C0209150043091510440915204DA
:1081000050915304F80160817181828193810E94B2
:1081100053EF811101C01D82F601408051806280C1
:108120007380209104023091050240910602509123
:108130000702C301B2010E9453EF882309F453C020
:108140004092040250920502609206027092070269
:1081500020E030E040E450E46091A6077091A7076A
:108160008091A8079091A9070E94ACF469837A8353
:108170008B839C838092941190929511A09296117A
:10818000B09297118091500490915104A0915204A3
:10819000B09153048093981190939911A0939A11E0
:1081A000B0939B11F60180819181A281B38180936C
:1081B0009C1190939D11A0939E11B0939F1180915B
:1081C000580490915904A0915A04B0915B04809393
:1081D000A0119093A111A093A211B093A311CE016D
:1081E0000196AEDD4DDFFD81FF2309F16090A2070E
:1081F0007090A3078090A4079090A507A0909E0779
:10820000B0909F07C090A007D090A1079501A6014C
:10821000B301C4010E94F6F5181614F0530164016D
:1082200020E030E040E251E4B501C6010CC020E09E
:1082300030E040EC5FE36091AA077091AB0780915A
:10824000AC079091AD070E94ACF469837A838B836D
:108250009C8320913004222349F0AB01BC0187E0CC
:108260009EE00E9485CE8AE00E94198FF7018081EE
:108270009181A281B3818093941190939511A093E1
:108280009611B0939711F80180819181A281B381F9
:108290008093981190939911A0939A11B0939B1188
:1082A000F10120813181428153816091A01170914F
:1082B000A1118091A2119091A3110E94D0F360931B
:1082C000A0117093A1118093A2119093A311CE01DC
:1082D000019636DDD5DE0F900F900F900F900F9026
:1082E000DF91CF911F910F91FF90EF90DF90CF9092
:1082F000BF90AF909F908F907F906F905F904F90C6
:108300003F902F90089580E1E4E9F1E1ACE4B4E01E
:1083100001900D928A95E1F708959C0197FD0EC09A
:108320008436910584F064E670E00E94B9F6CB01D2
:108330006AE070E00E94B9F6805D06C03195219533
:1083400031098DE201C080E280933B042A3031057F
:1083500064F0EAE0F0E0C901BF010E94B9F6CB0188
:10836000BF010E94B9F6805D01C080E280933C04A9
:10837000C9016AE070E00E94B9F6805D80933D0417
:108380008BE394E008958D3791051CF02DE780E094
:1083900002C0282F892F20934204809343040C9419
:1083A0004A592F923F924F925F926F927F928F9293
:1083B0009F92AF92BF92CF92DF92EF92FF920F9374
:1083C0001F93CF93DF93CDB7DEB7C455D1090FB656
:1083D000F894DEBF0FBECDBFE6ECF0E184918F01D3
:1083E0000F5F1F4F882321F00E94198FF801F6CFED
:1083F0000E9453B781110C94B24B80E090E0A0E84A
:10840000BFE380938C1190938D11A0938E11B09344
:108410008F1180E090E0A0ECB0E4809390119093F5
:108420009111A0939211B09393118DEC9CECACE45C
:10843000BEE38093881190938911A0938A11B09321
:108440008B1180E090E0A8ECB1E48093DE0490937F
:10845000DF04A093E004B093E1048CE390E09093F8
:10846000DD048093DC0488EC90E09093DB0480933F
:10847000DA041092D9048FE4F7DD882311F074DD5B
:1084800004C060E070E080E190E46BAF7CAF8DAF42
:108490009EAF83E4E9DD882311F057DD02C083E459
:1084A0009ADD61968FAF61978BE4DEDD882311F052
:1084B0004CDD02C08BE48FDD60968FAF609782E465
:1084C000D3DD8823E9F050DD0E9414F57093DD04BC
:1084D0006093DC046115710599F068527109653685
:1084E000710570F0E1E9F0E184918F010F5F1F4F9A
:1084F000882311F40C94B24B0E94198FF801F4CF29
:108500008CE4B2DD882351F12FDD6B017C01609397
:1085100088117093891180938A1190938B1120E0B8
:1085200030E0A9010E94F6F587FD0AC020E030E0A6
:1085300040E050E4C701B6010E9453EF181674F4EE
:10854000E9E6F0E184918F010F5F1F4F882311F45A
:108550000C94B24B0E94198FF801F4CF81E53BDDFA
:10856000882309F440C080914D0890914E08892BD2
:1085700019F4EEE3F0E12BC0F7DC6B017C016093B2
:1085800090117093911180939211909393112DEC0F
:108590003CEC4CE45DE30E94F6F587FD0AC020E068
:1085A00030E040E751E4C701B6010E9453EF1816CE
:1085B000D4F4EDE0F0E184918F010F5F1F4F882329
:1085C00011F40C94B24B0E94198FF801F4CF8491EE
:1085D0008F010F5F1F4F882311F40C94B24B0E9440
:1085E000198FF801F4CF83E53FDD882319F1BCDC56
:1085F0004B015C012DEC3CEC4CEC5DE30E94F6F58C
:1086000087FD0AC020E030E040E85FE3C501B40127
:108610000E9453EF1816ACF4E6EEFFE084918F0150
:108620000F5F1F4F882311F40C94B24B0E94198FD7
:10863000F801F4CF5DEC852E5CEC952EA92C5EE361
:10864000B52E80E5C8DC882309F443C080914D082D
:1086500090914E08892B71F4EEEAFFE084918F012E
:108660000F5F1F4F882311F40C94B24B0E94198F97
:10867000F801F4CF8091D9048F5F8093D90474DC22
:108680006B017C016093DE047093DF048093E0044F
:108690009093E10420E030E0A9010E94F6F587FD07
:1086A0000AC020E030E048EC51E4C701B6010E9466
:1086B00053EF181674F4E6E8FFE084918F010F5F22
:1086C0001F4F882311F40C94B24B0E94198FF801AC
:1086D000F4CF86E4C9DC882319F146DC6B017C0108
:1086E00020E030E040E85FE30E94F6F587FD0AC035
:1086F00020E030E040E850E4C701B6010E9453EFAB
:108700001816A4F4EDE5FFE084918F010F5F1F4F71
:10871000882311F40C94B24B0E94198FF801F4CF06
:10872000C12CD12C40EEE42E4FE3F42EA70196018C
:10873000C701B6010E94B8EF9B01AC0160E070E098
:1087400084E490E40E94ACF420918C1130918D115E
:1087500040918E1150918F110E94B8EF2B013C0176
:10876000A5019401C501B4010E94B8EFA7019601CB
:108770000E94B8EF2CEE31E548EB5DE30E94ACF4CB
:108780009B01AC01C301B2010E94B8EF60938C1150
:1087900070938D1180938E1190938F1188E464DC17
:1087A0008823C9F0E1DB0E9414F57093DB04609329
:1087B000DA04655A71096437710568F0EFE2FFE089
:1087C00084918F010F5F1F4F882309F4CBC70E944C
:1087D000198FF801F5CF85E5FEDB8823E9F00E94CB
:1087E0004E62611571058105910511F00E944BEBF8
:1087F00080914D0890914E08892B11F0B5DB04C093
:1088000060E070E088E492E46093D5047093D6044D
:108810008093D7049093D80482E5DDDB81110DC0ED
:10882000EBEFFEE084918F010F5F1F4F882309F467
:1088300099C70E94198FF801F5CF80914D0890914A
:108840004E08892BA9F060DB2F967FAF6EAF2F9774
:10885000161617069CF0E7ECFEE084918F010F5F7F
:108860001F4F882309F47EC70E94198FF801F5CFA6
:108870008AE190E02F969FAF8EAF2F9788E5F4DBCB
:10888000882361F071DB209124043091250440910C
:108890002604509127040E94CFF308C060914C0435
:1088A00070914D0480914E0490914F046093D104D7
:1088B0007093D2048093D3049093D40489E5D4DBDD
:1088C000882361F051DB20912804309129044091E4
:1088D0002A0450912B040E94CFF308C060915004E9
:1088E0007091510480915204909153046093CD048F
:1088F0007093CE048093CF049093D0046091D10400
:108900007091D2048091D3049091D4044DEC54E042
:1089100039D981110DC0EDE9FEE084918F010F5F1F
:108920001F4F882309F41EC70E94198FF801F5CF45
:1089300084E451DB91E089270E94418520E030E00A
:1089400040EA50E4609154047091550480915604BB
:10895000909157040E9453EF87FF14C0198A1A8A16
:108960001B8A1C8A80E090E0A0EAB0E489839A83A5
:10897000AB83BC83BE016F5E7F4FCE0101960E9428
:10898000A586C1DC0E944E626B017C01A8E8CA0E7C
:10899000A3E1DA1EE11CF11C8091DC049091DD045E
:1089A000F2DC6091DC047091DD04072E000C880B72
:1089B000990B0E9459EF9B01AC01609144047091A6
:1089C000450480914604909147040E94CFF34B01E7
:1089D0005C0120E030E0A9010E94F6F587FF04C0A9
:1089E000B7FAB094B7F8B09420E030E040E450E437
:1089F000C501B4010E94F6F51816FCF40E944E62FF
:108A0000DC01CB018C199D09AE09BF09B7FD0FC070
:108A10000E944E626B017C01B8E8CB0EB3E1DB1E15
:108A2000E11CF11C0E9490588AE00E94198F80E09E
:108A30000E948EAE0E944B93B4CF8091DA04909145
:108A4000DB040E94E2596091DA047091DB04072E86
:108A5000000C880B990B0E9459EF9B01AC016091AF
:108A60005C0470915D0480915E0490915F040E94AB
:108A7000CFF34B015C0120E030E0A9010E94F6F544
:108A800087FF04C0B7FAB094B7F8B09420E030E0A4
:108A900040E450E4C501B4010E94F6F51816FCF458
:108AA0000E944E62DC01CB018C199D09AE09BF0901
:108AB000B7FD0FC00E944E626B017C01E8E8CE0E4C
:108AC000E3E1DE1EE11CF11C0E9490588AE00E9446
:108AD000198F80E00E948EAE0E944B93B4CF10920B
:108AE00058041092590410925A0410925B0488E5BD
:108AF00094E00E94F2B68091D904882399F1C0DAFB
:108B00002091A0113091A1114091A2115091A31177
:108B10006091DE047091DF048091E0049091E104A3
:108B20000E94D0F36093A0117093A1118093A211C1
:108B30009093A31120E030E040E751E46091AA0750
:108B40007091AB078091AC079091AD070E94ACF497
:108B500069837A838B839C83CE010196F1D890DA66
:108B60000E94FFB480E2EDEAF4E0DF01282F1D92BD
:108B70002A95E9F7EDE8F4E0DF01282F1D922A9508
:108B8000E9F7EDE6F4E0DF011D928A95E9F778DA7E
:108B90008091881190918911A0918A11B0918B11C7
:108BA00080939C1190939D11A0939E11B0939F115F
:108BB00019821A821B821C829E012F5F3F4F4CE953
:108BC00051E168E971E184E991E164DA9E01255C93
:108BD0003F4F4CE951E168E971E184E991E15ADAEA
:108BE0006196BFAD6197BB2329F060E574E08CE42A
:108BF00094E004C06DEC74E081ED94E00E948FE19C
:108C00003FAF2D962FAF2D972D96EFAD2D97E7FD0A
:108C100082C4FFADF7FD7FC424E0E202F00111241D
:108C2000E65DF44F40805180628073803FAD84E008
:108C30003802F0011124EA5EF44FD080C180328006
:108C400023808D2D9C2DA32DB22D8FAB98AFA9AF76
:108C5000BAAFAE01495C5F4FB201C3010E94C23D91
:108C6000882309F45AC420E030E040EA50E4B2011D
:108C7000C3010E94D0F3F62E072F182FE92E862F5E
:108C8000902FA12FBE2D8BAB9CABADABBEAB8D2D72
:108C90009C2DA32DB22D8FA798ABA9ABBAAB2D9667
:108CA0009FAD2D97911152C0AFADA11105C05F2DA1
:108CB000402F312F2E2D04C0542D452D362D272D1C
:108CC000852F942FA32FB22F8BAB9CABADABBEAB3C
:108CD000BFADB43034F4F42C052D162DE72CBB2396
:108CE00069F020E030E040EA50E46D2D7C2D832DCA
:108CF000922D0E94CFF3362F272F03C09601832D8C
:108D0000922D432F522FBC014FA758AB69AB7AABC2
:108D1000EFADE4300CF0A7C020E030E040EA50E4D2
:108D20006D2D7C2D832D922D0E94D0F321966FAF57
:108D3000219723967FAF239725968FAF2597279668
:108D40009FAF2797FFADF11185C099C02D962FAD2C
:108D50002D9724300CF453C03FAD34305CF020E04C
:108D600030E040EA50E4B201C3010E94CFF3362F55
:108D7000272F03C0342D252DC301432F522FBC01B3
:108D80004BAB5CAB6DAB7EAB8FAD8111E2C420E031
:108D900030E040EA50E4B201C3010E94CFF3F62E66
:108DA000072F182FE92E20E030E040EA50E46D2D27
:108DB0007C2D832D922D0E94D0F36FA778AB89ABC9
:108DC0009AAB9FAD992309F44EC020E030E040EA11
:108DD00050E46D2D7C2D832D922D0E94CFF3219692
:108DE0006FAF219723967FAF239725968FAF259757
:108DF00027969FAF2797AFADA43064F140C0BFADB9
:108E0000B1110DC020E030E040EA50E4B201C301EE
:108E10000E94CFF3F62E072F182FE92E0FC0EFADCB
:108E2000E430B4F120E030E040EA50E4B201C301A4
:108E30000E94CFF36BAB7CAB8DAB9EAB2196DFAECC
:108E400021972396CFAE239725963FAE2597279659
:108E50002FAE279732ED832E33E5932E3BE7A32EDB
:108E600031E4B32E29C02196DFAE21972396CFAEF1
:108E7000239725963FAE259727962FAE279722ED6D
:108E8000822E23E5922E2BEFA22E20E4B22E14C0C8
:108E90002196DFAE21972396CFAE239725963FAE3E
:108EA000259727962FAE279792ED892E93E5992E39
:108EB0009BEFA92E91E4B92E8BA99CA9ADA9BEA9BF
:108EC0002C968CAF9DAFAEAFBFAF2C979C01AD0180
:108ED000B201C3010E94CFF3698B7A8B8B8B9C8B81
:108EE0004FA458A869A87AA8A30192016D2D7C2DE2
:108EF000832D922D0E94CFF36D8B7E8B8F8B988F5D
:108F00002C962CAD3DAD4EAD5FAD2C9760914C04D1
:108F100070914D0480914E0490914F040E94CFF3C4
:108F20002C966CAF7DAF8EAF9FAF2C97A3019201B3
:108F300060915004709151048091520490915304B7
:108F40000E94CFF32B013C018F2D902FA12FBE2D1E
:108F500089839A83AB83BC8321968FAD2197239617
:108F60009FAD23972596AFAD25972796BFAD279741
:108F70008D839E83AF83B8878091881190918911EA
:108F8000A0918A11B0918B1189879A87AB87BC8792
:108F90002DEC3CEC4CEC5CE3C501B4010E94B8EF55
:108FA00020918C1130918D1140918E1150918F1123
:108FB0000E94B8EF209158043091590440915A040E
:108FC00050915B040E94D0F36D877E878F87988BCA
:108FD0002C962CAD3DAD4EAD5FAD2C97CA01B901BD
:108FE0000E94B8EF6B017C01A3019201C301B201A1
:108FF0000E94B8EF9B01AC01C701B6010E94D0F3FB
:1090000020E030E040E050E40E94F6F518160CF045
:1090100046C00E94FFB41BA21CA21DA21EA220E0FB
:1090200030E040E05FE3609154047091550480911A
:109030005604909157040E94D0F36F8F78A389A3B0
:109040009AA39E012D5D3F4FAE01415E5F4F60E5EB
:1090500074E08CE494E01ED81BA21CA21DA21EA2E8
:1090600020E030E040E05FE3609188117091891169
:1090700080918A1190918B110E94D0F36F8F78A309
:1090800089A39AA39E012D5D3F4FAE01415E5F4FC4
:10909000BE01615D7F4FCE01C3960E944A401F8E84
:1090A00018A219A21AA29E01215E3F4F48E851E181
:1090B000BE01615D7F4FCE01C3960E944A400E946F
:1090C0002BB540904302509044026090450270904E
:1090D0004602E090A207F090A3070091A407109128
:1090E000A507A0909E07B0909F07C090A007D090C2
:1090F000A1079501A601B701C8010E94F6F518164F
:1091000014F47501860120E030E040E251E4B7013B
:10911000C8010E94ACF460934302709344028093B0
:1091200045029093460240E0BE016F5E7F4FCE0144
:1091300001960E94A6C3409243025092440260925C
:109140004502709246020E944040AAE2BBE024968B
:10915000BFAFAEAF249722961FAE1EAE229701E09E
:1091600010E021960FAC219702C0000F111F0A9446
:10917000E2F72296EEADFFAD229731962296FFAF31
:10918000EEAF229721E030E021960FAC219702C08C
:10919000220F331F0A94E2F763963FAF2EAF639717
:1091A0008DE6282E84E0382E8DEA94E02A969FAF33
:1091B0008EAF2A97ADE8B4E02896BFAFAEAF289740
:1091C000E6E1FBE02696FFAFEEAF26972A962EAD9E
:1091D0003FAD2A9765963FAF2EAF6597D9018D9128
:1091E0009C919C0120233123232B09F4ADC063966D
:1091F000EEADFFAD63978E239F23892B09F4A4C0A6
:109200002896AEADBFAD28978D919C918023912378
:10921000892B09F099C020E030E040E050E424962A
:10922000AEADBFAD24976D917D918D919C910E94C3
:10923000D0F36B017C0120E030E040E050E4249664
:10924000EEADFFAD249764817581868197810E9480
:10925000CFF34B015C0120E030E040E850ECC70167
:10926000B6010E9453EF87FD6EC120E030E046E575
:1092700053E4C701B6010E94F6F5181634F4C12C68
:10928000D12CB6E5EB2EB3E4FB2ECBA6DCA6EDA6E7
:10929000FEA62696AEADBFAD26974D905D906D9023
:1092A0007C9020E030E040E85FE3C301B2010E941F
:1092B00053EF87FD4FC120E030E046E553E4C301A2
:1092C000B2010E94F6F5181634F4412C512CF6E543
:1092D0006F2EF3E47F2E4F8E58A269A27AA24FA27E
:1092E00058A669A67AA620E030E040E850ECC50117
:1092F000B4010E9453EF87FD34C120E030E046E521
:1093000053E4C501B4010E94F6F5181634F4812C1B
:10931000912C76E5A72E73E4B72E8BA29CA2ADA26A
:10932000BEA2AE01495D5F4FC701B6010E94C23DBA
:1093300081111EC12896EEADFFAD289780819181E5
:10934000802B912B918380832A962EAD3FAD2A9757
:109350002E5F3F4F2A963FAF2EAF2A976596AEAD50
:10936000BFAD65978D919C9180239123892B09F442
:10937000A6C0F9018081918180239123892B09F472
:109380009EC0F1018081918180239123892B09F076
:1093900096C020E030E040E050E42696AEADBFAD90
:1093A00026976D917D918D919C910E94D0F32B0118
:1093B0003C0120E030E040E050E42696EEADFFAD09
:1093C000269764817581868197810E94CFF34B0136
:1093D0005C012496AEADBFAD2497CD90DD90ED90AD
:1093E000FC9020E030E040E850ECC701B6010E945C
:1093F00053EF87FDFDC020E030E046E553E4C701B0
:10940000B6010E94F6F5181634F4C12CD12C56E59D
:10941000E52E53E4F52ECBA2DCA2EDA2FEA2CBA654
:10942000DCA6EDA6FEA620E030E040E85FE3C30145
:10943000B2010E9453EF87FDE2C020E030E046E534
:1094400053E4C301B2010E94F6F5181634F4412C1E
:10945000512C36E5632E33E4732E4FA258A669A62D
:109460007AA620E030E040E85FE3C501B4010E9445
:1094700053EF87FDCBC020E030E046E553E4C50163
:10948000B4010E94F6F5181634F4812C912C96E55F
:10949000A92E93E4B92E8F8E98A2A9A2BAA2AE01EA
:1094A000495D5F4FC701B6010E94C23D8111B5C041
:1094B000F10180819181802B912B91838083F2E057
:1094C0002F0E311C28962EAD3FAD28972E5F3F4FB3
:1094D00028963FAF2EAF289726968EAD9FAD269744
:1094E000049626969FAF8EAF269797E7291694E0AD
:1094F000390609F06BCE2496AEADBFAD2497149615
:109500002496BFAFAEAF24972296EEADFFAD229763
:10951000359709F024CE0E944B932F962EAD3FAD88
:109520002F97215031092F963FAF2EAF2F97232B26
:1095300009F4B3C02D963FAD2D9737FDAEC08FAD6A
:1095400087FF4ECBAAC0C12CD12CA0E8EA2EA0ECFC
:10955000FA2E9BCE412C512CE0E86E2EEFE37E2EAE
:10956000BACE812C912C60E8A62E60ECB62ED5CE1A
:10957000AE01415E5F4FC501B4010E94C23D882328
:1095800009F4D8CE80913004882321F1B701A601D7
:1095900087E79EE00E9485CE4FA158A569A57AA5D0
:1095A00081E79EE00E9485CE4BA15CA16DA17EA1CA
:1095B00087E69EE00E9485CE4F8D58A169A17AA1D1
:1095C00081E69EE00E9485CE89E20E94198F8AE0A2
:1095D0000E94198F9E01215E3F4FAE014D5D5F4F8E
:1095E000BE01695D7F4FCE018B960E945BB5A2CE16
:1095F000C12CD12C40E8E42E40ECF42E0CCF412CB1
:10960000512C20E8622E2FE3722E27CF812C912C33
:1096100080E8A82E8FE3B82E3ECFAE01415E5F4FAB
:10962000C701B6010E94C23D882309F441CF809151
:109630003004882321F1B701A6018DE39EE00E944A
:1096400085CE4FA158A569A57AA587E39EE00E9423
:1096500085CE4BA15CA16DA17EA18DE29EE00E9412
:1096600085CE4F8D58A169A17AA187E29EE00E9424
:1096700085CE89E20E94198F8AE00E94198F9E018F
:10968000215E3F4FAE014D5D5F4FBE01695D7F4F73
:10969000CE018B960E945BB50BCF0E94FFB480E099
:1096A00090E0A0EAB0E480939C1190939D11A09368
:1096B0009E11B0939F1119821A821B821C829E01F7
:1096C0002F5F3F4F4CE951E168E971E184E991E195
:1096D0000E944A408091D1049091D204A091D30479
:1096E000B091D4048093941190939511A093961106
:1096F000B09397118091CD049091CE04A091CF04A6
:10970000B091D0048093981190939911A0939A11DD
:10971000B0939B1119821A821B821C829E012F5FBB
:109720003F4F4CE951E168E971E184E991E10E9420
:109730004A406096FFAD6097F11114C01092430447
:10974000109242040E944A5980E090E00E94E2593F
:1097500009C02FADF42C052D162DE72C24300CF06C
:1097600034CB21CBCC5ADF4F0FB6F894DEBF0FBEFF
:10977000CDBFDF91CF911F910F91FF90EF90DF90C0
:10978000CF90BF90AF909F908F907F906F905F90A1
:109790004F903F902F9008951F920F920FB60F9207
:1097A00011240BB60F922F933F938F939F93EF93B8
:1097B000FF9320913F103091401080914110909183
:1097C00042102817390731F4809131018F7D809341
:1097D000310114C0E0914110F0914210E154F04F7A
:1097E0002081809141109091421001968F779927A6
:1097F000909342108093411020933601FF91EF9196
:109800009F918F913F912F910F900BBE0F900FBEA4
:109810000F901F9018951F920F920FB60F92112460
:109820000BB60F922F934F935F938F939F93EF936A
:10983000FF938091300182FD1CC020913601809100
:10984000C3109091C4104091C5105091C61001965C
:109850008F7799274817590771F0E091C310F0915D
:10986000C410ED5BFF4E20839093C4108093C3100F
:1098700002C080913601FF91EF919F918F915F918E
:109880004F912F910F900BBE0F900FBE0F901F9016
:1098900018952F923F924F925F926F927F928F9284
:1098A0009F92AF92BF92CF92DF92EF92FF920F936F
:1098B0001F93CF93DF93CDB7DEB762970FB6F894BF
:1098C000DEBF0FBECDBFF8948FEF9FEF909389005E
:1098D000809388002AE02A8B212C312C7894809167
:1098E000350590913605A0913705B0913805892B43
:1098F0008A2B8B2B09F00FC280913B058823E1F066
:1099000010923B058091390590913A05892B09F415
:1099100002C21092ED0410923A051092390590910E
:10992000E00A8091E10A981709F4F5C18091E10AF3
:109930008F5F8F708093E10A8091390590913A058D
:10994000892B09F4E8C140913105509132056091AD
:1099500033057091340580912D0590912E05A091CD
:109960002F05B09130050091240510E020E030E093
:10997000841B950BA60BB70B081719072A073B0783
:1099800010F4D901C801E82F840F951FA61FB71F37
:109990008093310590933205A0933305B09334053D
:1099A0002091840030918500245E3F4F409109054D
:1099B00050910A0560910B0570910C058091F90496
:1099C0009091FA04A091FB04B091FC04840F951FC0
:1099D000A61FB71F8093090590930A05A0930B0556
:1099E000B0930C05B7FD1CC0889A809168119091C6
:1099F0006911A0916A11B0916B1140910802042E77
:109A0000000C550B660B770B840F951FA61FB71F15
:109A10008093681190936911A0936A11B0936B11B0
:109A200040910D0550910E0560910F057091100544
:109A30008091FD049091FE04A091FF04B091000577
:109A4000840F951FA61FB71F80930D0590930E05D9
:109A5000A0930F05B0931005B7FD1CC08E9A80919E
:109A60006C1190916D11A0916E11B0916F11409198
:109A70000902042E000C550B660B770B840F951F03
:109A8000A61FB71F80936C1190936D11A0936E1158
:109A9000B0936F114091110550911205609113051B
:109AA000709114058091010590910205A091030524
:109AB000B0910405840F951FA61FB71F8093110551
:109AC00090931205A0931305B0931405B7FD3FC002
:109AD0008091E704F0910A028823C9F08091E5049F
:109AE00082FF02C0F7FD06C08091E404882311F4D0
:109AF0000C94F0558091E5049091E60493FF02C028
:109B0000F7FD0CC08091E304811108C006C080916C
:109B10000B018095887080930901419A40917011E2
:109B20005091711160917211709173118F2FFF0F0D
:109B3000990BAA0BBB0B840F951FA61FB71F809311
:109B4000701190937111A0937211B09373114091A1
:109B500015055091160560911705709118058091B3
:109B6000050590910605A0910705B0910805840FA1
:109B7000951FA61FB71F8093150590931605A093F8
:109B80001705B0931805B7FD3AC040917411509174
:109B900075116091761170917711C0900B020C2CA9
:109BA000000CDD08EE08FF084C0D5D1D6E1D7F1DCD
:109BB00040937411509375116093761170937711DF
:109BC0004091F5045091F6046091F7047091F80407
:109BD000841B950BA60BB70B809315059093160568
:109BE000A0931705B09318059091E8048091220581
:109BF00093FF02C0815001C08F5F80932205809146
:109C0000090590910A05A0910B05B0910C05B7FDCF
:109C100015C04091F5045091F6046091F7047091DD
:109C2000F804841B950BA60BB70B80930905909342
:109C30000A05A0930B05B0930C05889880910D053B
:109C400090910E05A0910F05B0911005B7FD15C0BC
:109C50004091F5045091F6046091F7047091F80476
:109C6000841B950BA60BB70B80930D0590930E05E7
:109C7000A0930F05B09310058E98809111059091D7
:109C80001205A0911305B0911405B7FD3AC040919B
:109C9000F5045091F6046091F7047091F804841B68
:109CA000950BA60BB70B8093110590931205A0930B
:109CB0001305B09314058091E7048823E1F08091A7
:109CC000E50482FF04C080910A0287FD05C08091EF
:109CD000E404882309F48CC78091E5049091E6049C
:109CE00093FF04C080910A0287FD0BC08091E304BA
:109CF000811107C005C080910B0188708093090114
:109D00004198E15041F08091840090918500821744
:109D10009307C8F34BCE8091150290911602A09143
:109D20001702B0911802892B8A2B8B2B09F08AC05D
:109D300080912305882309F453C0809031059090C9
:109D40003205A0903305B0903405C0901E05D09028
:109D50001F05E0902005F090210540912205C814D0
:109D6000D904EA04FB0480F48091EE049091EF049E
:109D70002091F2043091F3042817390728F4415058
:109D800040932205019714C08C149D04AE04BF04B7
:109D9000E0F48091EE049091EF042091F004309172
:109DA000F1048217930788F44F5F409322050196D0
:109DB0009093EF048093EE044091110250911202AF
:109DC00060911302709114020EC08FEF9FEFDC01BF
:109DD0008093110290931202A0931302B093140285
:109DE0004FEF5FEFBA018091220587FD02C0169AFE
:109DF00001C0169880918400909185004C96209126
:109E000022052223B9F0149A2091220527FF02C0CF
:109E10002F5F01C021502093220514982091220524
:109E2000222369F320918400309185002817390797
:109E3000C8F3E5CF409315025093160260931702C2
:109E4000709318028091350590913605A0913705E1
:109E5000B0913805892B8A2B8B2B09F046C6A0912F
:109E60003905B0913A05109711F40C949A578090E7
:109E7000310590903205A0903305B09034054091A3
:109E80002D0550912E0560912F0570913005841697
:109E90009506A606B706D8F01092ED0410923A0582
:109EA000109239059091E00A8091E10A981711F417
:109EB0000C949A578091E10A8F5F8F708093E10A2A
:109EC00040EDC42E47E0D42EE12CF12C1AC4409171
:109ED000290550912A0560912B0570912C05481594
:109EE00059056A057B0508F4AAC1409125055091E2
:109EF00026056091270570912805D6960D911D9134
:109F00002D913C91D997401751076207730708F0CC
:109F100077C1411551056105710549F48090E90447
:109F20009090EA04A090EB04B090EC0464C1E12CA2
:109F3000F980842E952F862F0A811B81FD81EE8169
:109F40003F8128859C80E0911119E89D912CFF2785
:109F500030911219389D900CF11D10901319189C16
:109F6000F00DE99F900CF11D399FF00DE89FF00D69
:109F7000092D1F2F099DE12D332722270F9FE00D6B
:109F8000311D2E1D199DE00D311D2E1D1F9F300D01
:109F9000211D032F122F099DF12C332722270F9FFC
:109FA000F00C311D2E1D199DF00C311D2E1D1F9F13
:109FB000300D211D032F122FEE278090E904909180
:109FC000EA048091EB0400906C040E2809F483C02D
:109FD00030916804309FE1198E089E098E09209106
:109FE0006904209FE01981089E098E09F0906A0497
:109FF000F09E801891098E09319FE01981089E0911
:10A000008E09219F801891098E09F19E901981096E
:10A01000099DF12C332722270F9FF00C311D2E1D97
:10A02000199DF00C311D2E1D1F9F300D211D032F7A
:10A03000122F30916404309FE10D8E1C9E1D8E1DE9
:10A0400020916504209FE00D811C9E1D8E1DF090C7
:10A050006604F09E800C911D8E1D319FE00D811CC9
:10A060009E1D8E1D219F800C911D8E1DF19E900DB9
:10A07000811D099DF12C332722270F9FF00C311DE4
:10A080002E1D199DF00C311D2E1D1F9F300D211D01
:10A09000032F122F30916004309FE1198E089E0922
:10A0A0008E0920916104209FE01981089E098E0984
:10A0B000F0906204F09E801891098E09319FE0199A
:10A0C00081089E098E09219F801891098E09F19EB1
:10A0D0009019810982C030916804309FE10D8E1C77
:10A0E0009E1D8E1D20916904209FE00D811C9E1DE8
:10A0F0008E1DF0906A04F09E800C911D8E1D319F84
:10A10000E00D811C9E1D8E1D219F800C911D8E1DBA
:10A11000F19E900D811D099DF12C332722270F9F61
:10A12000F00C311D2E1D199DF00C311D2E1D1F9F91
:10A13000300D211D032F122F30916404309FE1193F
:10A140008E089E098E0920916504209FE0198108E0
:10A150009E098E09F0906604F09E801891098E0980
:10A16000319FE01981089E098E09219F801891096D
:10A170008E09F19E90198109099DF12C3327222720
:10A180000F9FF00C311D2E1D199DF00C311D2E1D41
:10A190001F9F300D211D032F122F30916004309F1F
:10A1A000E10D8E1C9E1D8E1D20916104209FE00DEF
:10A1B000811C9E1D8E1DF0906204F09E800C911DEE
:10A1C0008E1D319FE00D811C9E1D8E1D219F800CD8
:10A1D000911D8E1DF19E900D811D11249C82F9828E
:10A1E0000A831B83FD83EE833F832887912C992A62
:10A1F000A12CB12CA82A83EF98E121E0298B14C06F
:10A20000D2968D909D90AD90BC90D597F4CFB6949A
:10A21000A79497948794D988DD0CD98A049629E16C
:10A220008F30920709F4EAC4FC010591159125913C
:10A230003491081519052A053B0548F3DFC4409001
:10A240001E0550901F056090200570902105481450
:10A2500059046A047B0408F0C3C180911D05811173
:10A2600021C0FD01EE5BFF4FE080F1800281138190
:10A2700078962081318142815381D2966D917D9172
:10A280008D919C91D5970E94B4CDDD24D394D0922A
:10A290001D05E0913905F0913A0582A993A9A4A979
:10A2A000B5A98EC14091190550911A0560911B0501
:10A2B00070911C05DA960D911D912D913C91DD97C1
:10A2C000401751076207730708F073C14115510524
:10A2D0006105710549F48091E9049091EA04A09127
:10A2E000EB04B091EC046CC1F0E0E985842F352FCC
:10A2F000262FAA857B856C855D85BE854F859889CF
:10A30000B0911119B89F612D552740911219489F9E
:10A31000600D511D10901319189E500DB39F600DC4
:10A32000511D439F500DB29F500DA62F752FA69F14
:10A33000B12D44279927A59FB00D411D9F1F769FE2
:10A34000B00D411D9F1F759F400D911DA42F792FAA
:10A35000A69FE12D44279927A59FE00D411D9F1F32
:10A36000769FE00D411D9F1F759F400D911DA42FED
:10A37000792FBB278091E9043091EA042091EB0406
:10A3800000906C040F2A09F483C0409168044A9F2E
:10A39000B1198F0B3F0B2F0B909169049A9FB01945
:10A3A00081093F0B2F0BE0916A04EA9F8019310964
:10A3B0002F0B479FB01981093F0B2F0B979F8019D7
:10A3C00031092F0BE79F30192109A69FE12D442762
:10A3D0009927A59FE00D411D9F1F769FE00D411D10
:10A3E0009F1F759F400D911DA42F792F40916404EC
:10A3F0004A9FB10D8F1F3F1F2F1F909165049A9F99
:10A40000B00D811D3F1F2F1FE0916604EA9F800D54
:10A41000311D2F1F479FB00D811D3F1F2F1F979F7D
:10A42000800D311D2F1FE79F300D211DA69FE12DAF
:10A4300044279927A59FE00D411D9F1F769FE00DA2
:10A44000411D9F1F759F400D911DA42F792F409195
:10A4500060044A9FB1198F0B3F0B2F0B9091610441
:10A460009A9FB01981093F0B2F0BE0916204EA9F7C
:10A47000801931092F0B479FB01981093F0B2F0B12
:10A48000979F801931092F0BE79F3019210982C04E
:10A49000409168044A9FB10D8F1F3F1F2F1F90915D
:10A4A00069049A9FB00D811D3F1F2F1FE0916A0420
:10A4B000EA9F800D311D2F1F479FB00D811D3F1F4B
:10A4C0002F1F979F800D311D2F1FE79F300D211DDE
:10A4D000A69FE12D44279927A59FE00D411D9F1FB1
:10A4E000769FE00D411D9F1F759F400D911DA42F6C
:10A4F000792F409164044A9FB1198F0B3F0B2F0BAA
:10A50000909165049A9FB01981093F0B2F0BE09140
:10A510006604EA9F801931092F0B479FB019810902
:10A520003F0B2F0B979F801931092F0BE79F301995
:10A530002109A69FE12D44279927A59FE00D411DE4
:10A540009F1F769FE00D411D9F1F759F400D911D20
:10A55000A42F792F409160044A9FB10D8F1F3F1F98
:10A560002F1F909161049A9FB00D811D3F1F2F1FD7
:10A57000E0916204EA9F800D311D2F1F479FB00DAF
:10A58000811D3F1F2F1F979F800D311D2F1FE79F9C
:10A59000300D211D1124E987AA877B876C875D8791
:10A5A000BE874F87988B90E0932BA0E0B0E0A22B62
:10A5B00007C0A65ABF4F8D919D910D90BC91A02DC3
:10A5C00023EF38E141E0498BF901459155916591BF
:10A5D0007491481759076A077B0708F499C3A7C302
:10A5E000809122058823E1F0FD01E85BFF4F408167
:10A5F000518160E070E000911102109112022091EF
:10A60000130230911402401751076207730741F09B
:10A610001092150210921602109217021092180250
:10A6200040910D0250910E0260910F027091100244
:10A6300077FF5FC0AE5ABF4FCD90DD90ED90FC909C
:10A6400083EF98E121E0FC0145915591659174916A
:10A650004C155D056E057F0550F4F694E794D7948C
:10A66000C794220F049679E18F30970761F7209302
:10A67000240580E2C816D104E104F10428F470E254
:10A68000C72ED12CE12CF12C90E2C91AD108E10897
:10A69000F108C114A8E0DA06E104F10408F403C4E7
:10A6A000B4E0DB9EC00111248D509B4EFC0132961C
:10A6B00025913491EC2D6627E39FA001E29F410D87
:10A6C000561F0694461F561F112460E070E0FC01DF
:10A6D00025913491C901A0E0B0E0841B950BA60B35
:10A6E000B70B80930D0290930E02A0930F02B093CC
:10A6F0001002C0900D02D0900E02E0900F02F09078
:10A7000010028091390590913A05892B09F0E5C135
:10A710000E9433CE90933A0580933905892B09F432
:10A72000DCC1E0913905F0913A05808183FF3EC09C
:10A7300085899689A789B08D809368119093691156
:10A74000A0936A11B0936B11818D928DA38DB48DFE
:10A7500080936C1190936D11A0936E11B0936F1153
:10A76000858D968DA78DB0A18093701190937111F6
:10A77000A0937211B093731181A192A1A3A1B4A16E
:10A780008093741190937511A0937611B093771103
:10A790009091E00A8091E10A981709F4B9CF80916D
:10A7A000E10A8F5F8F708093E10AB2CFC588D688A7
:10A7B000E788F08C81E0C114D104E104F10409F4CC
:10A7C00080E0018D128D238D348D01151105210539
:10A7D000310509F08260458D568D678D70A1411558
:10A7E00051056105710509F084608093ED041092B4
:10A7F000190510921A0510921B0510921C05109253
:10A80000250510922605109227051092280585A18E
:10A8100096A1A7A1B0A580932D0590932E05A09396
:10A820002F05B0933005882499245401881A990A79
:10A83000AA0ABB0A8092150590921605A0921705E8
:10A84000B09218058092110590921205A0921305FE
:10A85000B092140580920D0590920E05A0920F05FE
:10A86000B09210058092090590920A05A0920B05FE
:10A87000B0920C05CC0CDD1CEE1CFF1CC092F90440
:10A88000D092FA04E092FB04F092FC04000F111F36
:10A89000221F331F0093FD041093FE042093FF0436
:10A8A00030930005440F551F661F771F4093010525
:10A8B00050930205609303057093040541A152A1D2
:10A8C00063A174A1440F551F661F771F40930505B0
:10A8D000509306056093070570930805880F991F2C
:10A8E000AA1FBB1F8093F5049093F604A093F7046E
:10A8F000B093F8041092310510923205109233058E
:10A900001092340582A593A5A4A5B5A58093290529
:10A9100090932A05A0932B05B0932C0586A597A5A7
:10A92000A0A9B1A980931E0590931F05A0932005AF
:10A93000B093210581A58093F404DF01A95BBF4F8B
:10A940009C9190932305992339F115962D913C9173
:10A9500011973093F3042093F20412972D913C91B8
:10A9600011973093F1042093F00410921502109285
:10A970001602109217021092180212972D913C9114
:10A98000A90160E070E040931102509312026093BD
:10A990001302709314020CC088248A94982C5401DA
:10A9A0008092110290921202A0921302B0921402AD
:10A9B000EA5BFF4F90812091E80492130AC0209136
:10A9C0000C0230E0482F082E000C550B421753079D
:10A9D00031F09093E80480930C020E9406CE0E940E
:10A9E000C1C22FEF3FEFA90120930D0230930E0259
:10A9F00040930F0250931002E0913905F0913A050F
:10AA0000DF01DE96ED90FD900D911C9122A933A9F6
:10AA100044A955A9EA5AFF4F6081718182819381CF
:10AA20000E94B4CD10921D05E0913905F0913A05D0
:10AA3000EA5AFF4F80809180A280B38083EF98E133
:10AA400021E0FC0145915591659174914815590596
:10AA50006A057B0558F4B694A79497948794220FBF
:10AA60000496AFE0B9E1A817B90759F72093240578
:10AA700090E289169104A104B10428F4B0E28B2E6F
:10AA8000912CA12CB12C30E2831A9108A108B108B5
:10AA9000811448E09406A104B10408F428C254E0EB
:10AAA000959EC00111248D509B4EFC01329625913C
:10AAB0003491782D6627739FA001729F410D561F18
:10AAC0000694461F561F1124FC01C590D490E12C1A
:10AAD000F12CC41AD50AE108F108C0923505D092CC
:10AAE0003605E0923705F092380500913505109152
:10AAF0003605209137053091380540911502509167
:10AB000016026091170270911802F02E198BF22F25
:10AB1000E32F401751076207730720F4F42E598B77
:10AB2000F62FE72F8F2D9989AF2FBE2F0097E1E0E9
:10AB3000AE07B10520F08FEF9FEFA0E0B0E0081B5B
:10AB4000190B2A0B3B0B0093350510933605209308
:10AB50003705309338054F3FFFEF5F076F077F07DB
:10AB600061F0481B590B6A0B7B0B40931502509305
:10AB700016026093170270931802F89420918400D3
:10AB800030918500205F3F4F4A8941504A8B4423D2
:10AB900041F0280E391E2216330610F40C946E4C28
:10ABA00001C0190130928900209288007894629641
:10ABB0000FB6F894DEBF0FBECDBFDF91CF911F91CE
:10ABC0000F91FF90EF90DF90CF90BF90AF909F904C
:10ABD0008F907F906F905F904F903F902F9008954F
:10ABE00080910B0180958870809309010C947A4DB7
:10ABF00080910B018870809309016EC83989309368
:10AC0000240580E288169104A104B10428F430E2FE
:10AC1000832E912CA12CB12C30E2831A9108A1082B
:10AC2000B108811488E09806A104B10420F1E4E0A1
:10AC30009E9EC00111248D509B4EFC0132962591A1
:10AC40003491F82DEE27F39F7001F29FE10CFE1E68
:10AC50000694EE1EFE1E1124FC01C590D4908601C0
:10AC600020E030E0480159018E189F08A108B10882
:10AC70007501640122C095018401369527951795C9
:10AC80000795F801EC7FCF018D509F4EFC01C590D8
:10AC9000D490FC01329625913491E82DE770E29F23
:10ACA000C001E39F900D112423E0969587952A9586
:10ACB000E1F7C81AD90AE12CF12C4C0D5D1D6E1D6F
:10ACC0007F1D4093250550932605609327057093BB
:10ACD00028059091230580912205992309F474C0D9
:10ACE000882309F40ECDA85BBF4F8D919C91A0E005
:10ACF000B0E04091110250911202609113027091E4
:10AD0000140284179507A607B70709F060C0F9CCAD
:10AD1000B695A79597958795D988DD0CD98A2C5F2C
:10AD20003F4F4FE059E14217530709F04DCC598985
:10AD30005093240580329105A105B10520F480E2ED
:10AD400090E0A0E0B0E08097A109B109811558E03A
:10AD50009507A105B10508F443C074E0979F9001E1
:10AD600011242D503B4EF901329645915491EE2716
:10AD7000859FB001849F610D7E1F06946E1F7E1F0C
:10AD80001124F901C590D490E12CF12CC61AD70AF0
:10AD9000E108F1088091190590911A05A0911B0511
:10ADA000B0911C058C0D9D1DAE1DBF1D8093190516
:10ADB00090931A05A0931B05B0931C058091230561
:10ADC000811130C080912205882309F49ACC109219
:10ADD000150210921602109217021092180291CCCE
:10ADE000AC01BD017695679557954795FA01EC7FC3
:10ADF0009F012D503F4EF901C590D490F901329634
:10AE0000459154918770849F9001859F300D112446
:10AE1000F3E036952795FA95E1F7C21AD30AE12CAB
:10AE2000F12CB8CF8989480E511C611C711C80918E
:10AE3000390590913A05481459046A047B04D8F402
:10AE400020912205222309F45CCCFC01E85BFF4F32
:10AE500020813181A90160E070E000911102109120
:10AE60001202209113023091140240175107620719
:10AE7000730709F446CC1092150210921602109234
:10AE8000170210921802FC01E85BFF4F808191814C
:10AE9000A0E0B0E08093110290931202A0931302FD
:10AEA000B09314022ECCD701C601B695A7959795FD
:10AEB0008795FC01EC7FCF018D509F4EFC012591C1
:10AEC0003491FC013296459154916C2D6770649FCA
:10AED000C001659F900D112463E0969587956A9552
:10AEE000E1F7281B390BC901A0E0B0E0FACBD5018E
:10AEF000C401B695A79597958795FC01EC7FCF0186
:10AF00008D509F4EFC01C590D490FC013296259146
:10AF10003491482D4770429FC001439F900D1124EA
:10AF2000A3E096958795AA95E1F7C81AD90AE12C6E
:10AF3000F12CD3CD80EDC82E87E0D82EE12CF12C5A
:10AF4000E7CBCF92DF92EF92FF920F931F93CF93B5
:10AF5000DF936C017A018B01C0E0D0E0CE15DF05F4
:10AF600081F0D8016D918D01D601ED91FC91019098
:10AF7000F081E02DC6011995892B11F02196EECFB5
:10AF80007E01C701DF91CF911F910F91FF90EF904C
:10AF9000DF90CF900895FF920F931F93CF93DF938D
:10AFA0008C01EB01F42E80E20E94198F8FEFF816CE
:10AFB00011F084E501C082E40E94198F8AE30E94A7
:10AFC000198FF801608171818281938142E00E9432
:10AFD000DA92488159816A817B8187EB9BE10E94EB
:10AFE00085CE62E070E080E090E0DF91CF911F912C
:10AFF0000F91FF900C9464BB8F929F92AF92BF927F
:10B00000CF92DF92EF92FF920F931F93CF93DF9334
:10B01000F0E2FF2EE12CAE2DB0E0BD016F0D711DF1
:10B02000759567956E1511F0F6120BC0E1E9F9E11F
:10B0300065917491072E000C880B990B0E9459EFB3
:10B0400062C09B0121503109220F331F220F331F91
:10B05000F901ED5EF64E05911491AB01440F551FB9
:10B06000440F551FFA01ED5EF64EC591D49180173D
:10B07000910714F4F62ED1CFC817D90714F4E62E91
:10B08000CACFF901EB5EF64EE590F490FA01EB5E63
:10B09000F64EC590D490BC01601B710B072E000CBE
:10B0A000880B990B0E9459EF4B015C01B6016E1998
:10B0B0007F09072E000C880B990B0E9459EF9B010A
:10B0C000AC01C501B4010E94B8EF4B015C01C01B8B
:10B0D000D10BBE01DD0F880B990B0E9459EF9B012C
:10B0E000AC01C501B4010E94ACF44B015C01B70195
:10B0F000FF0C880B990B0E9459EF9B01AC01C50115
:10B10000B4010E94D0F3DF91CF911F910F91FF9076
:10B11000EF90DF90CF90BF90AF909F908F90089569
:10B120000F931F93CF93DF93CDB7DEB728970FB65A
:10B13000F894DEBF0FBECDBF609148047091490402
:10B14000072E000C880B990B0E9459EF6D837E83AC
:10B150008F83988780915C0490915D04A0915E0438
:10B16000B0915F0489839A83AB83BC834DEFBE01AA
:10B170006B5F7F4FCE0101960EDF609142047091AC
:10B180004304072E000C880B990B0E9459EF6D8326
:10B190007E838F8398878091440490914504A09189
:10B1A0004604B091470489839A83AB83BC834FEFF5
:10B1B000BE016B5F7F4FCE010196EDDEEFEBFBE151
:10B1C00084918F010F5F1F4F882321F00E94198FF8
:10B1D000F801F6CFE0917805F0E0EA58FA4F608187
:10B1E00070E080E090E00E94C092EAEBFBE1849185
:10B1F0008F010F5F1F4F882321F00E94198FF801E4
:10B20000F6CF6091770570E080E090E00E94C092F8
:10B2100028960FB6F894DEBF0FBECDBFDF91CF9159
:10B220001F910F9108950F930FB70F9300916E0028
:10B230000B7F00936E0078940F930BB70F930CB7AE
:10B240000F921F922F933F934F935F936F937F9330
:10B250008F939F93AF93BF93EF93FF931124F0D1FC
:10B26000FF91EF91BF91AF919F918F917F916F91DE
:10B270005F914F913F912F911F900F900CBF0F91B5
:10B280000BBF0F910460F89400936E000F910FBFF5
:10B290000F911895CF92DF92EF92FF92C0904404E5
:10B2A000D0904504E0904604F09047046091420439
:10B2B0007091430466507109072E000C880B990B9E
:10B2C0000E9459EF9B01AC01C701B6010E9453EFE8
:10B2D00087FF1FC020E030E040E050E4C701B60126
:10B2E0000E94D0F30E9419F57093A8056093A705FA
:10B2F0000E944E62DC01CB01805A9541AF4FBF4F97
:10B300008093A3059093A405A093A505B093A605EB
:10B3100008C01092A3051092A4051092A5051092E2
:10B32000A605FF90EF90DF90CF900895CF92DF9227
:10B33000EF92FF92C0905C04D0905D04E0905E04B8
:10B34000F0905F046091480470914904675071095E
:10B35000072E000C880B990B0E9459EF9B01AC0142
:10B36000C701B6010E9453EF87FF1FC020E030E005
:10B3700040E450E4C701B6010E94D0F30E9419F5E1
:10B380007093A2056093A1050E944E62DC01CB017F
:10B39000805A9541AF4FBF4F80939D0590939E0576
:10B3A000A0939F05B093A00508C010929D05109230
:10B3B0009E0510929F051092A005FF90EF90DF90E0
:10B3C000CF90089520912202309123022A50310912
:10B3D000821793070CF49C0130934904209348048E
:10B3E00080E0A4CF1092720580E090E0EBDF109235
:10B3F0004304109242044EDF0E941DCF80E090E093
:10B40000E1DF109276052C981092430410924204CA
:10B410001092770580910201807280930001089557
:10B420008F929F92AF92BF92CF92DF92EF92FF9254
:10B430000F931F93CF93DF93F0E4FF2EE12CAE2DFB
:10B44000B0E0BD016F0D711D759567956E1511F01A
:10B45000F6120BC0ECE0FBE165917491072E000C35
:10B46000880B990B0E9459EF62C09B012150310952
:10B47000220F331F220F331FF901E25FF54E0591B2
:10B480001491AB01440F551F440F551FFA01E25FA1
:10B49000F54EC591D4918017910714F4F62ED1CFB3
:10B4A000C817D90714F4E62ECACFF901E05FF54EAC
:10B4B000E590F490FA01E05FF54EC590D490BC01A0
:10B4C000601B710B072E000C880B990B0E9459EF23
:10B4D0004B015C01B6016E197F09072E000C880B29
:10B4E000990B0E9459EF9B01AC01C501B4010E9468
:10B4F000B8EF4B015C01C01BD10BBE01DD0F880B07
:10B50000990B0E9459EF9B01AC01C501B4010E9447
:10B51000ACF44B015C01B701FF0C880B990B0E9446
:10B5200059EF9B01AC01C501B4010E94D0F3DF913A
:10B53000CF911F910F91FF90EF90DF90CF90BF9030
:10B54000AF909F908F90089560E08091B4059091A6
:10B55000B50552DD60935C0470935D0480935E04D6
:10B5600090935F048091B2059091B30559DF609389
:10B570004404709345048093460490934704A8952F
:10B58000109273050895DF92EF92FF920F931F932D
:10B59000CF93DF93F82ED62EE72E8A0180911902E1
:10B5A000882309F439C0E5E5F4E28491EF0121969E
:10B5B000882321F00E94198FFE01F7CFED2DFE2D7B
:10B5C0008491EF012196882321F00E94198FFE01BA
:10B5D000F7CFE4EAF9E18491EF012196882321F085
:10B5E0000E94198FFE01F7CFF7FC0BC06F2DFF0CE7
:10B5F000770B880B990B0E94C0928AE00E94198FEA
:10B600000BC0EFE9F9E18491EF012196882321F045
:10B610000E94198FFE01F7CF80917905811108C032
:10B620001092190281E080937905C8010E9447AE0B
:10B63000DF91CF911F910F91FF90EF90DF90D2CECD
:10B640000F931F93CF93DF9380911C028F37A0F04D
:10B650008F57909176059093C505992311F02C9AF8
:10B6600001C02C98209177052093C4059091020188
:10B67000222369F090950BC09091C505891708F0B9
:10B680002C989091C405891728F09091020190722E
:10B69000909300018F5F80931C029091C30581E01D
:10B6A00089278093C30580911B0285301CF4C1E07B
:10B6B000C80F01C0C0E0823009F4B8C054F4882338
:10B6C00001F1813009F0E7C088E080937B0085E4D8
:10B6D000C4C0843009F4C9C00CF4BBC0853009F083
:10B6E000DAC09091C205911102C08093C205809189
:10B6F000C20581508093C205882309F4CCC0C5E0FF
:10B70000CAC080911A028F5F80311CF480931A02A4
:10B71000C2C010921A0280917305811113C08091EA
:10B72000B8059091B9059093B5058093B4058091C3
:10B73000B6059091B7059093B3058093B20581E06B
:10B74000809373058AE0E8EBF5E0DF011D928A95AE
:10B75000E9F71092B7051092B6050091B405109163
:10B76000B5051195019511098091480490914904FE
:10B77000D1E0181619062CF080917605811101C0D0
:10B78000D0E08091D0059091D10591958195910956
:10B790008017910734F445E45BE166E67BE180E0E5
:10B7A000F2DE80912002909121029195819591097C
:10B7B0000817190744F4DD2331F048E75BE169E934
:10B7C0007BE180E0E0DE809142049091430411E04F
:10B7D000181619062CF080917705811101C010E030
:10B7E0002091B2053091B3058091CE059091CF059F
:10B7F0008217930734F045E55BE166E67BE18FEF66
:10B80000C2DE20911E0230911F028091B2059091FC
:10B81000B305821793070CF43EC01123E1F148E809
:10B820005BE169E97BE18FEFAEDE35C080917A00A4
:10B8300086FD2EC080917800909179002091B80506
:10B840003091B905820F931F9093B9058093B80585
:10B8500022C088E080937B0086E480937C00809106
:10B860007A00806480937A0016C080917A0086FD09
:10B8700011C080917800909179002091B6053091A7
:10B88000B705820F931F9093B7058093B60503C049
:10B89000C2E001C0C4E0C0931B020E94C1C28091FB
:10B8A000740590917505009799F00197909375052F
:10B8B00080937405892B61F48BEA9BE190934B0490
:10B8C00080934A04DF91CF911F910F910C94818F47
:10B8D000DF91CF911F910F9108952F923F924F9238
:10B8E0005F926F927F928F929F92AF92BF92CF9210
:10B8F000DF92EF92FF920F931F93CF93DF9300D0CD
:10B900001F92CDB7DEB75C017A8369831A0107FD08
:10B910000DC0802F002E000C990B9C838B83FC01A3
:10B92000E75AFE4E80818823E1F008C08091B1057E
:10B93000882399F0E1E0F0E0FC83EB83F5011082CD
:10B94000EB81FC81EE0FFF1FEE0FFF1FE755FA4F53
:10B95000108211821282138230C081E090E09C83B9
:10B960008B83F90140805180628073808B819C8140
:10B97000880F991F880F991F9C0127553A4F49013D
:10B98000A3019201F40160817181828193810E94FF
:10B9900053EF882391F0F4014082518262827382D6
:10B9A00011E020E030E0A901C301B2010E94F6F5E8
:10B9B00018160CF010E0F5011083F501808182303B
:10B9C000F1F0833009F464C0813009F082C0EB816A
:10B9D000FC81EE0FFF1FEE0FFF1FE755FA4F20818E
:10B9E000318142815381F101608171818281938132
:10B9F0000E9453EF87FD6DC082E0F50180832B81AB
:10BA00003C81220F331F220F331F27553A4F3C83AF
:10BA10002B83B60180E090E00E9457EF9B01AC01C0
:10BA2000EB81FC8160817181828193810E94CFF3DF
:10BA30009B01AC01F10160817181828193810E943F
:10BA4000F6F587FD13C02AD54B015C019701A8EEDE
:10BA5000B3E00E94C0F3860E971EA81EB91EE981AE
:10BA6000FA8180829182A282B38233C017D5E981A4
:10BA7000FA81C080D180E280F380DC01CB018C1997
:10BA80009D09AE09BF09B7FD24C083E0F50180839D
:10BA90000F3F19F04EE05BE102C041E25BE165E37C
:10BAA0007BE1802F0F900F900F900F90DF91CF913F
:10BAB0001F910F91FF90EF90DF90CF90BF90AF90CC
:10BAC0009F908F907F906F905F904F903F902F90BE
:10BAD0005ACD0F900F900F900F90DF91CF911F9143
:10BAE0000F91FF90EF90DF90CF90BF90AF909F901D
:10BAF0008F907F906F905F904F903F902F90089520
:10BB00007F928F929F92AF92BF92CF92DF92EF92ED
:10BB1000FF920F931F93CF93DF9320E030E048E430
:10BB200052E460915C0470915D0480915E04909198
:10BB30005F040E94F6F518164CF4E9E9F9E1E49186
:10BB4000C1E001C0CC0FEA95EAF701C0C0E083E98B
:10BB5000E82E89E1F82E09E919E196E0A92E912C49
:10BB6000D0E0CC24C394D12CF7017490F8018490D8
:10BB700077FC23C0892D90E0082C02C0959587950D
:10BB80000A94E2F780FD19C0BE01082C02C0759529
:10BB900067950A94E2F76170B62EB1946B2D872DEC
:10BBA0000E9433BA6B2D70E0872D0E949DBAC601AA
:10BBB00001C0880F8A94EAF7982AAA94FFEFEF1A37
:10BBC000FF0A0F5F1F4FA110CFCFDF91CF911F91C1
:10BBD0000F91FF90EF90DF90CF90BF90AF909F902C
:10BBE0008F907F9008954F925F926F927F928F9285
:10BBF0009F92AF92BF92CF92DF92EF92FF920F93FC
:10BC00001F93CF93DF93CDB7DEB760970FB6F8944D
:10BC1000DEBF0FBECDBF80917105811138C180910B
:10BC20007305811117C060960FB6F894DEBF0FBE82
:10BC3000CDBFDF91CF911F910F91FF90EF90DF90DB
:10BC4000CF90BF90AF909F908F907F906F905F90BC
:10BC50004F90089579DC22D44B015C0180915911F9
:10BC6000811117C080913E1190913F11A091401118
:10BC7000B09141110097A105B10559F0A5019401BA
:10BC8000281B390B4A0B5B0B57FD03C081E08093E7
:10BC900059116091480470914904072E000C880BDB
:10BCA000990B0E9459EF69837A838B839C8344E1CB
:10BCB000C42ED12C5CE3E52EF12C00E09E012F5F19
:10BCC0003F4F4CE554E069E975E088E995E005DE11
:10BCD00040905C0450905D0460905E0470905F043E
:10BCE0006091D2057091D305072E000C880B990B3B
:10BCF0000E9459EF9B01AC01C301B2010E94F6F50D
:10BD000018160CF4C8C060E06093760580919D051C
:10BD100090919E05A0919F05B091A0050097A10567
:10BD2000B10521F1A5019401281B390B4A0B5B0BCE
:10BD300057FD1CC06091A1057091A20580E090E0C4
:10BD40000E9457EF9B01AC0160915C0470915D040F
:10BD500080915E0490915F040E9453EF87FF4BC275
:10BD600044EE59E166EF79E180E00DDC80916D05EC
:10BD700090916E05A0916F05B0917005A501940199
:10BD8000281B390B4A0B5B0B57FD0FC0B9DED501E1
:10BD9000C4018C53964FAF4FBF4F80936D05909366
:10BDA0006E05A0936F05B09370058091A3059091E7
:10BDB000A405A091A505B091A6050097A105B10520
:10BDC00011F1881A990AAA0ABB0AB7FC1CC0609133
:10BDD000A7057091A80580E090E00E9457EF9B01B5
:10BDE000AC016091440470914504809146049091A7
:10BDF00047040E9453EF87FF3BC142EC59E165EDD8
:10BE000079E18FEFC0DB6091420470914304072E0B
:10BE1000000C880B990B0E9459EF69837A838B83FE
:10BE20009C8395E0C92ED12C24E1E22EF12C0FEF5A
:10BE30009E012F5F3F4F44E454E063E975E087E9DA
:10BE400095E04BDD8091B10581110FC1C090440494
:10BE5000D0904504E0904604F090470420E030E0A4
:10BE600040EA50E4C701B6010E94F6F587FD0BC019
:10BE700020E030E047E053E4C701B6010E9453EFF1
:10BE800018160CF0F7C060E060937705CCCE85E023
:10BE90009AE10E9447AE6091220270912302072E20
:10BEA000000C880B990B0E9459EF9B01AC01C30158
:10BEB000B2010E9453EF87FF26CF009148041091F2
:10BEC000490420ED3CEC4CE45DE360916905709120
:10BED0006A0580916B0590916C050E94B8EF6B012B
:10BEE0007C0120918F0530919005409191055091F2
:10BEF0009205C301B2010E94CFF39B01AC01C701BF
:10BF0000B6010E94B8EF6B017C0123E333E343E702
:10BF10005FE360918B0570918C0580918D05909108
:10BF20008E050E94B8EF9B01AC01C701B6010E94CB
:10BF3000D0F36B017C0160938B0570938C0580932B
:10BF40008D0590938E0540928F05509290056092DA
:10BF50009105709292058091591181114FC1B801DC
:10BF6000012E000C880B990B0E9459EFA30192013E
:10BF70000E94CFF32B013C0120E030E040E251E48D
:10BF80000E94F6F518160CF44AC120E030E040E2B9
:10BF900051ECC301B2010E9453EF87FD2FC1012B69
:10BFA00009F42CC180918A05811170C180918605A8
:10BFB00090918705A0918805B09189058D839E8316
:10BFC000AF83B8872091650530916605409167057C
:10BFD00050916805C301B2010E94B8EF69877A8762
:10BFE0008B879C87A30192016D817E818F819885CB
:10BFF0000E94D0F36D837E838F839887609386053C
:10C000007093870580938805909389052091610539
:10C010003091620540916305509164050E94B8EF2C
:10C0200029853A854B855C850E94D0F3A70196014E
:10C030000E94CFF36B017C0120E030E04FE753E436
:10C040000E94F6F520E030E0A90118160CF406C1B4
:10C05000C701B6010E9453EF87FD1FC1C701B6019A
:10C060000E9414F5759567954FCE10927705DBCD3C
:10C0700011D9C9CE6091420470914304072E000C7F
:10C08000880B990B0E9459EFA70196010E94CFF3EC
:10C090004B015C0120915D0530915E0540915F058B
:10C0A000509160050E94B8EF69877A878B879C87DB
:10C0B000209182053091830540918405509185053A
:10C0C000C501B4010E94D0F36D837E838F8398876E
:10C0D0006093820570938305809384059093850512
:10C0E0002091590530915A0540915B0550915C05AE
:10C0F0000E94B8EF6D877E878F87988B20ED3CEC90
:10C100004CE45DE3609155057091560580915705AB
:10C11000909158050E94B8EF2B013C0120917E05BB
:10C1200030917F054091800550918105C701B6018E
:10C130000E94CFF39B01AC01C301B2010E94B8EF92
:10C140002B013C0123E333E343E75FE360917A058E
:10C1500070917B0580917C0590917D050E94B8EFE0
:10C160009B01AC01C301B2010E94D0F32B013C0141
:10C1700060937A0570937B0580937C0590937D0591
:10C18000C0927E05D0927F05E0928005F0928105F5
:10C190002D853E854F85588969857A858B859C8557
:10C1A0000E94D0F3A30192010E94CFF36B017C01A6
:10C1B00020E030E04FE753E40E94F6F520E030E065
:10C1C000A9011816FCF4C501B4010E94F6F5181671
:10C1D00084F4A50194016D817E818F8198850E94F0
:10C1E000CFF36093820570938305809384059093C9
:10C1F00085056FE749CE80E099D8B8CD81E080937E
:10C200008A0581CDC701B6010E9453EF87FD0CC09E
:10C21000C701B6010E9414F57595679535CE81E08A
:10C2200080938A056FE770CD20E030E0A901C50159
:10C23000B4010E9453EF87FF26CEA50194016D81C2
:10C240007E818F8198850E94CFF3609382057093E1
:10C250008305809384059093850515CEC301B201B3
:10C260000E94F6F51816F4F6A30192016D817E8105
:10C270008F8198850E94CFF3609386057093870520
:10C2800080938805909389056FE73ECD10928A05CB
:10C290001D821E821F82188695CE20E030E0A90103
:10C2A000C301B2010E9453EF87FF2DCDA30192017C
:10C2B0006D817E818F8198850E94CFF36093860582
:10C2C0007093870580938805909389051CCDCF9244
:10C2D000DF92EF92FF926B017C0183E3C816D104D9
:10C2E000E104F10468F082E3C81AD108E108F1081A
:10C2F00062E370E080E090E00E9464BB74DCEDCF0C
:10C30000C701B6010E9464BBFF90EF90DF90CF9011
:10C310006ACC0F931F9380915405813011F4BED0E5
:10C3200008C060915005709151058091520590911F
:10C33000530500914C0510914D0520914E0530910B
:10C340004F05601B710B820B930B28EE33E040E02E
:10C3500050E00E9472F38091480590914905A091A8
:10C360004A05B0914B05BC01CD01620F731F841FBC
:10C37000951F1F910F9108951092540510924C052E
:10C3800010924D0510924E0510924F0510925005D7
:10C3900010925105109252051092530510924805C3
:10C3A0001092490510924A0510924B05089580910C
:10C3B0005405813071F482E0809354056FD060930E
:10C3C000500570935105809352059093530581E079
:10C3D000089580E0089590916F00292F227091FFB9
:10C3E00005C090916F009D7F90936F0034E0839F14
:10C3F000C0011124FC01E859FE4E40815181628147
:10C400007381FC01E45CFA4F408351836283738340
:10C4100081E080933B05222329F080916F008260A8
:10C4200080936F000895BC012091390530913A0541
:10C430004091390550913A052417350711F09A01BA
:10C44000F7CF81E02617370709F080E008950E94B2
:10C45000E0F63FB7F89480917E0790917F07A09116
:10C460008007B091810726B5A89B05C02F3F19F022
:10C470000196A11DB11D3FBFBA2FA92F982F882764
:10C48000820F911DA11DB11DBC01CD0142E0660FBF
:10C49000771F881F991F4A95D1F708952FB7F894F1
:10C4A00060917A0770917B0780917C0790917D075E
:10C4B0002FBF08951F920F920FB60F9211242F9342
:10C4C0003F938F939F93AF93BF9380917A079091FF
:10C4D0007B07A0917C07B0917D073091790723E01D
:10C4E000230F2D3720F40196A11DB11D05C026E8AC
:10C4F000230F0296A11DB11D2093790780937A071F
:10C5000090937B07A0937C07B0937D0780917E0773
:10C5100090917F07A0918007B09181070196A11D9E
:10C52000B11D80937E0790937F07A0938007B093FF
:10C530008107BF91AF919F918F913F912F910F9064
:10C540000FBE0F901F9018951F920F920FB60F926B
:10C5500011240BB60F922F933F934F935F936F93DA
:10C560007F938F939F93AF93BF93EF93FF938091AC
:10C57000C9059091CA05A091CB05B091CC05892B36
:10C580008A2B8B2B59F19091C805E091C605F0914B
:10C59000C7058081892780838091C9059091CA054C
:10C5A000A091CB05B091CC05181619061A061B06EA
:10C5B0000CF056C08091C9059091CA05A091CB0599
:10C5C000B091CC050197A109B1098093C905909359
:10C5D000CA05A093CB05B093CC0542C080911D0243
:10C5E000E3ECFBE1E4919FEF90931D02E230C9F090
:10C5F00050F4EE2399F0E13081F590916F009D7F2A
:10C6000090936F002AC0E43019F1E0F0E53029F58D
:10C61000909173009D7F909373001FC010926E00E5
:10C620001CC0909170009D7F9093700091E090935A
:10C63000B0009091B100987F94609093B1001092F7
:10C64000B3000BC0909171009D7F9093710005C065
:10C65000909172009D7F9093720060E00E9433BAC7
:10C66000FF91EF91BF91AF919F918F917F916F91CA
:10C670005F914F913F912F910F900BBE0F900FBE86
:10C680000F901F901895CF92DF92EF92FF920F9329
:10C690001F93CF93DF93CDB7DEB7A0970FB6F89473
:10C6A000DEBF0FBECDBF80E090E0A0EAB0E489839A
:10C6B0009A83AB83BC8380E090E0ADE4B3E48D83E8
:10C6C0009E83AF83B88780E090E0A0EAB1E48987D9
:10C6D0009A87AB87BC8788E592E00E94208F811102
:10C6E00095C185E40E94EB3F882381F00E94B43F0E
:10C6F0006B017C0120E030E0A9010E94F6F587FF84
:10C700000BC0F7FAF094F7F8F09406C0C12CD12CC6
:10C7100080E8E82E80E4F82EF7FAF094F7F8F09429
:10C72000C98ADA8AEB8AFC8A8AE50E943440882327
:10C7300079F08AE50E943440882319F00E94B43FC2
:10C7400003C060E070E0CB0169877A878B879C87A4
:10C7500088E50E943440882379F088E50E943440BF
:10C76000882319F00E94B43F03C060E070E0CB0161
:10C7700069837A838B839C8389E50E943440882374
:10C7800079F089E50E943440882319F00E94B43F73
:10C7900003C060E070E0CB016D837E838F83988758
:10C7A00085E50E94EB3F882329F00E94B43F6B018E
:10C7B0007C010CC0E091101184E0E89FF00111248D
:10C7C000E75EF64EC080D180E280F38020E030E06A
:10C7D000A901C701B6010E94F6F587FF04C0F7FA68
:10C7E000F094F7F8F094F7FAF094F7F8F094CD8A13
:10C7F000DE8AEF8AF88E198E1A8E1B8E1C8E8CE4C0
:10C800000E94EB3F882329F00E94B43F6B017C011A
:10C810000CC0E091101194E0E99FF0011124E35E57
:10C82000F64EC080D180E280F38020E030E0A901A4
:10C83000C701B6010E94F6F587FF04C0F7FAF0942D
:10C84000F7F8F094CD8EDE8EEF8EF8A282E40E948F
:10C850003440882321F00E94843F162F01C01AE043
:10C8600000915405AE014B5E5F4FBE016F5F7F4F7D
:10C87000CE0141960E9466B3882309F4C3C0EAE65C
:10C88000F4E284917F019FEFE91AF90A882321F0ED
:10C890000E94198FF701F5CFE6E2F0E284917F0163
:10C8A0009FEFE91AF90A882321F00E94198FF701F6
:10C8B000F5CF61E0812F0E948B82F0DDDC01CB019E
:10C8C00080529C46AB4FBF4F80933E1190933F11D7
:10C8D000A0934011B09341111092591183E08093BD
:10C8E000471181E08093461180914611882309F415
:10C8F0006FC060E0812F0E948B8280915911882344
:10C9000009F462C0EAE6F4E284917F019FEFE91A3C
:10C91000F90A882321F00E94198FF701F5CFECE086
:10C92000F0E284917F019FEFE91AF90A882339F038
:10C930000E94198FF701F5CF81E00E948EAE8091A1
:10C9400046118111F9CF10923E1110923F111092B1
:10C95000401110924111109259110E9496590E9453
:10C96000ECB2EAE6F4E284917F019FEFE91AF90A5A
:10C97000882321F00E94198FF701F5CFEDEEFFE13A
:10C9800084917F019FEFE91AF90A811119C086DDB0
:10C99000DC01CB0180529C46AB4FBF4F80933E11D0
:10C9A00090933F11A0934011B093411110925911EF
:10C9B00081E08093461161E0812F0E948B8204C048
:10C9C0000E94198FF701DCCF81E00E948EAE8CCFE0
:10C9D00081E08093471180E090E0A0E2B1E48D8790
:10C9E0009E87AF87B88B8091D108882359F0212F7B
:10C9F000AE01435F5F4FBE01635E7F4FCE0149963C
:10CA00000E9484B8013011F40E94D6CEA0960FB6D1
:10CA1000F894DEBF0FBECDBFDF91CF911F910F9174
:10CA2000FF90EF90DF90CF900895CF92DF92EF923A
:10CA3000FF920F931F93CF93DF9388E50E94EB3F04
:10CA4000D82E89E40E94EB3FC82E882319F00E945B
:10CA5000843F1CC0DD20C1F00E94B43F20E030E0E4
:10CA600040E251E40E94CFF320E030E040EC51E49A
:10CA70000E94D0F32BEA3AEA4AEA5CE30E94B8EF5C
:10CA80000E9414F5653010F01FEF01C0162F89E5E4
:10CA90000E94EB3F082F8AE40E94EB3FC82F8823B7
:10CAA00019F00E94843F1CC00023C1F00E94B43FD3
:10CAB00020E030E040E251E40E94CFF320E030E09B
:10CAC00040EC51E40E94D0F32BEA3AEA4AEA5CE3F4
:10CAD0000E94B8EF0E9414F5653010F0DFEF01C03E
:10CAE000D62F8AE50E94EB3FE82E811105C081E533
:10CAF0000E94EB3FF82E01C0F12CC11001C0C0E034
:10CB00002C2F30E0D11001C000E0200F311D21306A
:10CB1000310521F4E1101AC0F11018C0E5E5F4E286
:10CB20008491EF012196811103C0EDECFFE104C077
:10CB30000E94198FFE01F4CF8491EF012196882382
:10CB400009F455C00E94198FFE01F6CF17FD02C0EF
:10CB5000D7FF17C0E5E5F4E28491EF01219681113A
:10CB600003C0EEEAFFE104C00E94198FFE01F4CF7A
:10CB70008491EF0121968823D1F10E94198FFE0143
:10CB8000F7CF0E94B43F9B01AC01012F110F110B95
:10CB9000AD2FDD0FBB0BFF2099F085E0809FF001EA
:10CBA000819FF00D1124EA0FFB1FEE0FFF1FEE0F08
:10CBB000FF1FE455FE4E608171818281938103C025
:10CBC00060E070E0CB01E5E0E09FE001E19FD00D87
:10CBD0001124CA0FDB1FCC0FDD1FCC0FDD1FC45586
:10CBE000DE4E0E94D0F3688379838A839B83DF9132
:10CBF000CF911F910F91FF90EF90DF90CF9008950C
:10CC00002F923F924F925F926F927F928F929F925C
:10CC1000AF92BF92CF92DF92EF92FF920F931F934A
:10CC2000CF93DF93CDB7DEB761970FB6F894DEBF31
:10CC30000FBECDBF83E50E94EB3F882349F00E94E1
:10CC4000A53F182F811106C080E00E94418502C0D7
:10CC50001091621180914C0490914D04A0914E046A
:10CC6000B0914F0489839A83AB83BC838091500435
:10CC700090915104A0915204B09153048D839E83EE
:10CC8000AF83B8878091540490915504A0915604C5
:10CC9000B091570489879A87AB87BC870E94148517
:10CCA000882309F49AC083E40E94EB3F882309F4A7
:10CCB00094C00E94B43F1B012C0105E0612C712C33
:10CCC00038EC388B82EC898BA12CB12C98EC9E87A8
:10CCD000E2E4EF87015080F125E02D87209F40019D
:10CCE00011243D8531503D873F3FA1F3F401E30F0F
:10CCF000F11DEE0FFF1FEE0FFF1FE455FE4EC0802B
:10CD0000D180E280F3809601A701B5018E859F85D1
:10CD10000E94F6F518161CF45601EE86FF86960161
:10CD2000A701B301888999890E9453EF87FFD9CF62
:10CD30003601E88AF98AD5CF930148895989B50126
:10CD40008E859F850E94D0F320E030E040E05FE3D5
:10CD50000E94B8EFA20191010E94D0F32B013C0187
:10CD60002DEB37E346E855EB0E94F6F587FD0AC048
:10CD70002DEB37E346E855E3C301B2010E9453EFC0
:10CD800018165CF580E00E94418535E0D32E45E021
:10CD9000C42EDA949FEFD91601F105E0CD9C500125
:10CDA00011240150B0F37501E00EF11CC701880F8A
:10CDB000991F880F991FFC01E455FE4E7F01A301C6
:10CDC000920160817181828193810E94CFF3F7018A
:10CDD0006083718382839383E4CF86E50E94EB3F77
:10CDE000882399F00E941485882379F0E8E9FFE10F
:10CDF00084917F012FEFE21AF20A882321F00E942A
:10CE0000198FF701F5CF0E94FEC18AE50E94EB3F22
:10CE1000882321F00E94B43F0E94BBB7812F0E945B
:10CE20004185111103C0EAE6F4E21CC08091621151
:10CE30008111F9CFE5E5F4E284918F010F5F1F4F77
:10CE4000882321F00E94198FF801F6CFE9E7FFE16E
:10CE500084918F010F5F1F4F882329F30E94198F40
:10CE6000F801F6CF84918F010F5F1F4F882321F0C7
:10CE70000E94198FF801F6CF80916211811103C0D1
:10CE800067E173E002C063E173E08BE69FE10E941B
:10CE9000BBCE8AE00E94198FEAE6F4E284918F010A
:10CEA0000F5F1F4F882321F00E94198FF801F6CFE2
:10CEB000EEE5FFE184918F010F5F1F4F882321F082
:10CEC0000E94198FF801F6CFC0906311D0906411C1
:10CED000E0906511F090661120E030E0A901C701F3
:10CEE000B6010E94F6F518164CF442E0C701B601EF
:10CEF0000E94DA928AE00E94198F0CC0E9E5FFE1F6
:10CF000084918F010F5F1F4F882321F00E94198F9A
:10CF1000F801F6CF4CE050E06CE474E0CE010196ED
:10CF20000E94ECF6892BD1F061960FB6F894DEBF23
:10CF30000FBECDBFDF91CF911F910F91FF90EF906A
:10CF4000DF90CF90BF90AF909F908F907F906F9029
:10CF50005F904F903F902F900C94C77E61960FB6D4
:10CF6000F894DEBF0FBECDBFDF91CF911F910F911F
:10CF7000FF90EF90DF90CF90BF90AF909F908F90F9
:10CF80007F906F905F904F903F902F900895809189
:10CF90006F00982F927081FF05C080916F008D7F88
:10CFA00080936F008091E10A8093E00A8093DF0A0A
:10CFB0008093DE0A84E68093DD0A28EE33E0309326
:10CFC000750520937405992329F080916F00826084
:10CFD00080936F0081E080933B050E94B67E0E94A3
:10CFE00092CB80916211882321F081E492E10E942A
:10CFF0009DCF8CE0E1E4F2E1ACE4B4E001900D926D
:10D000008A95E1F70C94E08D2F923F924F925F92B8
:10D010006F927F928F929F92AF92BF92CF92DF9248
:10D02000EF92FF920F931F93CF93DF93CDB7DEB7AD
:10D03000CD54D1090FB6F894DEBF0FBECDBF85E445
:10D040000E943440882321F00E94843F8B0102C05B
:10D0500000E010E083E40E943440882321F00E9425
:10D06000843F6AA302C025E02AA385E50E943440DC
:10D07000882319F00E94A53F03C085E50E94EB3F7D
:10D080008CA717FD07C0C12CD12CB6E1EB2EB3E461
:10D09000FB2E06C0C12CD12CACE8EA2EA2E4FA2E5D
:10D0A00083E50E943440882321F00E94B43F6B0145
:10D0B0007C010115110511F41092780510924711A9
:10D0C000102FECD92B013C01302F331F3327331F96
:10D0D00083E0831B8983D301C2018C53964FAF4FEA
:10D0E000BF4F80936D0590936E05A0936F05B0932D
:10D0F00070050F5F023080F0EFE2FFE18491AF0135
:10D100004F5F5F4F5A834983882309F472C30E949B
:10D11000198FE981FA81F2CF17FD12C0E12FEE0FCE
:10D12000FF0BEE5DFD4F608171816A507109072E22
:10D13000000C880B990B0E9459EF4B015C0106C053
:10D14000812C912CFAEFAF2EF2E4BF2EC701B6016D
:10D150000E9414F5072E000C880B990B0E9459EFC2
:10D1600069877A878B879C87A50194010E94F6F5D1
:10D1700018167CF4E0EFFEE18491DF011196BA838A
:10D18000A983882309F435C30E94198FE981FA81A4
:10D19000F3CFEBE1FFE184917F01BFEFEB1AFB0AD4
:10D1A000882321F00E94198FF701F5CF0E94F259D0
:10D1B00017FF04C08FE78093770508C0E12F012E89
:10D1C000000CFF0BEA58FA4F8FE78083E9818E2F1E
:10D1D00090E0A3019201205A35414F4F5F4F2EAB93
:10D1E0003FAB48AF59AF21E0209324021F3F49F4E1
:10D1F0004AE55EE15BAF4AAFA4E2BEE1BDAFACAFD2
:10D2000008C0E8E4FEE1FBAFEAAF21E13EE13DAF5B
:10D210002CAF4CA25DA26EA27FA24DA65EA66FA609
:10D2200078AA19AA1AAA1BAA1CAA1DAA2A961FAE76
:10D230002A9730E4398F4CE14A8F56E45B8F1C8E7D
:10D240001D8E1E8E1F8E1D8A1E8A1F8A188E198A99
:10D250001A8A1B8A1C8A19821A821B821C822FE757
:10D2600030E040E050E02D833E834F8358877FE7D6
:10D27000C72ED12CE12CF12C18A619A61AA61BA694
:10D2800031E03D87188A1F8629961FAE2997212CE9
:10D29000312C00E0212F012E000C330BA9014A583C
:10D2A0005A4F5FAF4EAF220F331F220F331FD901EA
:10D2B000A45ABB4FB9A3A8A39C01092E000C440B90
:10D2C000550B24962CAF3DAF4EAF5FAF249704961D
:10D2D0009C01990F440B550B28962CAF3DAF4EAFD8
:10D2E0005FAF28974AA1042E000C550B5BA34AA3FD
:10D2F00080912402882309F47AC2D0D84B015C01C2
:10D3000080917305882309F4D8C00E94A45A17FDA0
:10D310000CC0A8A1B9A1BC912996BFAF2997E8A1DB
:10D32000F9A12180328003810BC0F0914404299639
:10D33000FFAF2997209045043090460400914704A0
:10D3400029962FAD2997322D432D502F6C8D7D8D31
:10D350008E8D9F8D0E9453EF87FF07C029962FADBA
:10D3600029972C8F2D8E3E8E0F8F2A962FAD2A97C0
:10D37000398D4A8D5B8D29966FAD2997722D832D3E
:10D38000902F0E9453EF87FF09C029963FAD299740
:10D390002A963FAF2A97298E3A8E0B8F80916D0582
:10D3A00090916E05A0916F05B0917005A501940153
:10D3B000281B390B4A0B5B0B57FD10C00E94805D88
:10D3C000D501C4018C53964FAF4FBF4F80936D056D
:10D3D00090936E05A0936F05B09370053D852996D7
:10D3E0002FAD2997332309F44BC0322D432D502FF5
:10D3F00069857A858B859C850E9453EF87FF5DC088
:10D40000D501C40184199509A609B7092E968CAFD8
:10D410009DAFAEAFBFAF2E9788589341A109B10918
:10D42000B7FD4BC0D701C6012D813E814F81588584
:10D43000821B930BA40BB50BB595A7959795879574
:10D4400017FF03C08093770503C0EEADFFAD808367
:10D450002E962CAD3DAD4EAD5FAD2E9728A739A7CA
:10D460004AA75BA739853C8F4A854D8F5B855E8FC8
:10D470008C858F8F8CA29DA2AEA2BFA21D861DC0DF
:10D48000322D432D502F69857A858B859C850E948E
:10D49000F6F5181694F4D501C4012CA13DA14EA1B6
:10D4A0005FA1821B930BA40BB50BAC01BD014858C7
:10D4B00053416109710977FFB9C120E030E040EACA
:10D4C00051E469857A858B859C850E94D0F32996E5
:10D4D0002FAD2997322D432D502F0E9453EF87FFF8
:10D4E0000FC0ECE7FEE18491DF011196BA83A983B6
:10D4F000882309F47CC10E94198FE981FA81F3CF56
:10D50000D501C4012DA53EA54FA558A9821B930B9B
:10D51000A40BB50BB7FD89C00E9490588AE00E9409
:10D52000198FD501C4018053984FAF4FBF4F8DA7BE
:10D530009EA7AFA7B8AB99A991115AC02AA93BA938
:10D540004CA95DA929966FAD2997722D832D902F37
:10D550000E94F6F51816DCF524966CAD7DAD8EAD07
:10D560009FAD24970E9459EF29962FAD2997322D10
:10D57000432D502F0E94D0F36AAB7BAB8CAB9DAB9D
:10D58000A5019401205A35414F4F5F4F2EAB3FAB61
:10D5900048AF59AF28966CAD7DAD8EAD9FAD289745
:10D5A0000E9459EF9B01AC0169857A858B859C852A
:10D5B0000E94CFF329962FAD2997322D432D502F5E
:10D5C0000E9453EF881F8827881F89AB2EC0D50182
:10D5D000C4012EA93FA948AD59AD821B930BA40BE2
:10D5E000B50BB7FD22C04AAD5BAD6DE67EE11AC05A
:10D5F00020E030E040EA51E469857A858B859C859E
:10D600000E94CFF39B01AC0129966FAD2997722D33
:10D61000832D902F0E9453EF87FF07C04CAD5DAD67
:10D6200068E37EE1812F0E94C35AD501C401880FAF
:10D63000991FAA1FBB1F2CA13DA14EA15FA1821B58
:10D64000930BA40BB50B84199509A609B709813072
:10D650009F49A442B10580F0E3EFFDE18491AF0161
:10D660004F5F5F4F5A834983882309F4C0C00E94EB
:10D67000198FE981FA81F2CF8AA19BA1AF85B88980
:10D680008A179B070CF034CEE6E9FDE184913F0157
:10D69000BFEF6B1A7B0A882321F00E94198FF301D8
:10D6A000F5CF17FD05C0E6E1F3E0FE83ED8304C08E
:10D6B0002CE034E03E832D836D817E8185E89DE101
:10D6C0000E94BBCE49815A816B817C8181E89DE1BA
:10D6D0000E9485CE8AE00E94198F6D817E8180E74D
:10D6E0009DE10E94BBCE49895A896B897C898CE671
:10D6F0009DE10E9485CE8AE00E94198F6D817E8116
:10D700008BE59DE10E94BBCE4D895E896F89788D46
:10D7100087E59DE10E9485CE8AE00E94198F3CA595
:10D72000332309F466C017FF31C089819A81AB8128
:10D73000BC8180935D0590935E05A0935F05B093D7
:10D7400060052CEA35EC47E25EE369897A898B89CA
:10D750009C890E94B8EF6093590570935A05809395
:10D760005B0590935C052CEA35EC47E25EE36D893E
:10D770007E898F89988D0E94ACF4609355057093D3
:10D780005605809357059093580533C029813A81F7
:10D790004B815C8120936505309366054093670556
:10D7A000509368052CEA35EC47E25EE369897A8993
:10D7B0008B899C890E94B8EF609361057093620524
:10D7C00080936305909364052CEA35EC47E25EE3B1
:10D7D0006D897E898F89988D0E94ACF4609369056C
:10D7E00070936A0580936B0590936C0502C00E944C
:10D7F000F25981E080934711C35BDF4F0FB6F89475
:10D80000DEBF0FBECDBFDF91CF911F910F91FF9073
:10D81000EF90DF90CF90BF90AF909F908F907F90D0
:10D820006F905F904F903F902F9008954F8558894B
:10D83000452B09F437C148A459A46AA47BA4480E17
:10D84000591E6A1E7B1E28A539A54AA55BA5281B63
:10D85000390B4A0B5B0B6D817E818F8198850E940D
:10D8600063F3A30192010E9494F3DA01C9018C0DC4
:10D870009D1DAE1DBF1D84319105A105B105FCF0B4
:10D880006C017D018C3E9105A105B1052CF05BEE8C
:10D89000C52ED12CE12CF12C80E8C816D104E1046E
:10D8A000F104DCF02EEF30E040E050E02C193D09AF
:10D8B0004E095F092D833E834F83588712C044E190
:10D8C000C42ED12CE12CF12C84E190E0A0E0B0E05A
:10D8D0008D839E83AF83B88704C0CD82DE82EF82C2
:10D8E000F886E8EEFEE18491DF011196BE87AD87F0
:10D8F000882329F00E94198FED85FE85F4CFC7019A
:10D90000B6010E94C092E3EEFEE184919F012F5F79
:10D910003F4F3E872D87882329F00E94198FED8580
:10D92000FE85F3CF6D817E818F8198850E94C092A4
:10D930002A964FAD2A97598D6A8D7B8D8CED9EE18D
:10D940000E9485CE4C8D5D8D6E8D7F8D85ED9EE127
:10D950000E9485CE4F855889433051050CF4A2C0F2
:10D960006D817E818F8198850E9459EF20E030E0A3
:10D9700040E850E40E94B8EF69837A838B839C83EC
:10D980002A962FAD2A97398D4A8D5B8D6C8D7D8DB2
:10D990008E8D9F8D0E94CFF32BED3FE049E450E444
:10D9A0000E94B8EF20E030E040E05FE30E94B8EF73
:10D9B0009B01AC0169817A818B819C810E94ACF4CE
:10D9C00069837A838B839C83C301B2010E9459EFE0
:10D9D0002FE632E143E85AE30E94B8EF2B013C0105
:10D9E00049815A816B817C818FEC9EE10E9485CEBA
:10D9F000B301A20189EC9EE10E9485CE2AE939E9B2
:10DA000049E15FE369817A818B819C810E94B8EF53
:10DA100069837A838B839C839B01AC010E94D0F342
:10DA2000A30192010E94ACF4698B7A8B8B8B9C8B47
:10DA300029813A814B815C81C301B2010E94B8EF18
:10DA400020E030E040E05EE30E94B8EF6D8B7E8B1B
:10DA50008F8B988FE9EBFEE184913F015FEF651AB0
:10DA6000750A882321F00E94198FF301F5CF4981AF
:10DA70005A816B817C8183EB9EE10E9485CE49892E
:10DA80005A896B897C898DEA9EE10E9485CE4D89F9
:10DA90005E896F89788D87EA9EE10E9485CE8AE053
:10DAA0000E94198F8D819E81AF81B8858C0D9D1D3F
:10DAB000AE1DBF1DB595A7959795879517FF03C018
:10DAC0008093770503C0EEADFFAD80832F85388945
:10DAD0002F5F3F4F388B2F8739852A963FAF2A9784
:10DAE0004A85498F5B855A8F8C858B8F2401350140
:10DAF00091E09D87E2CCCF93DF93EAE6F4E2849154
:10DB0000EF012196882321F00E94198FFE01F7CFA3
:10DB100083E50E94EB3F882321F00E94A53F80937C
:10DB20004202E7E4FDE18491EF012196882321F090
:10DB30000E94198FFE01F7CF80914202811103C02C
:10DB4000E3E4FDE102C0EFE3FDE18491EF01219602
:10DB5000882321F00E94198FFE01F7CFE7E3FDE152
:10DB60008491EF012196882321F00E94198FFE01F4
:10DB7000F7CF209124043091250440912604509140
:10DB80002704609104117091051180910611909104
:10DB900007110E94D0F3AB01BC0185E39DE10E9417
:10DBA00085CE209128043091290440912A04509177
:10DBB0002B04609108117091091180910A119091C4
:10DBC0000B110E94D0F3AB01BC0182E39DE10E94E6
:10DBD00085CE20912C0430912D0440912E0450913B
:10DBE0002F0460910C1170910D1180910E11909184
:10DBF0000F110E94D0F3AB01BC018FE29DE10E94A6
:10DC000085CEE7E2FDE18491EF012196882321F0A2
:10DC10000E94198FFE01F7CF209124043091250432
:10DC2000409126045091270460912E0270912F029A
:10DC300080913002909131020E94D0F3AB01BC017F
:10DC400085E29DE10E9485CE20912804309129042F
:10DC500040912A0450912B0460913202709133025A
:10DC600080913402909135020E94D0F3AB01BC0147
:10DC700082E29DE10E9485CE20912C0430912D04FA
:10DC800040912E0450912F0460913602709137021A
:10DC900080913802909139020E94D0F3AB01BC010F
:10DCA0008FE19DE10E9485CE8AE0DF91CF910C94B7
:10DCB000198FFF920F931F93CF93DF93F82E092FA5
:10DCC000162FEAE1FDE18491EF012196882321F0EE
:10DCD0000E94198FFE01F7CFEF2DF02F8491EF01F5
:10DCE0002196882321F00E94198FFE01F7CFE8E1E9
:10DCF000FDE18491EF012196882321F00E94198F84
:10DD0000FE01F7CF612F70E080E090E00E94C092AA
:10DD10008AE0DF91CF911F910F91FF900C94198FA2
:10DD20002F923F924F925F926F927F928F929F922B
:10DD3000AF92BF92CF92DF92EF92FF920F931F9319
:10DD4000CF93DF93CDB7DEB7C857D1090FB6F8949C
:10DD5000DEBF0FBECDBFE0917405F0917505EF2BCE
:10DD600011F00C9451772896DFAECEAE28976E2C2A
:10DD700079016A015B01FC0120813181428153817B
:10DD80006C962CAF3DAF4EAF5FAF6C972091781182
:10DD90003091791140917A1150917B116C966CAD54
:10DDA0007DAD8EAD9FAD6C970E94B8EF0E9401F6DD
:10DDB000E0966CAF7DAF8EAF9FAFE097D5018D91B0
:10DDC0009D910D90BC91A02DA0968CAF9DAFAEAF54
:10DDD000BFAFA09720917C1130917D1140917E11B1
:10DDE00050917F11BC01CD010E94B8EF0E9401F655
:10DDF000E4966CAF7DAF8EAF9FAFE497D6012D91C7
:10DE00003D914D915C91A4962CAF3DAF4EAF5FAF6D
:10DE1000A4972091801130918111409182115091ED
:10DE20008311A4966CAD7DAD8EAD9FADA4970E947D
:10DE3000B8EF0E9401F6E8966CAF7DAF8EAF9FAF52
:10DE4000E897D7012D913D914D915C9122962CAF91
:10DE50003DAF4EAF5FAF2297209184113091851175
:10DE6000409186115091871122966CAD7DAD8EAD9B
:10DE70009FAD22970E94B8EF0E9401F660966CAFAA
:10DE80007DAF8EAF9FAF60978091BA0783FF1CC0B4
:10DE900060962CAD3DAD4EAD5FAD60972093120BFB
:10DEA0003093130B4093140B5093150B22968CADAB
:10DEB0009DADAEADBFAD22978093020B9093030B47
:10DEC000A093040BB093050BD801BC91B9A7F8013E
:10DED000F181F9ABD8011296BC91BEABF801F38188
:10DEE000FAAF8091E00A9091E10A891B8F708F3020
:10DEF00021F480E00E948EAEF4CF0091E00AE99612
:10DF00000FAFE9978091E00A082F10E01CA30BA344
:10DF10008091060B9091070BA091080BB091090B13
:10DF2000E0968CAC9DACAEACBFACE097881A990A79
:10DF3000AA0ABB0A80910A0B90910B0BA0910C0BC3
:10DF4000B0910D0BE4962CAC3DAC4EAC5FACE497BD
:10DF5000281A390A4A0A5B0A80910E0B90910F0B1E
:10DF6000A091100BB091110BE8962CAD3DAD4EADCC
:10DF70005FADE897281B390B4A0B5B0B2DA33EA323
:10DF80004FA358A78091120B9091130BA091140BE3
:10DF9000B091150B60960CAD1DAD2EAD3FAD6097E9
:10DFA000081B190B2A0B3B0B0DA71EA72FA738AB7D
:10DFB000012B022B032B09F4BCC080915811811155
:10DFC0004BC060915C0470915D0480915E049091FF
:10DFD0005F040E9414F520913A0230913B026217CF
:10DFE00073070CF039C060962CAD3DAD4EAD5FAD02
:10DFF00060972093120B3093130B4093140B5093A4
:10E00000150B22968CAD9DADAEADBFAD2297809322
:10E01000020B9093030BA093040BB093050BEAE65D
:10E02000F4E284918F010F5F1F4F811103C0E1E77C
:10E03000F0E204C00E94198FF801F3CF84918F01A0
:10E040000F5F1F4F882321F00E94198FF801F6CF30
:10E050001DA61EA61FA618AA94E0699E8001112481
:10E060000B5D1D4F6DA57EA58FA598A90E9459EF48
:10E07000D8012D913D914D915C910E94B8EF6B01BB
:10E080007C0120E030E0A9010E94F6F587FF04C082
:10E09000F7FAF094F7F8F09460918411709185117B
:10E0A00080918611909187110E9414F59B01AC011B
:10E0B000A8E5B2E00E94B0F30E9459EFA7019601D3
:10E0C0000E9453EF87FF39C060960CAD1DAD2EAD99
:10E0D0003FAD60970093120B1093130B2093140B1A
:10E0E0003093150B22962CAD3DAD4EAD5FAD229712
:10E0F0002093020B3093030B4093040B5093050BBA
:10E10000EAE6F4E284918F010F5F1F4F811103C093
:10E11000E2E5F0E204C00E94198FF801F3CF849188
:10E120008F010F5F1F4F882321F00E94198FF80184
:10E13000F6CF1DA61EA61FA618AAD501C4018827C2
:10E14000B7FD83959927AA27BB27782E57FE03C0D2
:10E15000382F3260732E8DA19EA1AFA1B8A5B7FF55
:10E1600003C0972D9460792E0DA51EA52FA538A963
:10E1700037FF03C0172D1860712E24E0629E8001C6
:10E1800011240B5D1D4F6DA57EA58FA598A90E943A
:10E1900059EFD8012D913D914D915C910E94B8EFBE
:10E1A0006B017C0120E030E0A9010E94F6F587FFB9
:10E1B00004C0C701B601905802C0C701B60120E0F3
:10E1C00030E040E05FE30E94D0F30E9419F56AABB3
:10E1D0007BAB8CAB9DAB88E60BA11CA1809FF001B3
:10E1E000819FF00D1124EF56FD4E1082EA5BFF4F28
:10E1F0007082B501A401B7FE07C044275527BA01B4
:10E20000481959096A097B0988E60BA11CA1809F5E
:10E21000F001819FF00D1124EF56FD4E458B568B7A
:10E22000678B708F2C962CAE3DAE4EAE5FAE2C97AA
:10E2300057FE0DC088279927DC0182199309A4098C
:10E24000B5092C968CAF9DAFAEAFBFAF2C9728E62B
:10E250000BA11CA1209FF001219FF00D1124EF566E
:10E26000FD4E2C968CAD9DADAEADBFAD2C97818F84
:10E27000928FA38FB48F0DA11EA12FA138A537FFB8
:10E2800007C030952095109501951F4F2F4F3F4F98
:10E29000E8E67E2EABA1BCA17A9EF0017B9EF00D3C
:10E2A0001124EF56FD4E058F168F278F30A38AA9B4
:10E2B0009BA9ACA9BDA981A392A3A3A3B4A32396B0
:10E2C0004FAF2397752EF62FE72F2C968CAD9DAD73
:10E2D000AEADBFAD2C97481759076A077B0778F496
:10E2E00029969FAD299723969FAF23972A967FACB7
:10E2F0002A972B96FFAD2B972C96EFAD2C97239654
:10E300008FAD2397972DAF2FBE2F80179107A207B0
:10E31000B30710F4D901C8010AA91BA92CA93DA96A
:10E3200080179107A207B30710F4D901C80128E6A6
:10E330000BA11CA1209FF001219FF00D1124EF568D
:10E34000FD4E85A396A3A7A3B0A70697A105B10587
:10E3500008F4A0C5DF01AE59BF4F809140049091F1
:10E3600041048D939C9361A6452B462B472B09F0C6
:10E370005F9888E60BA11CA1809FF001819FF00DA2
:10E380001124EF56FD4E818D928DA38DB48D892B76
:10E390008A2B8B2B11F08A98479888E60BA11CA139
:10E3A000809FF001819FF00D1124EF56FD4E858D69
:10E3B000968DA78DB0A1892B8A2B8B2B31F0809164
:10E3C000080181708093060147982AA93BA94CA9AE
:10E3D0005DA9232B242B252B09F465C58091BF074C
:10E3E000882319F081508093BF07611004C01298F0
:10E3F00080E28093BF076090B6077090B7070091E6
:10E40000B8071091B9079301A80169A579A98EA948
:10E410009AAD0E9453EF87FF04C069A679AA0EAB9C
:10E420001AAFC501B4010E9459EF20917D123091BD
:10E430007E1240917F12509180120E94B8EF269672
:10E440006CAF7DAF8EAF9FAF2697698B7A8B8B8B2E
:10E450009C8BC201B1010E9459EF20918112309131
:10E46000821240918312509184120E94B8EF2B01C6
:10E470003C016D8B7E8B8F8B988F6DA17EA18FA1C0
:10E4800098A50E9459EF20918512309186124091F3
:10E490008712509188120E94B8EF4B015C01698F7E
:10E4A0007A8F8B8F9C8F2091891230918A124091A4
:10E4B0008B1250918C12C701B6010E94B8EF6B010C
:10E4C0007C016D8F7E8F8F8F98A388E60BA11CA196
:10E4D000809FF001819FF00D1124EF56FD4E25899C
:10E4E00036894789508D2DA33EA34FA358A72630C8
:10E4F00031054105510508F4DFC42896AEADBFAD26
:10E500002897CD90DD90ED90FC9020E030E0A901BF
:10E51000C701B6010E9453EF8111EDC426962CADC0
:10E520003DAD4EAD5FAD2697CA01B9010E94B8EF6F
:10E530006B017C01A3019201C301B2010E94B8EFFB
:10E540009B01AC01C701B6010E94D0F36B017C01B5
:10E55000A5019401C501B4010E94B8EF9B01AC0173
:10E56000C701B6010E94D0F30E943BF628E60BA13A
:10E570001CA1209FF001219FF00D1124EF56FD4EAC
:10E58000658776878787908B88E60BA11CA1809F83
:10E59000F001819FF00D1124EF56FD4E4584568405
:10E5A00067847088A301920160E070E080E89FE3D7
:10E5B0000E94ACF464966CAF7DAF8EAF9FAF649752
:10E5C00029A539A94EA95AAD0E94B8EF4B015C01AB
:10E5D0008091E00A9091DE0A891B8F7027968FAF99
:10E5E0002797A501940160E074E284E799E40E9412
:10E5F000ACF40E9401F66B017C0127968FAD279742
:10E600008250863008F486C4A5019401C301B2018A
:10E610000E94B8EF9B01AC010E94B8EF68966CAF06
:10E620007DAF8EAF9FAF689788E6ABA1BCA18A9FF4
:10E6300080018B9F100D11240F561D4E68962CAD36
:10E640003DAD4EAD5FAD6897D80111962D933D93CA
:10E650004D935C93149795962D913D914D915C91BE
:10E6600098972EAB3FAB48AF59AFCA01B9010E9492
:10E6700057EF6AAF7BAF8CAF9DAF9B01AC01C5017B
:10E68000B4010E94B8EF0E9496F40E9419F5A89672
:10E690006CAF7DAF8EAF9FAFA897F801EE5AFF4FDA
:10E6A00060837183828393838E010F5E1F4F2A964E
:10E6B0001FAF0EAF2A970051110924961FAF0EAF5E
:10E6C00024970EE917E0AC961FAF0EAFAC978E0102
:10E6D0000F5D1F4F1AA309A324960EAD1FAD2497FB
:10E6E000AA961FAF0EAFAA97312C212C10E819A7BC
:10E6F0000FE309AB2A96AEADBFAD2A972D913D91A0
:10E700004D915D912A96BFAFAEAF2A97C501B40176
:10E710000E94B8EF6B017C01AA96EEADFFADAA97FF
:10E720006193719381939193AA96FFAFEEAFAA97ED
:10E7300020E030E0A9010E94F6F587FF04C0F7FA57
:10E74000F094F7F8F094AC96AEADBFADAC974D90A9
:10E750005D906D907D90AC96BFAFAEAFAC97A701CA
:10E760009601C301B2010E9453EF87FD0DC409A1B8
:10E770001AA12A962EAD3FAD2A970217130709F06A
:10E78000B9CF20E030E040E85FE3632D722D89A52A
:10E7900099A90E9453EF87FF58C07E0131E1E30E33
:10E7A000F11C24960EAD1FAD2497232D322D49A5C3
:10E7B00059A9D8016D917D918D919C910E94B8EFDE
:10E7C000F80161937193819391938F01EE16FF0687
:10E7D00061F728E60BA11CA1209FC001219F900D8D
:10E7E00011249C012F563D4E790189010E5A1F4F6D
:10E7F000A8966CAD7DAD8EAD9FADA8970E9457EFEA
:10E80000232D322D49A559A90E94B8EF0E9419F570
:10E81000D8016D937D938D939C931397232D322D67
:10E8200049A559A9632D722D89A599A90E94B8EF10
:10E8300068962CAD3DAD4EAD5FAD68970E94B8EFC8
:10E84000F70161837283838394832AAD3BAD4CAD22
:10E850005DAD64966CAD7DAD8EAD9FAD64970E944D
:10E86000B8EF69A77AA78BA79CA70DA11EA12FA11E
:10E8700038A5012B022B032B09F09EC388E62BA1A0
:10E880003CA1829F8001839F100D11240F561D4EC5
:10E89000F801818D928DA38DB48D892B8A2B8B2BC2
:10E8A00009F08AC3858D968DA78DB0A1892B8A2BFF
:10E8B0008B2B09F081C3209142113091431140917B
:10E8C00044115091451169A57AA58BA59CA50E947C
:10E8D000B8EF0E9496F40E9419F52B013C01F80153
:10E8E000E95BFF4F108288E62BA13CA1829F80014B
:10E8F000839F100D11240F561D4EF801E25AFF4F51
:10E900004082518262827382C301B2010E9457EF3A
:10E9100029A53AA54BA55CA50E94ACF46AAF7BAFD4
:10E920008CAF9DAFD80151966D937D938D939C9341
:10E930005497F801E95BFF4F8081882381F17801CA
:10E94000B8E4EB0EF11C37962091920730919307B3
:10E9500040919407509195076081718182819381E4
:10E960000E94B8EF2AAD3BAD4CAD5DAD0E94B8EF53
:10E970002091841130918511409186115091871119
:10E980000E94B8EF9B01AC0160E074E284EF99E46F
:10E990000E94ACF40E9419F5F7017183608388E648
:10E9A0000BA11CA1809FF001819FF00D1124EF5657
:10E9B000FD4E21813281438154812C962CAF3DAF95
:10E9C0004EAF5FAF2C97CA01B9010E943BF6362EBD
:10E9D000272E8C0142E857E062965FAF4EAF6297F8
:10E9E0003E0151E1650E711C82E897E09FAB8EAB52
:10E9F00024964EAC5FAC24973DA62DA209A719AB77
:10EA00001AAAD201CD90DD90ED90FD902D0120E06D
:10EA100030E0A901C701B6010E94F6F587FF04C0E6
:10EA2000F7FAF094F7F8F094EEA9FFA9819091908D
:10EA3000A190B190FFABEEABA7019601C501B40167
:10EA40000E9453EF87FDD8C564147504D1F627964C
:10EA50005FAD2797552309F448C6C090E20AD090CD
:10EA6000E30AE090E40AF090E50A2DEB37E346E88C
:10EA700055E3C701B6010E9453EF87FD36C6C701B3
:10EA8000B6010E943BF66B017C019B01AC01632D3A
:10EA9000722DC8010E9453EF87FD03C03C2C2D2C22
:10EAA00087019601A701632D722DC8010E94ACF465
:10EAB00068966CAF7DAF8EAF9FAF689786EE9AE099
:10EAC00028969FAF8EAF289720E030E040E85FE3C4
:10EAD0002AAB3BAB4CAB5DAB1EAA2896AEADBFAD2F
:10EAE00028972D913D914D915D912896BFAFAEAF86
:10EAF000289768966CAD7DAD8EAD9FAD68970E94EE
:10EB0000B8EF4B015C012496EEADFFAD2497C190A8
:10EB1000D190E190F1902496FFAFEEAF2497FEA93B
:10EB2000FF2391F02AA93BA94CA95DA90E94B8EF47
:10EB30004B015C012AA93BA94CA95DA9C701B601FB
:10EB40000E94B8EF6B017C01A7019601C501B401D9
:10EB50000E94F6F520E030E0A90118160CF092C5ED
:10EB6000C701B6010E94F6F518160CF486C520E020
:10EB700030E0A901C501B4010E9453EF87FD7DC5B6
:10EB80002601370177FA709477F87094A301920107
:10EB9000C501B4010E94F6F5181614F424013501DC
:10EBA0006296AEADBFAD6297CD90DD90ED90FD90D9
:10EBB0006296BFAFAEAF6297A3019201C701B601E3
:10EBC0000E9453EF87FF15C0A3019201C701B60150
:10EBD0000E94ACF49B01AC016AA97BA98CA99DA9F8
:10EBE0000E94B8EF6AAB7BAB8CAB9DABBEA9BF5F9D
:10EBF000BEABE6EFFAE028962EAD3FAD2897E217C0
:10EC0000F30709F06ACF3EA9332361F02AA93BA993
:10EC10004CA95DA9632D722DC8010E94B8EF362E54
:10EC2000272E8C0124EA30E74DE75FE3632D722D38
:10EC3000C8010E94B8EF6B017C012091BB073091A5
:10EC4000BC074091BD075091BE070E9453EF87FD5E
:10EC500042C58DA59DA1A9A5B9A98093BB07909395
:10EC6000BC07A093BD07B093BE0728E64BA15CA1EB
:10EC7000249FC001259F900D1124DC01AF56BD4E8D
:10EC80007D01232D322DA801632D722DC8010E9414
:10EC9000B8EFF70161877287838794876AAD7BAD90
:10ECA0008CAD9DAD90589B01AC010E94D0F3D70173
:10ECB0001D962D913D914D915C9150970E94B8EF1A
:10ECC0009B01AC016BE077ED83E29BE30E94CFF305
:10ECD0009B01AC018BE097EDA3E2BBE3F7018583D9
:10ECE0009683A783B08710812C966CAD7DAD8EADD9
:10ECF0009FAD2C970E9453EF18160CF4FBC483E0D1
:10ED0000182B88E62BA13CA1829FF001839FF00D78
:10ED10001124EF56FD4E108380E1FE013196A6EEE0
:10ED2000BAE001900D928A95E1F72C968CAD9DADDD
:10ED3000AEADBFAD2C978093E20A9093E30AA09307
:10ED4000E40AB093E50AE0960CAD1DAD2EAD3FADE3
:10ED5000E0970093060B1093070B2093080B30935A
:10ED6000090BE4962CAD3DAD4EAD5FADE49720931D
:10ED70000A0B30930B0B40930C0B50930D0BE89642
:10ED80008CAD9DADAEADBFADE89780930E0B90936B
:10ED90000F0BA093100BB093110B60960CAD1DAD33
:10EDA0002EAD3FAD60970093120B1093130B209381
:10EDB000140B3093150B6C962CAD3DAD4EAD5FAD85
:10EDC0006C972093F60A3093F70A4093F80A509311
:10EDD000F90AA0968CAD9DADAEADBFADA097809366
:10EDE000FA0A9093FB0AA093FC0AB093FD0AA4963A
:10EDF0000CAD1DAD2EAD3FADA4970093FE0A109350
:10EE0000FF0A2093000B3093010B22962CAD3DADF1
:10EE10004EAD5FAD22972093020B3093030B4093CE
:10EE2000040B5093050B9091E00A8091E10A98132E
:10EE300003C084E68093DD0AE9968FADE9978F5F82
:10EE40008F708093E00A8091E00A9091DF0A8150F0
:10EE50008F70891351C41091E10A1BA30091E00A3D
:10EE60000DA728E61BA10DA51013D1C4812C912C50
:10EE7000A12CB12C1DA219A619AA1EAE212C312C31
:10EE800000E010E02DA53BA12313CEC421143104D2
:10EE900009F07FC580916F00826080936F0081E0F0
:10EEA000ECC680E0EAC66090B2077090B3070091AC
:10EEB000B4071091B507A7CA818D928DA38DB48D2B
:10EEC0000697A105B10508F018CB858D968DA78D05
:10EED000B0A10697A105B10508F00FCB20E030E006
:10EEE000A901C701B6010E94F6F587FF04C0F7FA31
:10EEF000F094F7F8F09488E60BA11CA1809FF00134
:10EF0000819FF00D1124EF56FD4EC586D686E7860B
:10EF1000F08A3ACB8091AE079091AF07A091B007ED
:10EF2000B091B107C816D906EA06FB0608F06CCB0B
:10EF30008C199D09AE09BF09BC01CD01660F771F71
:10EF4000881F991F27964FAD2797042F10E020E0C8
:10EF500030E0A90198010E9472F3CA01B9010E9430
:10EF600057EF0E9401F66C0D7D1D8E1D9F1D0E94A6
:10EF700057EF9B01AC0160E074E284E799E40E94E2
:10EF8000ACF44B015C0140CBA7019601C301B20177
:10EF90000E94ACF47B018C019B01AC01632D722DAE
:10EFA00089A599A90E94F6F518160CF0E0CB3E2C25
:10EFB0002F2C09A719ABDBCB0AA91BA92CA93DA9AA
:10EFC000012B022B032B49F020919A0730919B07CC
:10EFD00040919C0750919D0708C020919607309161
:10EFE0009707409198075091990769A57AA58BA535
:10EFF0009CA50E94B8EF0E9496F40E9419F52B017F
:10F000003C012AA93BA94CA95DA9232B242B252B24
:10F01000C9F020E030E0A901609192077091930758
:10F0200080919407909195070E9453EF882351F0A7
:10F0300081E00DA51EA52FA538A9101611061206F0
:10F0400013060CF080E098E62BA13CA1929F800172
:10F05000939F100D11240F561D4E180137E4230EF7
:10F06000311CD1018C93882309F4B3C02091F60A96
:10F070003091F70A4091F80A5091F90A6C966CADFC
:10F080007DAD8EAD9FAD6C970E94CFF36DA77EA72F
:10F090008FA798AB2091FA0A3091FB0A4091FC0AA5
:10F0A0005091FD0AA0966CAD7DAD8EAD9FADA09741
:10F0B0000E94CFF34B015C012091FE0A3091FF0AC0
:10F0C0004091000B5091010BA4966CAD7DAD8EADBF
:10F0D0009FADA4970E94CFF36B017C012DA53EA5A7
:10F0E0004FA558A9CA01B9010E94B8EF6DA77EA724
:10F0F0008FA798ABA5019401C501B4010E94B8EF98
:10F100009B01AC016DA57EA58FA598A90E94D0F3A7
:10F110004B015C01A7019601C701B6010E94B8EF3F
:10F120009B01AC01C501B4010E94D0F30E943BF6E3
:10F130006B017C012091020B3091030B4091040B79
:10F140005091050B22966CAD7DAD8EAD9FAD229793
:10F150000E94CFF3A70196010E94ACF46B017C01E1
:10F16000F801E25BFF4F608371838283938320E029
:10F1700030E040E450E40E94F6F518161CF4F1016A
:10F18000108227C0209192073091930740919407F5
:10F1900050919507C701B6010E94B8EF9B01AC01E1
:10F1A00060918E0770918F078091900790919107E1
:10F1B0000E94ACF429A53AA54BA55CA50E94B8EF26
:10F1C0000E9419F5641575058605970510F42B0145
:10F1D0003C018091591290915A12A0915B12B0910A
:10F1E0005C120EA91FA928AD39AD80179107A2079F
:10F1F000B30708F4DFC02DA13EA14FA158A5232BD2
:10F20000242B252B41F160915D1270915E1280914B
:10F210005F12909160126415750586059705D8F404
:10F220002EA93FA948AD59AD0E9463F36B017C0143
:10F230002DA13EA14FA158A5C301B2010E9463F3C5
:10F24000C616D706E806F90630F4C701B6010E94D3
:10F2500072F329013A0188E60BA11CA1809FF001FD
:10F26000819FF00D1124EF56FD4EC18CD28CE38CA2
:10F27000F48CC114D104E104F10431F16091611204
:10F2800070916212809163129091641264157505F9
:10F2900086059705C8F42EA93FA948AD59AD0E942F
:10F2A00063F34B015C01A7019601C301B2010E9407
:10F2B00063F386169706A806B90630F4C501B401B3
:10F2C0000E9472F329013A0188E60BA11CA1809FDC
:10F2D000F001819FF00D1124EF56FD4EC58CD68CA8
:10F2E000E78CF0A0C114D104E104F10431F1609184
:10F2F0006512709166128091671290916812641580
:10F30000750586059705C8F42EA93FA948AD59ADE6
:10F310000E9463F34B015C01A7019601C301B20196
:10F320000E9463F386169706A806B90630F4C50155
:10F33000B4010E9472F329013A0188E60BA11CA1D5
:10F34000809FF001819FF00D1124EF56FD4EC1A06A
:10F35000D2A0E3A0F4A0C114D104E104F10409F4A3
:10F36000C2CA6091691270916A1280916B12909179
:10F370006C12641575058605970508F0B4CA2EA9A8
:10F380003FA948AD59AD0E9463F34B015C01A70151
:10F390009601C301B2010E9463F386169706A80680
:10F3A000B90608F0A0CAC501B4010E9472F3290190
:10F3B0003A0199CA2DA13EA14FA158A5232B242B78
:10F3C000252BC9F160915D1270915E1280915F12E0
:10F3D00090916012641575058605970560F50E9489
:10F3E00057EF2AAD3BAD4CAD5DAD0E94B8EF6B0160
:10F3F0007C016DA17EA18FA198A50E9457EF4B01C2
:10F400005C01C301B2010E9457EFA50194010E9463
:10F41000B8EF9B01AC01C701B6010E9453EF87FF13
:10F420000AC0A5019401C701B6010E94ACF40E9474
:10F4300019F52B013C0188E60BA11CA1809FF0016E
:10F44000819FF00D1124EF56FD4E818C928CA38C80
:10F45000B48C81149104A104B104B9F160916112DA
:10F460007091621280916312909164126415750517
:10F470008605970550F50E9457EF2AAD3BAD4CAD80
:10F480005DAD0E94B8EF6B017C01C501B4010E9423
:10F4900057EF4B015C01C301B2010E9457EFA50178
:10F4A00094010E94B8EF9B01AC01C701B6010E9414
:10F4B00053EF87FF0AC0A5019401C701B6010E945E
:10F4C000ACF40E9419F52B013C0188E60BA11CA1AC
:10F4D000809FF001819FF00D1124EF56FD4E858C29
:10F4E000968CA78CB0A081149104A104B104B9F149
:10F4F0006091651270916612809167129091681206
:10F50000641575058605970550F50E9457EF2AADDD
:10F510003BAD4CAD5DAD0E94B8EF6B017C01C50108
:10F52000B4010E9457EF4B015C01C301B2010E947C
:10F5300057EFA50194010E94B8EF9B01AC01C701F0
:10F54000B6010E9453EF87FF0AC0A5019401C701CD
:10F55000B6010E94ACF40E9419F52B013C0188E62B
:10F560000BA11CA1809FF001819FF00D1124EF568B
:10F57000FD4EC1A0D2A0E3A0F4A0C114D104E104C7
:10F58000F10409F4B0C96091691270916A12809116
:10F590006B1290916C12641575058605970508F03D
:10F5A000A2C90E9457EF2AAD3BAD4CAD5DAD0E94A4
:10F5B000B8EF4B015C01C701B6010E9457EF6B0128
:10F5C0007C01C301B2010E9457EFA70196010E947E
:10F5D000B8EF9B01AC01C501B4010E9453EF87FF56
:10F5E00082C9A7019601C501B4010E94ACF40E9432
:10F5F00019F52B013C0177C9FAA9FF2331F1A501C7
:10F600009401632D722DC8010E94B8EF4B015C017B
:10F610002DA53DA149A559A9C701B6010E94B8EF82
:10F620009B01AC01C501B4010E9453EF87FF22C0CA
:10F63000A7019601C501B4010E94ACF46DA77DA39A
:10F6400089A799AB21E02AABFFC9A7019601C501A3
:10F65000B4010E94ACF49B01AC016DA57DA189A50C
:10F6600099A90E94B8EF6DA77DA389A799AB31E056
:10F670003AABEAC941E04AABE7C9A7019601C50127
:10F68000B40113C0C701B6010E9453EF87FD09C042
:10F6900020E030E0A901C501B4010E94F6F518167A
:10F6A0004CF4A5019401C701B6010E94CFF32B01D0
:10F6B0003C0176CA2401350177FA709477F870948A
:10F6C000A3019201C701B6010E9453EF87FD68CAEA
:10F6D0002601370165CA2DA53DA149A559A9C70134
:10F6E000B6010E9453EF87FFB4CA3DA42DA009A51F
:10F6F00019A9AFCA81E004CBF090E00A8FEF8F0D1B
:10F700008F708BA3B090DF0A8091E00AB81609F4DD
:10F7100054C0C12CD12C0BA10B1509F44EC0602E86
:10F72000712C28E6269D8001279D100D11240F566F
:10F730001D4ED8018C9183FD2BC00EAF1AAB011565
:10F74000110541F11996BC91BDA7F801F285FDA301
:10F75000D8011B96BC91B9A7F801F485F9ABD80183
:10F7600015962D903D904D905C901897A2019101B7
:10F770006DA57DA189A59F2F0E9453EF811186C1A0
:10F78000C114D10439F0F601808180FD7FC102C02F
:10F79000CEAEDAAA8BA181508F708BA38091DF0A45
:10F7A0008B1103C0CEACDAA8B6CF0BA10B1529F094
:10F7B00081E08B0D8F70B82EF1CF1091DF0A1BA363
:10F7C000C12CD12C8091E00A0BA1801709F443CB06
:10F7D000802E912C28E6289D8001299D100D112452
:10F7E0000F561D4ED8018C9183FD0AC05801C114DB
:10F7F000D10439F0C6010E941362811102C0C5C153
:10F8000056018BA18F5F8F708BA36501DBCF802F9B
:10F8100081508F70289FF0011124EF56FD4E90818A
:10F8200093FF24CB8DA71ECB48E6439FC001112434
:10F83000DC01AF56BD4E1D018C9183FD19C015969C
:10F840006D917D918D919C9118970E943BF6F62EBB
:10F85000E72ED82EC92E0115110509F48CC0F80128
:10F86000808180FD0AC0D1018C9180FD06C083C0DB
:10F87000FDA0E9A4D9A8CEAC83C0F8018081816045
:10F880008083C8010E941362811171C0F8016181F7
:10F890007281838194810E943BF62B013C019B0184
:10F8A000AC0160E070E080E89FE30E94ACF44B01A3
:10F8B0005C019B01AC016F2D7E2D8D2D9C2D0E9436
:10F8C000B8EF69837A838B839C832DA139A549A9DD
:10F8D0005EADC501B4010E94B8EF698B7A8B8B8B4A
:10F8E0009C8BAE014F5F5F4FBE016F5E7F4FC801C3
:10F8F0000E94A2BCF801E95BFF4F80818823B9F127
:10F900002091920730919307409194075091950769
:10F91000379660817181828193810E94B8EF209136
:10F9200084113091851140918611509187110E9468
:10F93000B8EF4B015C019B01AC01C301B2010E9415
:10F94000B8EF0E9419F5F801E65BFF4F7183608301
:10F95000A50194016F2D7E2D8D2D9C2D0E94B8EF59
:10F960000E9419F5F801E45BFF4F71836083D801B1
:10F970008C918E7F8C938F2C9E2CAD2CBC2C810176
:10F980008BA18F5F8F708BA3FDA2E9A6D9AACEAE03
:10F9900079CAF101808181608083C8010E9413626D
:10F9A00081116FC0D10111966D917D918D919C91C6
:10F9B00014970E943BF66B017C019B01AC0160E057
:10F9C00070E080E89FE30E94ACF42B013C012DEC39
:10F9D0003CEC4CE45DE30E94B8EF69837A838B834F
:10F9E0009C839401A501C301B2010E94B8EF698B09
:10F9F0007A8B8B8B9C8BAE014F5F5F4FBE016F5E2E
:10FA00007F4FC1010E94A2BCF101E95BFF4F8081E1
:10FA10008823B9F120919207309193074091940780
:10FA200050919507379660817181828193810E9400
:10FA3000B8EF209184113091851140918611509139
:10FA400087110E94B8EF4B015C019B01AC01C7011B
:10FA5000B6010E94B8EF0E9419F5F101E65BFF4F75
:10FA6000718360832DEC3CEC4CE45DE3C501B40193
:10FA70000E94B8EF0E9419F5F101E45BFF4F71831A
:10FA80006083F10180818E7F808304CA28E6269DF1
:10FA9000F001279DF00D1124EF56FD4E808181FD70
:10FAA00043C0C114D10441F0D6011596CD90DD902C
:10FAB000ED90FC90189708C08BE0C82E87EDD82EEB
:10FAC00083E2E82E8BE3F82EB8E6B69DF001B79DF1
:10FAD000F00D1124EF56FD4E81899289A389B489D6
:10FAE000BC01CD0190589B01AC010E94D0F3F801FC
:10FAF00025853685478550890E94B8EF9B01AC016A
:10FB0000C701B6010E94CFF3E62E872E982EA92EAC
:10FB1000262F372F482F592F6DA57DA189A599A98B
:10FB20000E9453EF87FF04C0EDA48DA099A4A9A85B
:10FB30002E2D382D492D5A2DC201B1010E9453EFAF
:10FB4000882309F427CEF8E6F69DC001F79D900DB5
:10FB500011249C012F563D4E6901D9018C91816081
:10FB60008C93C8010E941362882329F0F6018081DA
:10FB70008E7F80830FCE8E2D982DA92DBA2DF60164
:10FB800085839683A783B08705CED6018C9181FDAE
:10FB900052C0D60115962D913D914D915C911897CB
:10FBA0002DA73EA74FA758AB1501B5E02B0E311C72
:10FBB000F8014580568067807084A30192016DA58D
:10FBC0007EA58FA598A90E9453EF87FF34C0F60148
:10FBD00081899289A389B489BC01CD0190589B0188
:10FBE000AC010E94D0F3D6011D962D913D914D910F
:10FBF0005C9150970E94B8EF9B01AC016DA57EA56A
:10FC00008FA598A90E94CFF36B017C019B01AC01E9
:10FC1000C301B2010E94F6F518166CF4D8018C915C
:10FC200081608C93C5010E9413628823E1F0F80182
:10FC300080818E7F808318E6189DF001199DF00D5C
:10FC40001124EF56FD4E218532854385548565810B
:10FC50007681878190850E9453EF8111D2CD0BA1CF
:10FC60000093DF0ACECDD101CD92DD92ED92FC92D0
:10FC700013970BA10093DF0ADECFC858DF4F0FB6F2
:10FC8000F894DEBF0FBECDBFDF91CF911F910F91D2
:10FC9000FF90EF90DF90CF90BF90AF909F908F90AC
:10FCA0007F906F905F904F903F902F90089580913C
:10FCB000E00A9091E10A891B8F708F3021F480E077
:10FCC0000E948EAEF4CF8091E00A8F5F8F70E0913A
:10FCD000E00A98E69E9FF0011124EF56FD4EDF01E9
:10FCE0001D929A95E9F798E090834091060B509108
:10FCF000070B6091080B7091090B458B568B678B36
:10FD0000708F40910A0B50910B0B60910C0B70910E
:10FD10000D0B418F528F638F748F40910E0B50915A
:10FD20000F0B6091100B7091110B458F568F678FE1
:10FD300070A34091120B5091130B6091140B7091B2
:10FD4000150B41A352A363A374A32091E00A9091E1
:10FD5000E10A291303C094E69093DD0A8093E00A38
:10FD600080916F00826080936F0008959091E00A07
:10FD70008091E10A981306C08091740590917505F1
:10FD8000892B21F080E00E948EAEF0CF08954F9233
:10FD90005F926F927F928F929F92AF92BF92CF921B
:10FDA000DF92EF92FF92CF93DF9320912404309162
:10FDB0002504409126045091270460914C047091D1
:10FDC0004D0480914E0490914F040E94D0F3AB01FA
:10FDD000BC0188E591E20E9485CE209128043091F3
:10FDE000290440912A0450912B0460915004709191
:10FDF000510480915204909153040E94D0F3AB01BE
:10FE0000BC0184E591E20E9485CE20912C043091C2
:10FE10002D0440912E0450912F0460915404709150
:10FE2000550480915604909157040E94D0F3AB0181
:10FE3000BC0180E591E20E9485CE4091580450912A
:10FE4000590460915A0470915B048CE491E20E9421
:10FE500085CE80916F00982F927081FF05C08091B0
:10FE60006F008D7F80936F004090681150906911F2
:10FE700060906A1170906B1180906C1190906D1170
:10FE8000A0906E11B0906F11C0907011D090711150
:10FE9000E0907211F0907311992329F080916F0016
:10FEA000826080936F00E2E4F1E28491EF01219699
:10FEB000882321F00E94198FFE01F7CFC301B20100
:10FEC0000E94C092EEE3F1E28491EF012196882333
:10FED00021F00E94198FFE01F7CFC501B4010E94E5
:10FEE000C092EAE3F1E28491EF012196882321F0A8
:10FEF0000E94198FFE01F7CFC701B6010E94C09280
:10FF00008AE0DF91CF91FF90EF90DF90CF90BF908C
:10FF1000AF909F908F907F906F905F904F900C94D8
:10FF2000198F2F923F924F925F926F927F928F9292
:10FF30009F92AF92BF92CF92DF92EF92FF920F9378
:10FF40001F93CF93DF93CDB7DEB762970FB6F894C8
:10FF5000DEBF0FBECDBF8091BA0783FDB4C183E57C
:10FF60000E9434408C87811106C082E50E94344093
:10FF7000882309F4A8C10E94B43F0E9414F5CB0164
:10FF80000E94C3410E94B43F20E030E040EA50E4C8
:10FF90000E94F6F5181614F40E94D6CEEEE2F1E2B5
:10FFA0008491FB83EA83882371F0082E000C990B5F
:10FFB0000E940BA04A815B814F5F5F4F5B834A8346
:10FFC000FA018491F0CF8DE090E00E940BA08AE0CE
:10FFD00090E00E940BA081E08093240210924711D0
:10FFE00080911011809378051A821B821C821D82D9
:10FFF000188619861A861B8619821D86FCE3FE87E1
:020000021000EC
:100000002CE12F8736E4388B312C212C40E8498BAA
:100010005FEB5A8B812C912C5401609142047091BA
:100020004304072E000C880B990B0E9459EF7B01AB
:100030008C019B01AC01632D722D89899A890E94E4
:1000400053EF882341F120914404309145044091BD
:100050004604509147048C85B70181110CC0C8013A
:100060000E9453EF881F8827881F89833E2C2F2CDE
:10007000098B1A8B10C0C8010E9453EF87FF06C07E
:10008000E2E3F1E28491FB83EA83E8C03E2C2F2C6B
:10009000098B1A8B19820E944E626B017C01DC0174
:1000A000CB01288539854A855B85821B930BA40B80
:1000B000B50BB7FD3BC0D701C60188519C4FAF4F70
:1000C000BF4F88879987AA87BB870E949058E6E32D
:1000D000F1E284913F019FEF691A790A882321F0A8
:1000E0000E94198FF301F5CF81149104A104B1048A
:1000F000B9F0D501C401805F984DAF4FBF4FBC012F
:10010000CD016C197D098E099F0928EE33E040E08E
:1001100050E00E9472F3CA01B9010E94C09203C06C
:100120008FE30E94198F8AE00E94198F80E00E945D
:100130008EAE0E944E626093EB107093EC10809331
:10014000ED109093EE10A0914404AE83B09145045D
:10015000BF8300914604109147040E94092D2E810F
:100160003F81A801632D722D89899A890E94CFF35E
:100170002B013C0120E030E0A9010E94F6F587FF49
:1001800004C077FA709477F8709481149104A104F4
:10019000B10459F420E030E040E85FE3C301B2016C
:1001A0000E9453EF87FF0DC00AC020E030E040E41A
:1001B00050E4C301B2010E94F6F5181614F446018A
:1001C0005701E981EE2391F12A813B814C815D81C8
:1001D000211531054105510541F0D701C601821BAA
:1001E000930BA40BB50BB7FD21C02E813F81A80155
:1001F0006D857E858F8598890E94CFF320E030E061
:1002000040EC5FE30E9453EF87FD3ACFD701C60170
:10021000805A9541AF4FBF4F8A839B83AC83BD8388
:100220009E819D87AF81AE870F87188B80912402B6
:10023000882309F425CF81149104A104B10409F4A1
:10024000ECCEB0E1CB1AB7E2DB0AE108F108C8183E
:10025000D908EA08FB08F7FE13CFDFCE882361F048
:10026000082E000C990B0E940BA0EA81FB813196AD
:10027000FB83EA838491F2CF8DE090E00E940BA093
:100280008AE090E00E940BA08091240281E080939C
:10029000471162960FB6F894DEBF0FBECDBFDF9157
:1002A000CF911F910F91FF90EF90DF90CF90BF9073
:1002B000AF909F908F907F906F905F904F903F9006
:1002C0002F900C944B9362960FB6F894DEBF0FBE3E
:1002D000CDBFDF91CF911F910F91FF90EF90DF90F5
:1002E000CF90BF90AF909F908F907F906F905F90D6
:1002F0004F903F902F900895EF92FF920F931F938E
:10030000CF93DF93CDB7DEB769970FB6F894DEBF12
:100310000FBECDBF83E50E943440811103C0E6E1EA
:10032000F1E208C00E94843F6E347105C1F70E945B
:100330008DCFE4C084918F010F5F1F4F882321F080
:100340000E94198FF801F6CFEDE0F1E284918F0160
:100350000F5F1F4F882321F00E94198FF801F6CFFD
:100360008091D5059091D6050E94BDE0E0E0F1E2D4
:1003700084918F010F5F1F4F882321F00E94198FF6
:10038000F801F6CF8091D7059091D8050E94BDE085
:10039000E5EFF0E284918F010F5F1F4F882321F07A
:1003A0000E94198FF801F6CF8091D5059091D6055E
:1003B0002091D7053091D805821B930B20915405CD
:1003C000215041E050E0223010F040E050E0841B2A
:1003D000950B0E94BDE08AE00E94198FEDEEF0E2DD
:1003E00084918F010F5F1F4F882321F00E94198F86
:1003F000F801F6CF8091D9059091DA05A091DB053F
:10040000B091DC058E8B9F8BA88FB98FBE016F5F7B
:100410007F4FCE0146960E94378EE0EEF0E2849147
:100420008F010F5F1F4F882321F00E94198FF80161
:10043000F6CFCE0101967C018C01F80181918F01EC
:10044000882319F00E94198FF8CF8091DD059091D3
:10045000DE05A091DF05B091E0058E8B9F8BA88F04
:10046000B98FBE016F5F7F4FCE0146960E94378ED7
:10047000E0EDF0E284918F010F5F1F4F882321F0A0
:100480000E94198FF801F6CFF70181917F0188232F
:1004900019F00E94198FF8CF8AE00E94198FE8ECBA
:1004A000F0E284918F010F5F1F4F882321F00E949B
:1004B000198FF801F6CFE8EBF0E284918F010F5F1E
:1004C0001F4F882321F00E94198FF801F6CF20E0FA
:1004D00030E04AE754E46091E1057091E2058091D3
:1004E000E3059091E4050E94ACF442E00E94DA92A8
:1004F0008DE60E94198F8AE00E94198F69960FB6C7
:10050000F894DEBF0FBECDBFDF91CF911F910F9149
:10051000FF90EF9008958F929F92AF92BF92CF92EB
:10052000DF92EF92FF920F931F93CF93DF9300D050
:100530001F92CDB7DEB7F82E662351F01092CA078E
:100540001092C6071092C7071092C8071092C907E9
:100550000E944E628090C6079090C707A090C8077F
:10056000B090C9079B01AC01281939094A095B09F8
:1005700057FD4CC02091CA07F7FC16C04F2D0F2C19
:10058000000C550B4C5F5F4FE22F022E000CFF0B4F
:100590004E175F07DCF12F153CF044EFC42EDD242D
:1005A000D394E12CF12C06C038EEC32E33E0D32EC9
:1005B000E12CF12CDC01CB018C0D9D1DAE1DBF1D6E
:1005C0008093C6079093C707A093C807B093C90745
:1005D000022F017010E024E2209FC001219F900DA6
:1005E000901B112480599C4F9C838B8382E390E065
:1005F0009A838983BE016D5F7F4FCE0101960E9471
:1006000050B88091CA078F5F8093CA070F900F90F0
:100610000F900F90DF91CF911F910F91FF90EF906E
:10062000DF90CF90BF90AF909F908F900895AF9242
:10063000BF92CF92DF92EF920F931F93CF93DF93EE
:10064000CDB7DEB760970FB6F894DEBF0FBECDBF53
:100650005C018B010E944040E090101184E9C82E9B
:1006600081E1D82E84E0E89EF0011124EB5DFD4F7E
:100670002081318142815381F501608171818281C4
:1006800093810E94ACF4F601248535854685578513
:100690000E94D0F3F60164877587868797871D8649
:1006A0001E861F86188A80819181A281B3818983E9
:1006B0009A83AB83BC8384819581A681B7818D8326
:1006C0009E83AF83B88780859185A285B38589870E
:1006D0009A87AB87BC87AE01475F5F4FBE016B5FF8
:1006E0007F4FCE0101960E941DC1CE010D966C0177
:1006F00020EA31E1AE01475F5F4FBE016B5F7F4F84
:100700000C970E94906E0E94834130DB60960FB67A
:10071000F894DEBF0FBECDBFDF91CF911F910F9137
:10072000EF90DF90CF90BF90AF9008959F92AF92DF
:10073000BF92CF92DF92EF92FF920F931F93CF93CE
:10074000DF9387E5A82E82E0B82E04E911E1CCE41E
:10075000D4E094E2C92E94E0D92E21E3E22E24E0E5
:10076000F22E912CF50181915F010E94EB3F8823CD
:1007700009F10E94B43FF7012081211104C02091AA
:100780003504222339F0288139814A815B810E9416
:10079000D0F30AC0F3E09F1639F0F60120813181D1
:1007A000428153810E94CFF3F80160837183828379
:1007B000938309C088819981AA81BB81F8018083D4
:1007C0009183A283B38393940C5F1F4F2496F4E02C
:1007D000CF0ED11C2FEFE21AF20A84E09812C2CF9A
:1007E00086E40E9434408823C9F00E94B43F20E090
:1007F00030E0A9010E94F6F5181684F40E94B43F77
:1008000020E030E040E752E40E94ACF46093430201
:100810007093440280934502909346028091BA07F8
:1008200083FD28C08091D405882321F120915804AC
:100830003091590440915A0450915B046091A01189
:100840007091A1118091A2119091A3110E94CFF3F8
:100850002091E1053091E2054091E3055091E405D6
:100860000E94D0F36093E1057093E2058093E30565
:100870009093E405DF91CF911F910F91FF90EF903E
:10088000DF90CF90BF90AF909F9008952F923F92AE
:100890004F925F926F927F929F92AF92BF92CF9250
:1008A000DF92EF92FF920F931F93CF93DF93CDB719
:1008B000DEB764970FB6F894DEBF0FBECDBF1A0146
:1008C0002B01922EF32EC82ED12CF601E255FA4DB3
:1008D000E491AA24A3941E160CF4A12CBB24B39477
:1008E00020E030E0A901C201B1010E94F6F518161E
:1008F0000CF0B12CCC0CDD1CCC0CDD1CC601845BD7
:100900009B4F3C01FC0110821182128213820E94D3
:10091000E08DF3012082318242825382E0901011F7
:1009200020E030E0A901B801892D9F2D0E9453EFEE
:1009300081110AC0F601EF59FA4D85919591A59163
:10094000B4918C019A2EFB2EC801A92DBF2D898B45
:100950009A8BAB8BBC8B8091540490915504A091E1
:100960005604B09157044091500450915104609145
:1009700052047091530400914C0410914D04209145
:100980004E0430914F0409831A832B833C834D839B
:100990005E836F83788789879A87AB87BC871D863C
:1009A0001E861F86188AAE01475F5F4FBE016B5FD0
:1009B0007F4FCE0101960E941DC1CE010D966C01A4
:1009C0008E010F5E1F4F28E534E0AE01475F5F4F99
:1009D000BE016B5F7F4F0C970E94906EC7D9AB141E
:1009E00059F08091F705882319F01092F70504C09B
:1009F0008CE890E20E9447AE64960FB6F894DEBF92
:100A00000FBECDBFDF91CF911F910F91FF90EF905F
:100A1000DF90CF90BF90AF909F907F906F905F904E
:100A20004F903F902F900895EF92FF921F93CF9396
:100A3000DF938CEAE82E81E1F82E15E0C0E0D0E0EB
:100A400020E030E0A901F701EC0FFD1F608171810A
:100A5000828193810E9453EF81110CC02496C4318E
:100A6000D10571F7115084E1E80EF11C1111E6CFA8
:100A700080E001C081E0DF91CF911F91FF90EF9066
:100A80000895CF93909162119817C1F0C82F6ED935
:100A9000C11112C044E554E060E574E08CE494E0D8
:100AA0000E941DC180E080936211882339F08CE49C
:100AB00094E0CF910C949DCFB7DFF5CFCF910895FF
:100AC000CF92DF92EF920F931F93CF93DF93CDB727
:100AD000DEB760970FB6F894DEBF0FBECDBFE090D3
:100AE0001011ECE4F4E080859185A285B385448102
:100AF000558166817781008111812281338109834B
:100B00001A832B833C834D835E836F837887898729
:100B10009A87AB87BC871D861E861F86188AAE0102
:100B2000475F5F4FBE016B5F7F4FCE0101960E9412
:100B30001DC1CE010D966C0103E412E028E534E0FE
:100B4000AE01475F5F4FBE016B5F7F4F0C970E9406
:100B5000906E60960FB6F894DEBF0FBECDBFDF91EA
:100B6000CF911F910F91EF90DF90CF9008952F922A
:100B70003F924F925F926F927F928F929F92AF922D
:100B8000BF92CF92DF92EF92FF920F931F93CF937A
:100B9000DF93CDB7DEB72A970FB6F894DEBF0FBE4E
:100BA000CDBF2B013C012D833E834F8358874701E6
:100BB0005801DA86C9868091430290914402A0913F
:100BC0004502B091460289839A83AB83BC83D601E8
:100BD0001C9111960C91119712963C9012971396B6
:100BE0002C9020E030E0A901612F702F832D922DF1
:100BF0000E9453EF81110AC0E9E6F5E285919591D3
:100C0000A591B491182F092F3A2E2B2EA5019401EE
:100C1000609154047091550480915604909157044A
:100C20000E9453EF87FF15C0812F902FA32DB22D67
:100C30008093430290934402A0934502B0934602EE
:100C40008092540490925504A0925604B092570496
:100C500037DFE985FA85C080D180E280F38020E02B
:100C600030E0A901C701B6010E9453EF811107C00E
:100C700085E5C82EDC2C85E0E82E83E4F82EC092B2
:100C80004302D0924402E0924502F0924602409222
:100C90004C0450924D0460924E0470924F048D812A
:100CA0009E81AF81B8858093500490935104A093A6
:100CB0005204B093530404DF20915404309155043E
:100CC0004091560450915704C501B4010E9453EF5E
:100CD00087FF15C0812F902FA32DB22D8093430243
:100CE00090934402A0934502B0934602809254042C
:100CF00090925504A0925604B0925704E1DE36D883
:100D000089819A81AB81BC81809343029093440294
:100D1000A0934502B09346022A960FB6F894DEBF20
:100D20000FBECDBFDF91CF911F910F91FF90EF903C
:100D3000DF90CF90BF90AF909F908F907F906F90FB
:100D40005F904F903F902F900895CF92DF92EF9257
:100D5000FF920F931F936B01FC01E080F1800281F1
:100D60001381ECE4F4E02481358146815781608170
:100D7000718182819381FBDE1F910F91FF90EF9033
:100D8000DF90CF9008958F929F92AF92BF92EF9293
:100D9000FF920F931F93CF93DF9300D01F92CDB795
:100DA000DEB7182F80913F048770873069F48FE495
:100DB0000E943440882319F00E94A53F03C08FE4AD
:100DC0000E94EB3F8111BCC00E94B67E80E059DEDC
:100DD0008091430290914402A0914502B091460255
:100DE0008093C2079093C307A093C407B093C5072D
:100DF00080910202909103029093C1078093C007F3
:100E000084E690E0909303028093020281E0809355
:100E1000E60511111BC088E50E94EB3FF82E89E51D
:100E20000E94EB3F082F8AE50E94EB3FE82EF1106D
:100E300006C0011109C0811107C0F02E0CC00023AB
:100E400019F0F02E182F08C010E006C0FF24F3940C
:100E500001E0EE24E39411E00E94404082E50E940C
:100E60003440882361F00E94B43F4B015C0120E0D4
:100E700030E0A9010E9453EF882369F106C0812C5C
:100E8000912C80EAA82E80E4B82E111104C0F11034
:100E900002C0002389F180929C1190929D11A09232
:100EA0009E11B0929F11A50194016091540470911C
:100EB000550480915604909157040E9453EF87FF88
:100EC0000AC019821A821B821C82BE016F5F7F4F8B
:100ED0008CE991E13ADF111105C0F11003C0011155
:100EE00006C00AC080E00E94EBAC1123C1F381E090
:100EF0000E94EBAC111102C0EE2019F082E00E94BA
:100F0000EBAC5ED68091E5058093E6058091C20743
:100F10009091C307A091C407B091C5078093430285
:100F200090934402A0934502B09346028091C0077B
:100F30009091C10790930302809302020E94C77EA2
:100F40000F900F900F900F90DF91CF911F910F9105
:100F5000FF90EF90BF90AF909F908F9008952F9249
:100F60003F924F925F926F927F928F929F92AF9239
:100F7000BF92CF92DF92EF92FF920F931F93CF9386
:100F8000DF93CDB7DEB762970FB6F894DEBF0FBE22
:100F9000CDBF8DE690E054D78111DCC18091BA07B6
:100FA00083FDD8C183E50E9434408C87811106C03F
:100FB00082E50E94344089838823B1F00E94B43FC7
:100FC0000E9414F5CB010E94E2590E94B43F20E038
:100FD00030E04AEA52E40E9453EF18160CF4B5C10F
:100FE0000E941DCF21E02983EEE1F1E284918F017F
:100FF000882351F0082E000C990B0E940BA00F5F64
:101000001F4FF8018491F4CF8DE090E00E940BA077
:101010008AE090E00E940BA00E94CFD0F981FF23CC
:1010200009F498C181E080932402109247111A823A
:101030001B821C821D82188619861A861B861982BD
:101040001D862CE32E873CE13F8746E4488B312CFC
:10105000212C50E8598B8FEB8A8B812C912C5401D9
:101060006091480470914904072E000C880B990B7D
:101070000E9459EF7B018C019B01AC01632D722D05
:1010800089899A890E9453EF882359F120915C0441
:1010900030915D0440915E0450915F049C85B701DE
:1010A000802F91110CC0912F0E9453EF881F882729
:1010B000881F89833E2C2F2C098B1A8B12C0912FED
:1010C0000E9453EF87FF08C080912402E6E2F1E21C
:1010D0008491FB83EA83E5C03E2C2F2C098B1A8B6D
:1010E00019820E944E626B017C01DC01CB012885D4
:1010F00039854A855B85821B930BA40BB50BB7FD25
:1011000038C0D701C60188519C4FAF4FBF4F888769
:101110009987AA87BB870E949058EAE2F1E28491FE
:101120003F019FEF691A790A882319F082D6F301EB
:10113000F6CF81149104A104B104B9F0D501C40122
:10114000805F984DAF4FBF4FBC01CD016C197D0939
:101150008E099F0928EE33E040E050E00E9472F3D0
:10116000CA01B9010E94C09202C08FE362D68AE030
:1011700060D680E00E948EAE0E944E626093EB10BB
:101180007093EC108093ED109093EE10A0915C049E
:10119000AE83B0915D04BF8300915E0410915F0443
:1011A0000E94092D2E813F81A801632D722D89890E
:1011B0009A890E94CFF32B013C0120E030E0A90185
:1011C0000E94F6F587FF04C077FA709477F8709460
:1011D00081149104A104B10459F420E030E040E806
:1011E0005FE3C301B2010E9453EF87FF0DC00AC045
:1011F00020E030E040E450E4C301B2010E94F6F583
:10120000181614F446015701E981EE2391F12A8161
:101210003B814C815D81211531054105510541F02E
:10122000D701C601821B930BA40BB50BB7FD21C0E0
:101230002E813F81A8016D857E858F8598890E94CA
:10124000CFF320E030E040EC5FE30E9453EF87FDF6
:101250003BCFD701C601805A9541AF4FBF4F8A831C
:101260009B83AC83BD839E819D87AF81AE870F87B3
:10127000188B80912402882309F426CF81149104CD
:10128000A104B10409F4ECCEB0E1CB1AB7E2DB0A59
:10129000E108F108C818D908EA08FB08F7FE14CFDE
:1012A000DFCE882361F0082E000C990B0E940BA062
:1012B000EA81FB813196FB83EA838491F2CF8DE052
:1012C00090E00E940BA08AE090E00E940BA0809129
:1012D0006C0F8130E9F4E2E2F1E28491FB83EA836E
:1012E000882371F0082E000C990B0E940BA04A81F4
:1012F0005B814F5F5F4F5B834A83FA018491F0CF3C
:101300008DE090E00E940BA08AE090E00E940BA08C
:1013100081E08093471162960FB6F894DEBF0FBE4E
:10132000CDBFDF91CF911F910F91FF90EF90DF9094
:10133000CF90BF90AF909F908F907F906F905F9075
:101340004F903F902F900C944B930E94D6CE31E05B
:1013500039834ACE62960FB6F894DEBF0FBECDBF7A
:10136000DF91CF911F910F91FF90EF90DF90CF9081
:10137000BF90AF909F908F907F906F905F904F90B5
:101380003F902F9008959091A511E92FF0E0ED5036
:10139000FA4F80839F5F943018F49093A51102C098
:1013A0001092A5118091A6118F5F8093A6110895C8
:1013B000CF93FC0120812B33A1F02091A611243082
:1013C00080F4C62FBC018091A511F0E68F9FC0016B
:1013D000112488509A4F0E9434F78C2FD4DF81E07B
:1013E00001C080E0CF9108952F923F924F925F927B
:1013F0006F927F928F929F92AF92BF92CF92DF9225
:10140000EF92FF920F931F93CF93DF9300D000D002
:10141000CDB7DEB79A8389830E944E62E981FA8153
:10142000C680D780E084F184C114D104E104F104C2
:1014300009F0ACC22485222309F469C33285215006
:10144000248721E0230F22874585241301C01286BB
:10145000E981FA8124E0329FE00DF11D1124C68458
:10146000D784E088F188E981FA81C282D382E4825C
:10147000F582DC01CB018C0D9D1DA11DB11D868364
:101480009783A087B18784819581892B09F43FC315
:10149000FFB7FD83F894E981FA812280338021012E
:1014A000612C712C0481158180911D028F3121F0F6
:1014B0008F3F09F068C205C0E3ECFBE124912E8365
:1014C000DAC08FE180931D02E3ECFBE184918E830F
:1014D0008F3F09F458C2823009F469C030F588237F
:1014E00009F44CC0813009F0C6C0109280001092FF
:1014F00081008091810088608093810080918100CB
:10150000816080938100E0E4F6E2E491F0E0EE0F88
:10151000FF1FE351FA4D85919491E6E8F6E2E491DC
:10152000E0935208E1E0EE8330C19E81943009F4EB
:1015300082C008F460C0953009F09DC0109220016F
:101540001092210180912101886080932101809176
:101550002101816080932101E0E4F6E2E491F0E072
:10156000EE0FFF1FE351FA4D85919491E6E8F6E204
:10157000E491E0934F0895E09E8307C114BC15BC2D
:1015800084B5826084BD85B5816085BDE0E4F6E206
:10159000E491F0E0EE0FFF1FE351FA4D8591949135
:1015A000E6E8F6E2E491E09353081E82ABC21092A3
:1015B000B0001092B1008091B00082608093B000C2
:1015C0008091B10081608093B100E0E4F6E2E491A3
:1015D000F0E0EE0FFF1FE351FA4D85919491909347
:1015E000C7058093C605E6E8F6E2E491E093C805F6
:1015F000F2E0FE8387C210929000109291008091D9
:101600009100886080939100809191008160809327
:101610009100E0E4F6E2E491F0E0EE0FFF1FE35109
:10162000FA4D85919491E6E8F6E2E491E093510851
:1016300023E02E83AAC01092A0001092A1008091F6
:10164000A10088608093A1008091A10081608093B7
:10165000A100E0E4F6E2E491F0E0EE0FFF1FE351B9
:10166000FA4D85919491E6E8F6E2E491E093500812
:1016700084E08E838AC0EE81E7FD85C161E08FE161
:101680000E9461BA8E818D7F09F083C04801A12C30
:10169000B12C60E072E18AE790E0A50194010E941C
:1016A00094F329833A834B835C8369017A01F1E0E7
:1016B000CF1AD108E108F1082FEFC216D104E104D6
:1016C000F10409F008F44EC060E472E48FE090E0A9
:1016D000A50194010E9494F369017A0181E0C81A7E
:1016E000D108E108F1089E81923009F5EFEFCE169E
:1016F000D104E104F10409F008F4CBC160E970ED14
:1017000083E090E0A50194010E9494F369017A01BD
:10171000F1E0CF1AD108E108F1082FEFC216D10489
:10172000E104F10411F008F041C183E027C08FEF1C
:10173000C816D104E104F104B9F0B0F068E478EE21
:1017400081E090E0A50194010E9494F369017A017F
:1017500091E0C91AD108E108F108EE81EE2309F4FD
:101760009AC163C181E001C082E09E81911106C0EF
:1017700095B5987F892B85BD7AC085E09091B100A1
:10178000987F892B8093B10072C061E08FE10E9445
:1017900061BA4801A12CB12C60E072E18AE790E0C7
:1017A000A50194010E9494F369017A01E1E0CE1A47
:1017B000D108E108F108C114D104F1E0EF06F10409
:1017C00088F068E478EE81E090E0A50194010E9441
:1017D00094F369017A0181E0C81AD108E108F1089F
:1017E00083E001C081E09E81913071F4909181008D
:1017F000987F892B80938100452846284728D9F572
:101800002FEF3FEFA90168C0EE81E33071F49091B2
:101810009100987F892B809391004528462847287E
:1018200051F52FEF3FEFA90179C0FE81F43071F43B
:101830009091A100987F892B8093A100452846288C
:101840004728C9F42FEF3FEFA9017AC02E81253038
:1018500071F490912101987F892B80932101452873
:101860004628472841F42FEF3FEFA9017BC04528C8
:101870004628472869F0D801AA0FBB1F91010E9492
:10188000C0F328EE33E040E050E00E9472F303C062
:101890002FEF3FEFA9018E81823081F12CF4882354
:1018A00061F08130C9F06FC09E81943009F448C066
:1018B000ACF1953009F456C066C0C7BC20936408EB
:1018C00030936508409366085093670880916E00D6
:1018D000826080936E0057C0D0928900C0928800C9
:1018E0002093600830936108409362085093630826
:1018F00080916F00826080936F0045C0C092B300FA
:101900002093C9053093CA054093CB055093CC056D
:101910008091700082608093700035C0D0929900F1
:10192000C092980020935C0830935D0840935E0855
:1019300050935F088091710082608093710023C092
:10194000D092A900C092A80020935808309359085B
:1019500040935A0850935B08809172008260809394
:10196000720011C0D0922901C0922801209354081E
:101970003093550840935608509357088091730050
:10198000826080937300ED81EFBFC1C0DC01CB01A9
:101990008C199D09AE09BF09B7FDB9C04698E98108
:1019A000FA811682178210861186B1C068E478EE3B
:1019B00081E090E0A50194010E9494F369017A010D
:1019C000F1E0CF1AD108E108F1082FEFC216D104D7
:1019D000E104F10441F138F164E274EF80E090E059
:1019E000A50194010E9494F369017A01F1E0CF1AF4
:1019F000D108E108F1082FEFC216D104E104F10487
:101A000009F008F4BACE62E17AE780E090E0A5013F
:101A100094010E9494F369017A0181E0C81AD10807
:101A2000E108F10819C084E0A9CE2FEFC216D10455
:101A3000E104F10409F008F463C062E17AE780E0B0
:101A400090E0A50194010E9494F369017A01F1E00C
:101A5000CF1AD108E108F1082FEFC216D104E10432
:101A6000F104A9F0A0F089819A81AB81BC812AE0C0
:101A7000B595A795979587952A95D1F76C017D0126
:101A8000F1E0CF1AD108E108F10887E077CE86E0CF
:101A900075CE82E073CEEFEFCE16D104E104F104EF
:101AA00069F160F162E17AE780E090E0A5019401DC
:101AB0000E9494F369017A0181E0C81AD108E10813
:101AC000F1089FEFC916D104E104F104A9F0A0F0D8
:101AD00089819A81AB81BC813AE0B595A7959795AC
:101AE00087953A95D1F76C017D01E1E0CE1AD108D6
:101AF000E108F10885E03CCE84E03ACE83E038CEC0
:101B000084E033CE61E08FE10E9461BABFCD2696BA
:101B10000FB6F894DEBF0FBECDBFDF91CF911F91FE
:101B20000F91FF90EF90DF90CF90BF90AF909F907C
:101B30008F907F906F905F904F903F902F9008957F
:101B40000F931F93CF93DF9394E0899FE0011124BB
:101B50008E010C5D1B4FFE01E951FA4FDE01A850CA
:101B6000BF4E2D913D914D915C916081718182813B
:101B700093810E94D0F3F801608371838283938301
:101B8000FE01E050FD4D85919591A591B491FE0126
:101B9000EC5FFE4E80839183A283B383FE01E45FFA
:101BA000FC4D85919591A591B491C25DDD4F8883DF
:101BB0009983AA83BB83DF91CF911F910F910895E1
:101BC0000F931F93CF93DF93CDB7DEB72C970FB64C
:101BD000F894DEBF0FBECDBFECE4F4E080859185C4
:101BE000A285B38544815581668177810081118109
:101BF0002281338109831A832B833C834D835E8347
:101C00006F83788789879A87AB87BC87AE01475FE8
